:020000040800F2
:10000000782A00205DB000089DB00008FB2700089A
:10001000A1B00008A3B00008A5B0000800000000CF
:10002000000000000000000000000000A7B0000871
:10003000A9B0000800000000ABB000081587000858
:10004000AFB00008AFB00008AFB00008AFB0000814
:10005000AFB00008AFB00008AFB000086F92000862
:10006000AFB00008AFB00008AFB00008AFB00008F4
:10007000AFB00008AFB00008E38C0008AFB00008D4
:10008000AFB00008AFB00008AFB00008AFB00008D4
:10009000AFB00008AFB00008AFB000087192000820
:1000A000AFB00008AFB00008AFB00008119B000867
:1000B000159B00081B9B00081F9B00083980000847
:1000C000177E00083D8000083B800008AFB00008A4
:1000D000AFB000080F8D00085D8D0008AFB00008BC
:1000E00055770008AFB00008AFB00008DFF80CD0BB
:1000F0000BF020FC0048004799250008782A0020D2
:1001000070B51546B0FBF5F40646A84203D3204669
:10011000FFF7F6FF014605FB1460FDA2105C0870B6
:10012000481C70BD70B50C46911E232900D30A22CD
:100130000025002804DA2D212170611C404200E0D6
:100140002146FFF7DDFF0570204670BD2DE9F04721
:10015000044600E0641C20782028FBD00928F9D050
:100160004FF07E58C1B247462D2902D02B2801D02E
:1001700001E0F14F641C0026DFF8C0930CE000BFE3
:100180000BF0B4F90546494630460BF02DF92946E7
:100190000BF0D2F80646641C207830380928EFD9D5
:1001A00020782E2815D14D460EE000BF0BF09EF9A9
:1001B00029460BF04FF931460BF0BEF8064649468A
:1001C00028460BF011F9054614F8010F30380928BC
:1001D000ECD921784046652901D0452935D114F85C
:1001E000011F4FF000082D2902D02B2902D002E078
:1001F0004FF00108641C00256FF02F0206E000BFDD
:1002000005EB850302EB4303CD18641C2178A1F1B3
:100210003003092BF4D94FF49A718D4204D90D465D
:10022000C7490BF0E1F8083D082DF9D203E0494633
:100230000BF0DAF86D1E002DF9D1B8F1000F04D0E3
:10024000014630460BF006F903E0014630460BF05C
:10025000CBF83946BDE8F0470BF0C6B8F0B587B02B
:1002600000260D46B84900960196B6A70296B0F54D
:10027000000F02DB0BF060F801E00BF0AFF8B349C0
:100280000BF0B2F80BF040F9041E00DC60420A22C9
:1002900003A9FFF747FF002C01DB202000E02D2001
:1002A0008DF8000003A80AF0F8FF302401280AD0D6
:1002B00003A80AF0F2FF02280CD003A80AF0EDFF11
:1002C00003280CD00DE08DF801408DF802408DF828
:1002D000034006E08DF801408DF8024001E08DF802
:1002E000014003A968460AF0A4FF68460AF0D5FF5A
:1002F000C01EC4B22246694628460AF0B8FF2E55F1
:10030000394628460AF095FF0DEB040128460AF00D
:1003100090FF07B02846F0BD70B505460C4608684A
:100320000AF0BBFF024621682868BDE870400AF069
:10033000DDBF70B506460AF0B0FF854D10F0FF0F27
:1003400010D030460AF0EBFF0446152818DA2021B9
:1003500030460AF098FF0AF0E2FF05EB4401A1F8ED
:10036000420070BD5FF0000405EB44002146B0F888
:10037000422078A00BF00CFC641C152CF4DB70BD43
:10038000BDE87040152176A00BF002BC2DE9F041CC
:10039000002588B007462E460AF07FFF7A4C10F001
:1003A000FF0FA84651D0052278A138460AF09EFFDB
:1003B00000287DD0042277A138460AF097FF002854
:1003C00077D038460AF0ABFF461E0C2E72DA202199
:1003D00038460AF058FF070007D0781C0746FFF799
:1003E000B5FE04EB061101250861202138460AF00C
:1003F0004AFF070007D0471C3846FFF7A7FE04EB6B
:1004000006116D1C4861202138460AF03CFF0700A8
:1004100007D0471C3846FFF799FE04EB06116D1C08
:100420008861202138460AF02EFF30B1401CFFF7CA
:100430008DFE04EB06116D1CC861042D66D057A01B
:1004400001F044F808B0BDE8F08163A001F03EF887
:100450005FF0000504EB0517386910F0FF4F2BD053
:10046000761C691C67A00BF093FB03A93869FFF7A2
:10047000F5FE014665A00BF08BFB03A97869FFF739
:10048000EDFE014661A00BF083FB03A9B869FFF7FD
:10049000E5FE01465DA00BF07BFB03A9F869FFF7C1
:1004A000DDFE01465AA00BF073FB6D1C0C2D02E023
:1004B000C8E0D0E0F5E0CDDBCDF80880CDF80480D1
:1004C0000025CDF8008011E004EB0517009879694C
:1004D0000AF032FF0090B96901980AF02DFF0190EF
:1004E000F96902980AF028FF6D1C0290B542EBDB17
:1004F00049A000F0EBFF4C4E00246D4655F8240057
:1005000020F00040B04202DD48A092E0C4E08FE05D
:100510003031323334353637383941424344454639
:100520004748494A4B4C4D4E4F50515253545556E3
:100530005758595A00000000000080BF00002041B9
:1005400020BCBE4C2E0000006F12033A00007A441B
:100550002C0800206175782025752025750D0A006E
:10056000496E76616C6964204665617475726520B8
:10057000696E6465783A206D757374206265203CFD
:100580002025750D0A000000940400207265736533
:10059000740000006C6F61640000000057726F6EA1
:1005A00067206E756D626572206F66206172677577
:1005B0006D656E74732C206E656564732069647854
:1005C0002074687220726F6C6C207069746368208C
:1005D0007961770D0A000000437573746F6D206DAB
:1005E000697865723A200D0A4D6F746F720954680C
:1005F0007209526F6C6C09506974636809596177AC
:100600000D0A00002325643A090000002573090043
:1006100025730D0A0000000053616E697479206330
:100620006865636B3A0900000AD7233C4E4709000E
:10063000FDA000F04BFF641C032CFFF65FAFAFF290
:100640004000FDE60020414604EB0012401C116111
:100650000C28F9DBF6E6202138460AF014FE0028C3
:10066000F8D0401C06460AF018FEF04DC7B2002430
:1006700055F8241031B13A4630460AF037FE18B129
:10068000641CF5E7EAA0DBE6204602F081F955F8A4
:100690002410EDA00BF07CFAAFF26810FFF776FEA5
:1006A000D0E60C21EDA00BF073FACBE610B5F5A067
:1006B00000F00CFF012001F0C4F9F9A000F006FFE2
:1006C0000A2008F055F8BDE81040002008F01DB9D8
:1006D0007CB504460D4600790021062814D2DFE8D7
:1006E00000F003060A0D111EA06801780CE0A06856
:1006F00090F9001008E0A068018805E0A068B0F952
:10070000001001E0A0680168E9A00BF041FA002D9B
:1007100004D0D4E90312E7A00BF03AFA7CBDA0683C
:1007200069460068FFF79AFD0146E4A00BF030FA35
:10073000002DF3D0E0680AF0D9FE6946FFF78EFD80
:100740000146DFA00BF024FA20690AF0CFFE6946CB
:10075000FFF784FD0146DAA00BF01AFA7CBD2DE903
:10076000FF47D8A00BF014FAD0A0FFF7E2FDE14D4F
:10077000AE49687901EB800050F8041CDEA00BF054
:1007800007FA286910F0FF4F4CD0DFF878A3002457
:1007900005EB0410066916F0FF4F3FD0D0E905982D
:1007A000C769611CD8A00BF0F3F9564502D3D8A055
:1007B0000BF0EEF969463046FFF750FD0146BFA049
:1007C0000BF0E6F95646B14502D3D1A00BF0E0F9A3
:1007D00069464846FFF742FD0146B8A00BF0D8F93C
:1007E000B04502D3CAA00BF0D3F969464046FFF7E3
:1007F00035FD0146B1A00BF0CBF9B74202D3C4A03E
:100800000BF0C6F969463846FFF728FD0146AFF2FE
:1008100000200BF0BDF9641C0C2CB9DB611CBDA0E1
:100820000BF0B6F901F03EF9804E002407465C3625
:1008300056F8241021B1BCA00BF0AAF9641CF7E70C
:1008400000244FF0010800BF56F8241041B108FA07
:1008500004F0384202D0B8A00BF09AF9641CF3E718
:10086000B94A002069462C18135C94F80841401CD2
:1008700008280B55F7DB00220A54B4A00BF088F9C6
:10088000B54D002404EB840005EB800655F82010DC
:10089000B2A00BF07DF900213046FFF719FF6EA0E2
:1008A00000F014FE641C6F2CECD3BDE8FF8710B57C
:1008B000ADA000F00BFE0121002000F002FFADA072
:1008C00000F004FE0A2007F053FFBDE810400020AE
:1008D00008F01BB810B50446AAA000F0F7FDAF4819
:1008E000AF4A002101705160117001F0BFFF204636
:1008F000BDE81040DBE72DE9F04706460AF0CDFCE5
:10090000054601F0CFF8DFF8248107464FF00109D2
:1009100008F15C0855B12A46A2A130460AF0E6FC6F
:10092000C0B1307800272D2823D025E09FA000F00B
:10093000CDFD00244D46464656F8241041B105FA37
:1009400004F0384202D09EA00BF022F9641CF3E7B9
:1009500041A01EE09BA000F0B9FD00244FEA08056D
:1009600055F824100029F3D095A00BF011F9641C60
:10097000F6E70127761C6D1E5FF0000458F824107E
:1009800031B12A4630460AF0B1FC30B1641CF5E7BB
:1009900092A0BDE8F04700F099BD09FA04F01FB13C
:1009A00001F07BF894A002E000F0ECFE95A000F0CE
:1009B0008DFD58F82410BDE8F04761A00BF0E8B8B1
:1009C00010B505F04CFD401C04D091A0BDE81040CE
:1009D00000F07CBD96A0F9E770B500249EA000F061
:1009E00075FD5D4DB5F1C00504EB440005EB8001DC
:1009F0004A6855F820109EA00BF0CAF8641C102C11
:100A0000F2D370BD3EB505460AF047FC082809D16F
:100A10000024285D0AF0C0FB2855641C082CF8D37C
:100A2000002429E13EE100004F4B090020CC0008E2
:100A3000496E76616C6964206D697865722074799D
:100A400070652E2E2E0D0A004C6F616465642025A2
:100A500073206D69782E2E2E0D0A00004D6F746F75
:100A600072206E756D626572206D7573742062659B
:100A7000206265747765656E203120616E64202583
:100A8000640D0A00526573657474696E6720746F33
:100A90002064656661756C74732E2E2E0D0A00003D
:100AA0005265626F6F74696E672E2E2E0000000013
:100AB00025640000202564202564000025730000C3
:100AC0002025730043757272656E7420436F6E66E5
:100AD00069673A20436F707920657665727974682A
:100AE000696E672062656C6F7720686572652E2E6F
:100AF0002E0D0A00940400206D697865722025731C
:100B00000D0A000000008080636D69782025640074
:100B100020000000636D697820256420302030209B
:100B20003020300D0A000000666561747572652022
:100B30002D25730D0A0000006665617475726520CD
:100B400025730D0A0000000064D600086D61702056
:100B500025730D0A00000000B8CD000873657420ED
:100B60002573203D20000000536176696E672E2EAC
:100B70002E0000000D0A5265626F6F74696E672E59
:100B80002E2E00000D0A4C656176696E6720434C7D
:100B900049206D6F64652E2E2E0D0A00640400201E
:100BA000000000206C69737400000000456E6162F3
:100BB0006C65642066656174757265733A20000027
:100BC00025732000417661696C61626C6520666501
:100BD0006174757265733A2000000000496E766199
:100BE0006C69642066656174757265206E616D65FF
:100BF0002E2E2E0D0A00000044697361626C65643C
:100C000020000000456E61626C65642000000000F9
:100C1000456E61626C696E67204750532070617346
:100C2000737468726F7567682E2E2E0D0A000000AF
:100C30004572726F723A20456E61626C6520616E1A
:100C40006420706C756720696E2047505320666978
:100C50007273740D0A000000417661696C61626C08
:100C60006520636F6D6D616E64733A0D0A0000005C
:100C700025730925730D0A00295DFC480AF003FB62
:100C800028B12819295D401C0AF0FDFA18B1F8A016
:100C900000F01CFC3EBD641C082CFFF4C2AE2846CC
:100CA00000F052FCFAA000F011FCF04BFE4A0020CC
:100CB000694615181C5C95F80851401C08284C55CD
:100CC000F7D300220A54AFF288100AF061FF3EBD4C
:100CD0002DE9F04180460AF0E0FAF34FF34D0600AB
:100CE00012D00246AFF2441140460AF0FFFA90B12A
:100CF0005FF0000455F82410F1B1324640460AF086
:100D0000F5FAF8B1641CF5E7787905EB800050F846
:100D1000041CE7A01BE0EBA000F0D8FB5FF0000490
:100D200055F8241029B1AFF268100AF031FF641CA5
:100D3000F6E7AFF2DC2001E0AFF20C30BDE8F041A5
:100D400000F0C4BB601C787155F82410E2A0BDE827
:100D5000F0410AF01DBF2DE9F041002507462C4661
:100D60002E460AF09AFA18B1AFF25C21384610E02C
:100D7000DEA02BE016B1012E07D103E00AF0CFFA76
:100D8000054602E00AF0CBFA0446761CAFF2802159
:100D900000200AF089FA0028ECD10C2D05D3BDE81B
:100DA000F0410C21E0A00AF0F3BEE94F022E07DA71
:100DB00037F915202946BDE8F041E6A00AF0E8BE63
:100DC000A4F57A70B0F57A7F04D9E8A0BDE8F041C7
:100DD0000AF0DEBE22462946EDA00AF0D9FE27F829
:100DE0001540BDE8F08170B505460AF056FAAE4CE4
:100DF00010F0FF0F0CD028460AF091FA02280ED806
:100E000084F894030021084600F05BFCA5A0EBE702
:100E100094F89413BDE87040E4A00AF0B9BE70BD28
:100E20002DE9F04782460AF038FAE64D060029D04F
:100E3000012E03D19AF800002A2823D0E2A15046BF
:100E40000AF003FA002871D0401C04460AF067FA41
:100E500081462046FFF77AF98046002606EB860792
:100E600005EB870455F827000AF017FA024655F8F3
:100E7000271050460AF03AFAF8B1761C6F2EEDD3DF
:100E8000D2A04FE0D9A000F021FB002404EB8400A5
:100E900005EB800755F82010AFF23C300AF078FEE1
:100EA00031463846FFF714FCAFF2544000F00EFB19
:100EB000641C6F2CEAD3BDE8F08706EB860605EBD1
:100EC0008607F8680AF012FB41460AF04BFB26D869
:100ED00038690AF00BFB41460AF04EFB1FD83979FE
:100EE000052907D0484606290ED2DFE801F005059E
:100EF00008080B0B4046F6E7A168087004E0A168FB
:100F0000088001E0A168086055F82610BDA00AF02D
:100F10003FFE2046BDE8F0470021FFF7D9BB00E0C7
:100F200004E0BBA0BDE8F04700F0D0BA5FF00004D9
:100F300004EB8406514655F826000AF086F978B18C
:100F400055F8261005EB8607AFF2EC300AF020FECC
:100F500000213846FFF7BCFBAFF204500AF018FE40
:100F6000641C6F2CE4D3A6E72DE9F04107F0F1FBF8
:100F70004FF47A71B0FBF1F1AF480378AF480278D3
:100F8000AFA00AF005FE00F07DFD0646BC48BD4955
:100F90000068B0FBF1F1BCA00AF0FAFD434F002459
:100FA00001259C3757F8241051B105FA04F030425E
:100FB00003D0AFF2F4300AF0EBFD641CE4B2F1E7C9
:100FC000022000F04DFDA0B1B74C38482178BC306C
:100FD00050F82110B5A00AF0DBFD2078022808D1D6
:100FE000B548007C08B16F2100E06E21B3A00AF083
:100FF000CFFDAFF29C5000F069FA07F098F8024676
:10100000AF484FF466730188BDE8F041ADA00AF027
:10101000BFBDB9A000F05ABA2DE9FF5FDFF8089311
:1010200099F8000038B9012189F80010BFA000F03C
:101030004DFA00F057FADFF82CB3DFF87CA25446E3
:10104000DAF8000009F03CF800280CD0206809F01C
:101050003AF8092808D03F2806D0D9F804104C46A1
:10106000002902D0D1E12FE27EE1CCE164D6000874
:101070004D75737420626520616E79206F726465AE
:1010800072206F662041455452313233340D0A00CC
:1010900043757272656E742061737369676E6D65F6
:1010A0006E743A20000000009404002020CC000858
:1010B00043757272656E74206D697865723A202589
:1010C000730D0A00417661696C61626C65206D691F
:1010D000786572733A2000004D69786572207365F7
:1010E0007420746F2025730D0A000000557361672A
:1010F000653A0D0A6D6F746F7220696E64657820B1
:101100005B76616C75655D202D2073686F77205B61
:101110006F72207365745D206D6F746F72207661DD
:101120006C75650D0A0000004E6F207375636820B2
:101130006D6F746F722C207573652061206E756DF4
:10114000626572205B302C2025645D0D0A00000072
:10115000540900204D6F746F72202564206973203C
:101160007365742061742025640D0A00496E7661F0
:101170006C6964206D6F746F722076616C75652C7C
:1011800020313030302E2E323030300D0A00000049
:1011900053657474696E67206D6F746F7220256477
:1011A00020746F2025640D0A0000000043757272E0
:1011B000656E742070726F66696C653A2025640DE7
:1011C0000A000000B8CD00083D0000004552523A28
:1011D00020556E6B6E6F776E207661726961626CFE
:1011E00065206E616D650D0A000000004375727226
:1011F000656E742073657474696E67733A200D0AA6
:101200000000000025732073657420746F200000B7
:101210004552523A2056616C756520617373696757
:101220006E6D656E74206F7574206F662072616ECE
:1012300067650D0A0000000068010020DA00002048
:1012400053797374656D20557074696D653A202506
:1012500064207365636F6E64732C20566F6C7461C9
:1012600067653A202564202A20302E315620282513
:1012700064532062617474657279290D0A0000005C
:101280002C04002040420F004350552025644D4857
:101290007A2C2064657465637465642073656E736D
:1012A0006F72733A200000007C01002041434348E4
:1012B000573A202573000000280900202E256300DE
:1012C000DC0000204379636C652054696D653A2029
:1012D00025642C20493243204572726F72733A2084
:1012E00025642C20636F6E6669672073697A653A9E
:1012F0002025640D0A0000004166726F33322043DE
:101300004C492076657273696F6E20322E3220410F
:1013100070722033302032303134202F2030303A78
:1013200033323A3334000000000000200D0A456ECD
:10133000746572696E6720434C49204D6F64652C5B
:1013400020747970652027657869742720746F2070
:1013500072657475726E2C206F72202768656C70D0
:10136000270D0A0064040020624F0024254607F17F
:10137000C008D9F804600BE0D9F8042022B15E4817
:10138000396809F0B3FF10B904B93C463D460C3743
:101390004745F1D39CB149465F46486822682B68AF
:1013A000125C1B5C9A420AD19AB92E2811D22022D3
:1013B0003A54401C0021C9F804000BF80010D9F879
:1013C00004004F4608B1AC4213D04CA000F07EF8A8
:1013D0000AE03A54401C4860DFE7206800F076F8E5
:1013E000092000F081F80C34AC42F6D900F07AF80C
:1013F00000265C4678688642BFF421AEA05D00F00E
:1014000073F8761CF6E7042812D00C2816D019B110
:101410000A2817D00D2815D07F283FD03029EBD2CD
:101420002028FFF40CAE7E283FF609AEA9B343E0B6
:1014300004B03148BDE8F05FFFF74CBA31A000F0CE
:1014400045F827E0AFF6F01000F040F8606800259E
:101450005E460BF800502E48CDE9000B0C231022FD
:101460002449029501A809F09DFE070007D03868BD
:1014700009F013FF3044B968401C884702E025A0FA
:1014800000F024F830211C4809F0C8FE656020787F
:10149000002819D000F026F8D1E50BE00029FBD098
:1014A000491E0020C9F804100BF8010022A000F02A
:1014B0000DF8C4E52028EFD00BF80100491CC9F84D
:1014C000041000F011F8BAE5BDE8FF9F70B50446BE
:1014D0001A4D03E0641C286808F0E2FD2178002919
:1014E000F8D170BD16A0F1E701461448006808F075
:1014F000D7BD0000F8CC0008640400200D1B5B4B36
:10150000000000001B5B324A1B5B313B314800008E
:10151000190300084552523A20556E6B6E6F776E74
:1015200020636F6D6D616E642C2074727920276862
:10153000656C7027000000000820080028090020C2
:101540000D0A2320000000002DE9F0410546044665
:10155000FD4EFE4F09E0FC4809F095FE20B1611BED
:10156000801B384480F80811641C21780029F2D1CE
:10157000BDE8F081F648002102783F2A12D1428866
:10158000B2F5667F0ED10279BE2A0BD190F8962370
:10159000EF2A07D100F5667210F8013B59409042DE
:1015A000FAD309B1002070470120704710B5FFF74A
:1015B000E1FF10B90A2007F087F94FF46672E44999
:1015C000E24809F012FEE14890F89413022902D98A
:1015D000002180F89413C9B201EB011101EB410124
:1015E00000EB8101BDE8104001F59871CC22D9488B
:1015F00009F0FBBD2DE9F05FD64AD74E002092F8E6
:101600002010D47F40F6C41500FB00F3193B4B4378
:1016100003F6C4134343634393FBF5F326F81030FA
:10162000401CC0B20728EFD3C84B9146D03392F884
:10163000212099F8224059881F880020DFF81CA338
:101640004FF00A0B4FF47A7EC4F1640802EB820C6F
:10165000B1EB070500EB8001C2EB41030121002B38
:1016600003DDC2F16401C9B201E000DA114603FBF7
:1016700003F604FB06F601FB01F196FBF1F1414490
:1016800001FB03F191FBFBF101EB4C0109B205FBFE
:1016900001F191FBFEF139442AF8101000F101002C
:1016A000C0B20C28D6D399F8000002F01FF9BDE8AB
:1016B000F05F03F0A7BF10B5FFF778FFBDE810405B
:1016C00098E72DE9F047A14D81463F2028704FF45F
:1016D000667400276C80BE202871EF2085F8960381
:1016E0003E4685F8977369B195F89403CC2200EBD8
:1016F000001000EB400005EB800000F59870954964
:1017000009F073FD9148934903E000BF10F8012BE5
:1017100057408842FAD385F897738D4F4FEA0408F3
:1017200009F024FC342009F08FFC384609F04CFC09
:1017300004280FD10024E019295909F061FC04287C
:1017400005D009F019FC761C032EE9DB02E0241D0C
:101750004445F0D309F010FC032E02D0FFF70AFF36
:1017600010B90A2007F0B0F8FFF7A5FFB9F1000F94
:1017700006D0BDE8F047012214210F2001F094BCEF
:10178000BDE8F08771498A6802438A6070472DE995
:10179000FC5F73A1D1E90001CDE900014FF466714E
:1017A0006A4809F03BFDCC216A4809F037FD674BD8
:1017B0003F20002518700320587102209D60FFF71C
:1017C000E1FF83F894534FF41670A3F8F000FA2069
:1017D000A3F8F200D0332A20D8831D855D859D852E
:1017E0009D74DD741D75DD821D835D831C334FF494
:1017F000FA705D70588101261E70202018726E20CC
:1018000018762B20587621209876DD7683F82450A0
:1018100083F83E5083F83F50263340F2DC529D76E9
:101820001A8040F24C405880423B40F26C70A3F862
:10183000460083F8485083F8495083F84A6040F2E4
:101840007E40188040F23A7058804FF47A70988049
:1018500040F27E50D88040F2EA50188140F2B450F5
:10186000588132209881C100D981188283F84C5068
:1018700083F84D504FF4E13119654FF41651596515
:1018800083F8585083F8595040F6AC5123F8C41CE3
:1018900003F8C25C2F4C83F84B50282725706770E3
:1018A0004FF01E0A84F80BA017216175A77084F809
:1018B0000CA0A1755521E1702D216173E575207192
:1018C000A57325760B216171E57365764FF0140BD6
:1018D00084F806B0082323742D23A3760E23E37126
:1018E00084F811B05021E1765A2121724FF00A0894
:1018F00084F812804FF0640984F81C906772782392
:10190000A3722D232375A677E177412184F8201057
:1019100084F8235084F8245084F82550E28484F815
:10192000210084F822506585A5852585042084F84A
:101930002E0084F82F7084F83070152084F8310060
:1019400009486063094813E064D600089404002045
:1019500000F801082C0800200A0B0020180B0020BA
:101960001E1E6464646464649A99193FF6287C3F7F
:10197000A0634E48E06384F840604DA0FFF7E4FDAB
:1019800084F86C5084F86D5084F86E7084F86F6041
:1019900084F872504FF44870A4F8700004F8B48FC3
:1019A000C82363704FF49660608040F2D930A08005
:1019B000424800216C4640F2DC554FF47F764FF4EC
:1019C000FA6C00BF00EBC10222F8746FA2F802C0EB
:1019D000958014F80180491C82F806800829F1DB03
:1019E000012100F8BA1F364D41708170838080F864
:1019F00006B080F807A00172A0F80A904FF4967123
:101A00008181C781522085F8950300204FEA0001AB
:101A100005EB0012401C11610C28F9DB5FF000049B
:101A200004EB041000EB400005EB800000F598701B
:101A3000CC22224909F0D9FB641C032CF0DBBDE861
:101A4000FC9F10B50446FFF795FD641E204206D1A9
:101A5000FFF79DFE0021BDE81040084631E610BDAD
:101A600018490968014201D00120704700207047E1
:101A700014490A6802430A60704712490A6882439F
:101A80000A6070470F48006870470D498968014235
:101A900001D0012070470020704709498A688243BD
:101AA0008A60704706488068704700003D0A773FAB
:101AB0004145545231323334000000002C080020DC
:101AC000940400200800002070B5FE480AF0E6FBF0
:101AD000FD4D0446288809F012FD214609F084FCDA
:101AE0000AF09CFCF94C2080288809F008FD01468A
:101AF000F74809F0AFFCF74909F0ACFCE065F6489F
:101B0000B0F8700009F0FBFC0146F44809F0A2FCB3
:101B1000F34909F069FC20660820FFF7A1FF0028BF
:101B200003D0BDE8704002F075BE70BD002801DD35
:101B3000024600E042428A4201DA00207047002853
:101B400002DDA0EB01007047FDDA084470472DE983
:101B5000F04F91B0D0E90045814686688846086814
:101B60000AF09CFB0490D8F800000AF07DFF059075
:101B7000D8F804000AF092FB0190D8F804000AF0AB
:101B800073FF0746D8F808000AF088FB8246D8F8A9
:101B900008000AF069FF83465046049909F024FCC6
:101BA00007905046019909F01FFC80465846049959
:101BB00009F01AFC06905146059809F015FC0890AA
:101BC0005946059809F010FC03900198594680F099
:101BD000004009F009FC82463946089809F004FCE7
:101BE000069909F0A9FB10903946039809F0FCFB0F
:101BF000079909F0F6FB0E900598019980F00040D6
:101C000009F0F2FB05903946079809F0EDFB0399BE
:101C100009F0E7FB02903946069809F0E5FB0899C0
:101C200009F08AFB83460499019809F0DDFB0490D2
:101C30003046029909F0D8FB01902846109909F026
:101C4000D3FB00904146204609F0CEFB009909F0F5
:101C500073FB019909F070FBC9F800005946304642
:101C600009F0C2FB834628460E9909F0BDFB804669
:101C70005146204609F0B8FB414609F05DFB594644
:101C800009F05AFBC9F804003046049909F0ACFB8E
:101C900006462846059909F0A7FB05463946204621
:101CA00009F0A2FB294609F047FB314609F044FB45
:101CB000C9F8080011B0BDE8F08F2DE9F043804667
:101CC000824887B08430016881F000410391406808
:101CD00080F0004004908348B0F9000009F006FC51
:101CE000814909F081FB794C05907634B4F9000004
:101CF00009F0FCFB0090B4F9020009F0F7FB019039
:101D0000B4F9040009F0F2FB029003A96846FFF75A
:101D10001EFF714E763C96F84000012804D06A48B8
:101D2000008809F0ECFB17E0704840780028E06A72
:101D30000CD1C11700EB9161A0EBA11009F0D6FB0B
:101D4000029909F0F9FA09F0DFFBE062C11700EB34
:101D50009160801109F0CAFB029909F042FB0290E0
:101D6000216B894609F03AFB0746404609F0C7FB5C
:101D700005465F4909F0E0FA0146284609F06AFB8A
:101D8000394609F031FB494609F0D6FA206300983C
:101D90000AF044FB2F367178FFF7C8FE554D2968CD
:101DA0000844286001980AF039FB7178FFF7BEFEFD
:101DB000696808446860206B0AF030FB3178FFF7EF
:101DC000B5FEA9680844A860A16801EB0800A060FE
:101DD000E068401CE06007B0BDE8F0832DE9F05FEB
:101DE0003A4D0446843528680AF058FA8346286834
:101DF0000AF03AFE824668680AF050FA814668683E
:101E00000AF032FE0546D4F808802946404609F01B
:101E1000EBFA594609F0E8FA676806465146384633
:101E200009F0E2FA294609F0DFFA0546494620683A
:101E300009F0DAFA294609F07FFA314609F07CFA0E
:101E400004465146404609F0CFFA05465946384601
:101E500009F0CAFA294609F0C1FA21460AF0F4F855
:101E6000254909F0C1FA254909F0F4FA1749496AE8
:101E700009F062FA224909F0EDFA0AF0CFFA00B24D
:101E8000002802DA00F5B47000B2BDE8F09F2DE939
:101E9000F041044680680D46014609F0A5FA074660
:101EA0006068014609F0A0FA06462068014609F07C
:101EB0009BFA314609F040FA394609F03DFA0AF03A
:101EC00099FE1FE0F366DF3E820100200C00002037
:101ED0000AE81C4100401C462C0800200000614418
:101EE0004C3D0F44B001002035FA8EBCD40A0020CE
:101EF0003661823C100900200000E144DB0F4940BC
:101F000000002041064610F0FF4F0ED031462068F9
:101F100009F0A0FA28603146606809F09BFA686011
:101F20003146A06809F096FAA860BDE8F0812DE975
:101F3000F04F87B0002606F0F2FBFF4C0546606BC1
:101F4000281A039009F0DBFAFC49C96809F04CFA39
:101F50000590FB486563DFF8E0A390F82E700AF166
:101F6000700A0024EB460AF106054FF07E58F2484D
:101F70006A3030F9140009F0B9FA059909F034FA19
:101F80004BF8240017B3384609F0B9FA0146404629
:101F900009F060FA814604903AF9140009F0A6FAB3
:101FA000494609F021FA81464146049809F019FA98
:101FB000E44951F8241009F017FA494609F0BCF930
:101FC000E04941F8240009F09FFA01E03AF81400D2
:101FD00025F8140035F91400641C00FB0066032C7E
:101FE000C5DB64204643D84869460088404396FBD9
:101FF000F0F4D4481830FFF7AAFD0820FFF730FDB1
:10200000694620B1CF480C38FFF7A1FD08E0CA4867
:102010008C30FFF79CFDC8498C310846FFF737FF2D
:10202000A0B2DFF820934938DFF820A309F118099E
:102030003C2826D20024AB46BAF8F00009F05FFA3B
:1020400045464146049009F077F90146284609F0D3
:1020500001FA05464FEA09063BF9140009F046FA71
:10206000074656F82410049809F0BEF9394609F0DD
:1020700063F9294609F0B8F946F82400641C032CDA
:10208000EADB0820FFF7ECFC48B34546AD4EDFF82D
:10209000A88200240C3E08F17C08BAF8F20009F08E
:1020A0002EFA8246294609F047F90146284609F0EA
:1020B000D1F9054638F9140009F018FA07465046D8
:1020C00056F8241009F090F9394609F035F92946F7
:1020D00009F08AF946F82400641C032CEADB964DCB
:1020E000B5F9000009F002FA4C46D9F8081009F0D9
:1020F00039FA01D2012100E0002195484173D4E969
:10210000010109F0A1FF8C4E84363060A0680146C1
:1021100009F06AF907466068014609F065F9394631
:1021200009F00AF90AF066FD0146206880F00040D7
:1021300009F08AFFDFF81C8270604146306809F0C0
:1021400053F90AF06BF9A6F15C07414638807068D4
:1021500009F04AF90AF062F978800820FFF780FC5C
:102160007D4E10B177480C3801E073488C30FFF792
:1021700035FE30800398FFF7A0FD714E96F872008F
:1021800000283CD0A068014609F02EF9804660681E
:10219000014609F029F907462068014609F024F9AB
:1021A000394609F0C9F8414609F0C6F80AF022FD9F
:1021B0000146A06809F04EF96849884201DC002018
:1021C0001CE009F0B1FE296E09F00EF90AF026F9BB
:1021D0004FF46171884200DD084609F087F96049D3
:1021E00009F038F90AF040FC044696F8720009F04C
:1021F00086F9214609F0F8F80AF010F9688007B06E
:1022000059E510B502F0FDFA0220FFF729FC20B1D4
:1022100002F0F9F9FFF78BFE05E047490020703125
:102220000880488088804948434940796A318A1F3C
:10223000012809D05FF0000031F8103022F810308A
:10224000401C0328F8D310BD3B4BB1F90400B3F98F
:10225000044000EB4400032490FBF4F0908098804D
:10226000088810804888508010BD364900200C3105
:102270000860486088603049C860886070472DE910
:10228000FC5F06F04CFA2C4C46F2A812A16BA0EBB6
:102290000108904502D20020BDE8FC9F314FA063A9
:1022A000274D3888DFF8C090DFF8C0A0DFF8C0B055
:1022B0004FF07E5640B3206D2269C11700EB51717B
:1022C000A0EBE10095F83110491EB2FBF1F1084492
:1022D000C117206500EB5170C01009F007F949469D
:1022E00009F0B8F851460AF0B1F8314609F079F82A
:1022F000594609F079F809F007F9E06400202064F4
:1023000060643888401E388095F831002169401E8D
:10231000B1FBF0F009F0F3F8494609F09BF851469B
:102320000AF094F84FF07E5109F05BF8594609F035
:102330005BF80AF073F81DE00C000020B80C0020D8
:102340002C080020040900208201002094040020B1
:10235000D40A00204C3D0F44B00100208FC2753CD0
:10236000EFB6B044AE01002080E6C547B1DC423E86
:10237000D048874AE16C6F6B461A39464FF07E5061
:1023800009F02CF88146304609F0B0F8494609F0CA
:102390002BF80646606909F0A9F8394609F024F8D7
:1023A000314608F0C9FF0AF039F860610190A06871
:1023B00009F0A5F807466E4909F016F80646E068E8
:1023C00009F094F881466B48806809F08FF8494617
:1023D00009F040F88146E16D09F006F8394609F048
:1023E00003F80746206C3146009008F0FDFF824656
:1023F0004FF0FF31384609F06DF8314608F0F4FF30
:10240000514608F099FF616C08F096FFD5F83CA0A2
:10241000834651464FF07E5008F0E0FF0646019893
:1024200009F064F8314608F0DFFF06465146584689
:1024300008F0DAFF314608F07FFF606409F064F8C5
:1024400060653946009808F077FF2064FFF70DFFBC
:10245000404609F054F806466769A06C381A09F03E
:1024600045F8454908F0C0FF314608F0F3FF09F090
:102470004BF84FF49678C8F1000A42465146A764DB
:1024800004F044FA0A21FFF751FBAF6B834639464B
:102490004FF07E5008F0A2FF0646584609F026F895
:1024A000314608F0A1FF06463946206C08F09CFF33
:1024B000314608F041FF206409F0B0FF06460521CF
:1024C000FFF734FB2062D4E91510401A4FF4FA727A
:1024D000514204F01BFA0A21FFF728FB0146287934
:1024E00042464843C11700EB5160C011514604F009
:1024F0000DFA861BA87A42467043C11700EBD160E3
:102500004011514604F002FAA061287D4FF4483290
:102510007043C11700EB5170E16901EBE0005142DB
:10252000E06104F0F3F9C117E06100EB9150A1699B
:1025300001EBA020A0614846E16B08F0FDFE0646D5
:10254000A87F08F0DCFF314608F04EFF6FF0050170
:1025500008F0C0FF08F0D8FF96226FF0950104F054
:10256000D5F9A169C4F83C90081AA061012093E64E
:10257000BD378635100900200024744970B5A24D7E
:102580000446286807F0A5FD0028FAD0E1B22868C3
:1025900007F086FD204670BD86B00020FFF751FA97
:1025A000FFF704F8994CA07B00B1012006F000F978
:1025B000FFF720F894F80701002518B101281DD075
:1025C00009281BD08DF8145084F8075105A804F091
:1025D0007FFF04F0A3F90E20FFF74AFA00F05DF93F
:1025E000607901260E280CD008280AD08DF80650F4
:1025F0004FF48070FFF749FA50B905E08DF81400E8
:10260000E4E78DF80660F3E70820FFF73EFA00B133
:1026100001208DF802004020FFF737FA8DF8030003
:102620000120FFF732FA8DF801000820FFF72DFA9C
:10263000DFF8D48180F001008DF80000744F98F825
:1026400012008DF8040097F8BC004FF47A7AC0F3BA
:1026500080008DF80500B4F8DE00ADF80800B4F88D
:10266000E000ADF80A00ADF80CA04FF48040FFF791
:102670000CFA18B1B4F8DA00ADF80C00BDF8080097
:10268000B0F5FA7F01D9ADF80C50B4F81201ADF8ED
:102690000E00B7F8B800ADF8100094F80701012853
:1026A00024D0092825D08DF80750684605F026FF6C
:1026B000584A002040F2DE5122F81010401CC0B2EF
:1026C0001228F9D3554954480827086088F8117032
:1026D0003846FFF7DAF9E0B194F8100168B1012843
:1026E0000BD002280DD0032817D10EE08DF807601B
:1026F000DBE707208DF80700D7E7484803F0CAFF5B
:102700000BE0464804F076FA07E0444804F00EFB7C
:1027100003E094F81D0102F0BEFF0120FFF7B5F9B8
:1027200030B14FF48060FFF7B0F908B102F0F6F86D
:102730003B494FF01009C1F80090A1F10408C8F816
:1027400000700025A8F1040BDBF8001081F01001E7
:10275000CBF80010DBF8001081F00801CBF8001076
:10276000192006F005F8012006F00DF8192005F0F3
:10277000FFFF002006F007F86D1CEDB20A2DE3D331
:10278000C8F80070C8F8009001F080FDFFF79CF9D0
:102790000220FFF77AF908B101F044FED4F82001D5
:1027A00002F0EDF94020FFF770F948B194F82811D4
:1027B000D4F8240107F09DFB94F8290107F0ACFB45
:1027C0004FF40060FFF761F908B104F025FD05F052
:1027D000A6FF144908606079052803D112494FF417
:1027E000C87008801149C820A1F800A010490880CD
:1027F0001048467301F082F8FCE70448B0F9D400B1
:1028000000F051F9FEE700002809002094040020A0
:102810002C080020E60A0020833400080401002070
:10282000140C0140000100207E01002080010020E6
:10283000AE010020D40A00200146F74800EBC10099
:10284000B0F97800122804DA082902DAF34931F9DC
:1028500010007047F04A02EBC00090F97A0008427D
:1028600002D04FF0FF307047012070472DE9F04152
:10287000EB4DEC4E00244FF480473846FFF705F946
:1028800010B1B5F8DA0001E0B5F8D40026F814006C
:10289000641C0C2CF1DBBDE8F0812DE9F047E04C25
:1028A000E14E607906EBC000407800B10120DF4DB9
:1028B000A8742020FFF7E9F84FF0010A08B185F865
:1028C00012A06079DFF85C93D94D09F11809162838
:1028D00008D016F8301006EBC0002970426842B3E9
:1028E000002024E00020CC4604EB00110A6912F01D
:1028F000FF4F1ED0D1E905670CEB0013C969401CDE
:10290000C3E90271C3E900262978491C29700C2803
:10291000EADB0EE002EB001609EB0013D6E9007CBF
:10292000D6E90286C3E90286C3E9007C401C8842DE
:10293000F0DB4FF48040FFF7A8F8D8B12F78012FD3
:1029400018D9002614E000BF09EB06154FF0FF3838
:102950004146A86808F0BEFDA8604146686808F0D6
:10296000B9FD68604146E86808F0B4FD761CE8608F
:10297000BE42E9DB6179AF48082906D00E2904D0B0
:1029800000210174BDE8F04770E780F810A0F9E776
:10299000F0B5401C0021A24A0B4600BF02EB011417
:1029A000491C23610C29F9DB9F4B03EBC0014C68E8
:1029B000002C11D0002113F830000BE004EB0113C0
:1029C00002EB011593E8C010DB68491CC5E906C39A
:1029D000C5E904678842F1DCF0BD944810B5807CFD
:1029E00000284DD0924C8E48241D4279E0882189E0
:1029F000082A27D006DC012A15D0042A29D0052A66
:102A000006D10AE00E2A29D0142A22D0152A25D070
:102A10002020FFF73AF8002832D02188002005F066
:102A200004FE618813E082497B48091D90F8BB00D1
:102A3000498908B100201FE07E4840780028F9D17C
:102A40000021F7E70146002005F0EFFD2189012074
:102A500012E0002005F0E9FD6189F8E70146002059
:102A600005F0E3FD2189012005F0DFFD61890220E9
:102A700005F0DBFDA1890320BDE8104005F0D5BDC0
:102A800010BD70B5674E0024183E694D07E000BFC9
:102A900036F81410204605F0C1FD641CE4B2287815
:102AA0008442F5D370BD624A5E4B00211278183B18
:102AB00004E000BF23F81100491CC9B29142F9D3C8
:102AC000DFE72DE9F047DFF86C91594C002599F8C4
:102AD0000100594F524E241D48B3B6F8D220B6F823
:102AE000D010B7F9060003F011FF4E49E081183904
:102AF000B046088096F81901474E4FF0640A48B373
:102B00000220FFF799FEB6F98620B6F9841003F08B
:102B1000FDFEB8F81231181A0FFA80FC4448B0F9DB
:102B20000220624506DA98F81911114407E0B6F858
:102B3000D400DAE704DD98F81911A2EB0101418015
:102B400096F98A10B0F9020001FB00F191FBFAF04E
:102B50001844A08099F80A0050B1388800EB0501AC
:102B6000E18000EB25402081B888608178880AE008
:102B70003248018801EB0502E28001EB2541218109
:102B8000818861814088A0814FF003024FEA0A03E7
:102B900006EBC20034F9121090F97A0000FB01F044
:102BA00090FBF3F024F812001046FFF745FE34F8CE
:102BB0001210084424F81200521C072AE8DBBDE872
:102BC000F0872DE9FC5F1A4C1B4F1C4D2078032821
:102BD00014D9B7F904004142002801DD024600E0A3
:102BE0000A4602F1640200DC08466FF06301A1EBC3
:102BF0000001B5F9040003F089FEA8800C48DFF855
:102C00002490DFF814A00078A9F1180901284DD903
:102C10000024804648E000002C080020E60A00203E
:102C20009404002054090020E0DA0008280900205C
:102C3000B8000020D40A0020440100203601002002
:102C40009AF9BA00B5F904104042484308F04EFC26
:102C5000FE4901EB0416F16808F0C6FB0190B5F9D6
:102C6000000008F043FC716808F0BEFB0090B5F965
:102C7000020008F03BFCB16808F0B6FB8346B7F9E8
:102C8000060008F033FC316808F0AEFB594608F046
:102C900053FB009908F050FB019908F04DFB08F038
:102CA00033FC29F81400641C4445C9D3E84EDFF80E
:102CB000A483E94C70794FF0320B082868D006DC09
:102CC000012837D0042809D0052840D140E00E283B
:102CD0005BD014287DD01528F7D1D8E00420FFF769
:102CE000ABFD074602210420FFF7B4FDB5F904103F
:102CF00000FB01F301210420FFF7ACFDB5F9021040
:102D000000FB0130384420810520FFF795FD074680
:102D100002210520FFF79EFDB5F9041000FB01F329
:102D200001210520FFF796FDB5F9021000FB0130E7
:102D300038440BE00520FFF77FFD03460121052005
:102D4000FFF788FDB5F9041000FB01306081C5E094
:102D50009AF97A00B8F902105D46484390FBF5F7FE
:102D60000AF17A0243460020FFF766FD38442080CE
:102D700092F90800B3F90010484390FBF5F20120E6
:102D8000FFF75AFD10446080A8E0FFF79AFEA5E027
:102D9000B248407890B3B6F8D220B6F8D010B7F960
:102DA000060003F0B3FDE081A9F80000AB484FF046
:102DB0000101807A00284FF0030023D0FFF74AFD7D
:102DC000B7F9021000FB01F302210320FFF742FDD7
:102DD00000E044E0B7F9001000FB0130E080012181
:102DE0000420FFF737FDB7F9021000FB01F30221C1
:102DF0000420FFF72FFDB7F9001020E0FFE7B6F839
:102E0000D400D0E7FFF726FDB5F9021000FB01F36F
:102E100002210320FFF71EFDB5F9001000FB013071
:102E2000E08001210420FFF715FDB5F9021000FB39
:102E300001F302210420FFF70DFDB5F9001000FB9E
:102E4000013020810320FFF7F7FCE1880844E0808F
:102E50000420FFF7F1FC2189084420813EE004238F
:102E600001211846FFF7F6FCC3F1050135F81110F2
:102E7000484324F813001846FFF7DEFC34F813101B
:102E8000084424F813005B1C062BE9D326E0032337
:102E900002211846FFF7DEFC8446B5F90400012143
:102EA0000CFB00FC1846FFF7D5FC0146C3F10600F9
:102EB00020F00100285E00FB01C024F81300184632
:102EC000FFF7BAFC014634F81300084424F8130055
:102ED0005B1C072BDCD3F988A9F800102020FEF733
:102EE000D4FDB8B30020FFF7A7FC20800120FFF736
:102EF000A3FC5B496080097A61B39AF8BC20514613
:102F0000920714D591F97A209AF982105542B8F9AE
:102F10000020B8F9023051435D4395FBFBF591FB6E
:102F2000FBF16B1A22882944D21A228010E091F911
:102F30007A50B8F902202788554395FBFBF53D44AC
:102F400025809AF98210B8F90030594391FBFBF1C2
:102F5000084460800025574607EBC5007430B0F97F
:102F60000220B0F9001034F9150003F0CFFC24F86A
:102F700015006D1C082DEFD397F8BC00DFF8E4A016
:102F8000400717D5707900250E281BD0082819D0C6
:102F9000354901EBC000407800B1022500245746B6
:102FA00007EB440001896019C0B205F03EFB641CC8
:102FB000042CF5D3284A0120121F4D46B9F90070A0
:102FC000117807E00425E9E735F91030BB4200DD50
:102FD0001F46401C8842F7D3002490465AE000BFA9
:102FE000B6F8D200B84205DA35F81410381A081AC3
:102FF00025F814004FF48040FEF747FD98B1BAF968
:103000000600B6F81211884204DDB6F8D220B6F8F0
:10301000D81003E0B6F8D620B6F8D41035F914006D
:1030200003F074FC27E0B6F8D220B6F8D01035F9DA
:10303000140003F06BFC25F81400BAF90600B6F88A
:103040001411884219DA102010E000006C090020E9
:103050009404002034000020BC000020D40A00208A
:10306000300B0020E60A0020E0DA0008FEF70DFD34
:1030700038B1B6F8D40025F814000948407818B1E2
:1030800007E0B6F8D000F6E7064830F8140025F857
:103090001400641C98F800008442A1D3BDE8FC9F92
:1030A000D40A0020540900202DE9F047174689462C
:1030B00006460025DFF83C841AE0002411E000BF3A
:1030C000D8F8001081F00801C8F80010012005F0C0
:1030D0005AFB484605F04CFB002005F054FB641CED
:1030E000E4B2B442ECD33C2005F042FB6D1CEDB2DF
:1030F000BD42E2D3BDE8F0872DE9FC5FFE4BFF4CFB
:103100000025B3F90600E28C904201DA64210DE05B
:10311000FA49B0F5FA6F91F8251005DA861A4E4390
:10312000C2F5FA6196FBF1F1C1F164018946F449F7
:10313000A24694F86CE094F86DB0B1F81241002208
:10314000ED49EF4B40F2E63C31F91260311B01F2E0
:10315000F317674503D8002903DCA11B01E04FF4F6
:10316000FA71022A34D0BEF1000F05D08E4502DA82
:10317000A1EB0E0100E00021642391FBF3F3DE4F8D
:103180006FF01808243707EB430C37F91370BCF9BC
:1031900002C003FB08F3ACEB070C01EB83030CFB51
:1031A00003FC64239CFBF3F33B44D64F27F8123017
:1031B0009AF823304B434FF4FA7193FBF1F1C1F1CC
:1031C000640189B201FB09F1642391FBF3F11CE076
:1031D000BBF1000F05D08B4502DAA1EB0B0100E03B
:1031E000002193F9EC30DFF81CC35B424B43ACF891
:1031F00004309AF82430002900DC49424B434FF454
:10320000FA7193FBF1F1C1F164010AEB0207642347
:1032100097F801C0DFF8EC820CFB01FC9CFBF3FC8F
:10322000A8F1540808F802C097F80BC008F1030889
:103230000CFB01FC9CFBF3FC08F802C07F7D4F43B4
:1032400097FBF3F108F10303A642995405DAAD495F
:1032500031F812305B4221F81230521C032AFFF67B
:103260006FAFDFF89CA24FF4FA625446BAF814111B
:1032700003F04CFBB4F814114FF47A72401A504327
:10328000C1F5FA61B0FBF1F1642291FBF2F09A4BC7
:103290006FF01806323303EB400433F910307043FB
:1032A000B4F9024001EB8000E41A444394FBF2F0CD
:1032B000DFF85082904E1844123EA8F80600707A4B
:1032C000A8F17804E8B39048B4F91C10B0F90000F4
:1032D000401A08F00BF98D4908F086F88C4908F07F
:1032E000B9F8074608F0DAFF0190384609F0BCFB50
:1032F00000904746B8F9000008F0F8F883460099B6
:1033000008F072F88046B7F9020008F0EFF881463D
:10331000019908F069F8414608F00EF808F0F4F851
:1033200080464846009908F05FF881465846019962
:1033300008F05AF8494608F051F808F0E5F83880E6
:1033400000E001E0A7F802800220FEF79EFB0027C4
:1033500050B3E079401CC0B20621B0FBF1F2E0713D
:1033600001FB1200B8B9002004F024F9217A624A66
:1033700001F00703AE3A491C22F813002172002025
:1033800032F81010401C29448DB20828F8DBE808F8
:1033900001F030F8A073A07B618C884203D89AF8C2
:1033A0000611814201D9A77101E00420A071A07922
:1033B00003F013FA57484F4D008818B10220FEF76A
:1033C0004FFB10B95448008820B1286880F00800ED
:1033D00028600CE0B178082011B14649091D086049
:1033E000717811B143490831086003F0FAFE80207A
:1033F000FEF74BFB48B1A16C206B411A05D44CF28F
:1034000050310844A06405F0DDFC616C206B411A6A
:1034100003D4717B39B10120B07002F063F83F48EA
:10342000007848B10FE0B770296881F00801296081
:103430003B4908446064F0E74FF40060FEF725FB69
:1034400008B103F006FF2020FEF70AFB68B1E16C2B
:10345000206B411A09D4E17B052906D33149084480
:10346000E064286880F0100028602F4881680029F7
:1034700005D002B02348BDE8F05F5A380847BDE8E0
:10348000FC9F10B51E4C204490F8080105F0D7F8B9
:10349000A0F2EE2140F2DD52914201D3B4F81201C4
:1034A00010BD2DE9F0470820FEF7EFFA154D124F39
:1034B000783D50B10024A96B2046884727F81400B6
:1034C000641CE4B2082CF6D314E6687ADFF828808E
:1034D000401C0024A8F19E086872A14608F140062D
:1034E000A96B204688476A7A08EBC40102F0030200
:1034F0001CE000000C0C0140E60A00202C08002013
:103500009404002044010020B0010020DB0F49405A
:10351000000034437E0100208001002000000020D4
:1035200020A10700F0490200B80C002021F8120089
:1035300026F814905FF0000036F8143031F81020AF
:10354000401C1A44C0B226F814200428F4D336F9DB
:103550001400801CC11700EB9170801026F8140035
:1035600037F91410C91E884202DA811C27F814109A
:1035700037F91410C91C884202DD801E27F8140098
:10358000641CE4B2082CABD3B4E5FE480288FE48C4
:10359000417852B9827842B1002905D101214170A8
:1035A000FA48FB490088888370470029FCD1012232
:1035B000FF21022078E52DE9FC5F0020F4498246D6
:1035C0007831054607460190B1F9020043420028D0
:1035D00001DD044600E01C468B46B1F900104A426A
:1035E000002901DD0E4600E01646B44203DD002846
:1035F00006DC184604E0002901DD084600E010461C
:10360000DFF8909300240090DF4EF07808B930790D
:10361000F0B3022C40DADE48403030F914103BF9A8
:10362000140001EB4000DC49B1F8F620514203F0F0
:103630006DF9DA49DFF868A331F91410411A0AEB81
:103640004400B0F92A0001EB00089AF80810642041
:1036500001FB08F191FBF0F09AF81C1001EB8102DC
:10366000494201EB810103F051F90190C84842F24F
:103670001072703050F8241001EB0800514203F032
:1036800045F9C349703141F824009AF8121000E05E
:1036900008E048434FEA203AF07818B1307908B989
:1036A000022C49D13BF91450B74F05EB85000101BD
:1036B000BB48A83F00EB04084FF47A5298F8010089
:1036C00091FBF0F039F91410401A57F8241008440F
:1036D000514203F01BF947F8240039F9140000F5B2
:1036E0002070B0F5A06F02D857F8240002E0002047
:1036F00047F824007D2190FBF1F098F80B10484327
:1037000087113079B0B1022C14DA0098009BC0F513
:10371000FA71019801FB00F2009801FB0AF105FB28
:1037200000204FF4FA7207FB031190FBF2F091FBBB
:10373000F2F608E0F07820B1022C02DA5646019841
:1037400001E028463E46924A39F9141024325023AB
:10375000125DDFF834824A4392FBF3F28C4B821AFB
:103760006433A8F13C0833F9140023F81410081A44
:1037700008F10C0158F8243051F824C041F82430E5
:103780009C44844448F8240081482A30005D00FBB2
:103790000CF0C11700EBD1609119A1EB60107C49CE
:1037A0006A3121F81400641C032CFFF62DAF66E685
:1037B0002DE9F05F744E4FF0000BDFF8E4A1DFF865
:1037C000D0915C46A83E704DE87808B92879D8B108
:1037D000022C19DA6E48403030F91410383030F9C4
:1037E000140001EB40006C49B1F8F620514203F09F
:1037F0008DF86A4931F91410411A0AEB4400B0F906
:103800002A0001EB000B01E0022C52D0E878E0B373
:103810009AF8080000FB0BF000115E490AEB040760
:1038200031F91410FA7A451A787856F8241068435A
:103830004FEAE018B9F810006843C01200FB02100C
:103840004FF4001246F82400514203F05FF846F8A6
:10385000240043134C480C3850F8241040F82450EE
:10386000B9F81000691A02094FF6FF70B0FBF2F0C8
:10387000484345498011243901F10C0251F824C014
:1038800052F824506544054400E01CE042F824C08E
:1038900041F82400787D08EB0301684301EB202008
:1038A0003B496A3121F81400641C032C8BDBBDE812
:1038B000F09F9AF8240036491B307831B1F9041092
:1038C00048434011A9E7324A9AF8230078321B3066
:1038D00032F9142050432A790011002A9DD09AF819
:1038E000121001FB0BF100EB212096E7284901287B
:1038F00001D02C4800E02C48C86370472DE9F84FF0
:103900000027B946B8460820FEF7BFF8DFF888B0B0
:1039100090B19BF8100130B1012804D0022805D0E5
:10392000032809D105E002F0D8FE04E003F080F995
:1039300001E003F00BFA8046DFF854A0124C4FF080
:103940000106DAF83010DAF850004FF00005081AD6
:1039500002D5B8F1000F7CD044F620621144CAF8B9
:103960005010FFF79EFD4FF48040FEF78EF828B10F
:1039700005485C30007808B900F07EFC9BF81B011C
:1039800060B313E080010020D40A0020B0010020C1
:10399000CC0000207000002094040020340000209F
:1039A0002C080020B7350008B1370008FB494FF458
:1039B0007A7201EB40000021B0F90600A0F57A70A0
:1039C00002F0A4FF07F092FDF54907F043FDF54929
:1039D00007F00AFD07F0B1FDAAF820004FF40070CF
:1039E000FEF753F8B0B3DFF8C083BAF9122098F8A5
:1039F000B4C00CEB8C0191421DDA6078D8B1BBF9F0
:103A00001231E649002000BF21F81030401C032885
:103A1000FADBB8F8B630CB8098F8B500604400EB1C
:103A20008000904202DA00F027FC2570BAF81410EA
:103A3000491CAAF8141098F8B40000EB8001BAF9F8
:103A40001200814204DA607810B900F015FC25708C
:103A500001E062E204E0BAF81210491CAAF8121060
:103A6000BBF81411BBF81621DFF830830020BF0823
:103A700038F910C08C4501DD47F08007944501DA24
:103A800047F04007401C0428F1DB9AF80B10504621
:103A90008F4205D1817AFA2903D2491C817200E054
:103AA00085728AF80B704FF480473846FDF7EDFFBA
:103AB00058B1BBF81211BBF8DC00B8F906200B1A9C
:103AC000934202DA0844904209DC3846FDF7DDFFF4
:103AD000F0B9B8F90610BBF81401814218DAAF4802
:103AE000BA38056045608560B04805604560AE48FD
:103AF000B0F8420060B1A9484A30007820B120787F
:103B000010B1FFF742FD03E0607808B100F0B4FBAC
:103B10009AF80A00142848D16078B8B1A24FB7F8D3
:103B2000420028B99AF80B005F2801D100F0A4FBED
:103B30009BF81801002838D0B7F84200A8BB9AF8C3
:103B40000B007D2831D100F097FB8FE09AF80B0035
:103B5000572809D00420FDF798FFE8B19AF80B1018
:103B600050465A2922D017E091494FF47A700880C4
:103B70004FF48070FDF789FF08B102F066F8042069
:103B8000FDF76EFF10B18B490A2008800820FDF771
:103B900067FF08B9884805809AF80B005D2816D0A1
:103BA0005B2816D05E2816D022E05FE0C17819B1FC
:103BB000C5708AF804601BE0817891F00101817082
:103BC00001D0022100E003218AF8001010E0012753
:103BD00002E0022700E00327781E8BF894030021FF
:103BE0000846FDF76EFD3A4628210220FFF75CFAF1
:103BF0006D4FB7F8420018B99AF80B106F290ED024
:103C00009BF8181121B118B99AF80B007E2806D03C
:103C10009AF80B00972805D0A72808D008E0FFF7EE
:103C2000B4FC05E065494FF4C870088000E0A67355
:103C30009AF80B00BB2806D0B72807D0BE2809D0B9
:103C4000BD280AD012E0B88D801C01E0B88D801E1E
:103C5000B88505E0788D801C01E0788D801E788520
:103C600001210846FDF72DFD8AF80A500420FDF7D2
:103C70000CFF28B39AF80220504632216AB16278CC
:103C80005AB1B8F90630BBF81421934205DD434A16
:103C90004A3212780AB9C1828570404A4A32527C4F
:103CA0003AB14279C3781A4300D1C1828AF80560DB
:103CB00006E0C17821B1617811B9C5708AF8046055
:103CC0000020C64640F2A4670EEB4001B1F908207F
:103CD00040F214518A4201DA012300E0002300EB94
:103CE00040018B40A2F2155CBCF5C77F02D84FF0B3
:103CF000010C01E04FF0000C01F101080CFA08FC86
:103D000043EA0C03BA4201DD012200E00022891CD3
:103D10008A40134343EA0903401C1FFA83F904282D
:103D2000D2DB1E4F00204A371F4901EB4001B1F89A
:103D3000421011EA090100D001213954401C152814
:103D4000F2DB787840B9184890F8B40000EB8001B5
:103D5000BAF9120081420ADA0220FDF781FE30B181
:103D6000E07828B9114805604560E67000E0E5702C
:103D7000B87838B1E570207928B90C4805604560FD
:103D8000267100E025713878B84600B92670E178D0
:103D9000102009B92179A9B1094914E0E60A0020E7
:103DA00000007A4400C07F442C0800203C01002021
:103DB00080010020AE010020B00100207E01002023
:103DC000140C0140FE4908600420FDF749FE00B3D1
:103DD00098F80300474678B1A07970B9F948A67100
:103DE0000168F9480160F948C188F948AAF8181033
:103DF0000560F848056000E0A5714FF40050FDF73C
:103E000044FE30B1387918B1E07B10B9E67300E0B8
:103E1000E5730220FDF724FE18B90820FDF720FE07
:103E2000D0B198F80510404639B1617931B9EA4905
:103E300066710A88E9490A8000E06571817919B1E3
:103E4000617A11B9667200E0657298F8070018B1DE
:103E5000E1480188AAF81C102020FDF701FEE0B31C
:103E6000E07AD8B39AF80F005746052843D398F85C
:103E70000A1061B1E07980BBD449E6712572143132
:103E80003D73081F02F01BFB0220787037E0E571DC
:103E900098F80B0038B3CD4AB2F90000002800DCD6
:103EA0004042CF49B1F8C81088421CDAB2F902008A
:103EB000002800DC4042884215DA207A68B9C348FD
:103EC000267208303D7300F1100102680A604068F4
:103ED00041F8040FBD48183001E010E00BE002F09B
:103EE000EEFA7E700BE02572387B40B98AF80C60E0
:103EF00002F08BFA03E0E57125728AF8015098F818
:103F00000C0008B1A67200E0A5729BF80500082815
:103F100001D00E283DD165723BE0DAF858005746D3
:103F2000052836D2DFE800F0030B151F2A00082011
:103F3000BE65FDF795FD10B100F079FC48BBB86D8A
:103F4000401CB8650420FDF78BFD10B100F07EFB2E
:103F5000F8B9B86D401CB8650420FDF781FD10B1BB
:103F6000FEF78DF9A8B9B86D401CB8654FF48070A4
:103F7000FDF78BFD10B102F005FA0AE01020BD65D7
:103F8000FDF76EFD08B100F0D4FC4FF40050FDF7D2
:103F90007CFD04F0C4FBCAF83000BBF80C20574687
:103FA00012B17B6DC31A76D41044D8467865FEF7FB
:103FB00028F9FFF7A1F804F0B2FB3863B98E411A73
:103FC000398278630820FDF74BFD40B37F49B1F992
:103FD000042002F145008A2822D8607900B37E4887
:103FE00003887E480088181A00B210F1B40F02DC72
:103FF00000F5B47000B2B42802DBA0F5B47000B2D2
:1040000098F9EC305B42434318B2637B3BB1744B8D
:104010005B7A43431E2093FBF0F0101A888003E084
:104020006D4801886D4801800420FDF719FD68B1D5
:10403000A07958B1207C80B16448664998F91A315A
:10404000B0F90220096801FB03214180644D95F815
:104050007200C0B3E078B8BB66E0614890F86F10BA
:1040600031B35A49B7F91820B1F90630A3EB020C65
:10407000BCF1000F01DCA2EB030C90F86E0084454C
:104080000ADDDFF84CC19342CCF800507E7300DDAE
:10409000404218440AE0EDE0787B20B149480368CB
:1040A000494803607D734B4800881044C880CDE7C1
:1040B000DFF81891B7F91830B9F90620D11A00299C
:1040C00003DD0A4602E037E030E09A1A90F86E000D
:1040D000824211DD788B4FF4FA65084401B291FBFE
:1040E000F5F0394AD2F800C0844405FB1010C2F83C
:1040F00000C078837E7307E0787B28B1314801687F
:10410000314801607D837D7332484D4600881844F4
:1041100000B2A9F80600B8F8D010B8F8D22096314D
:1041200002F0F4FBE88091E7207928B127482D4A76
:10413000C18812881144C1802020FDF791FCE8B3AA
:10414000E07908B9207AC8B3207BB8B3224CB4F91F
:10415000000007F0CBF9244E314607F045F908F08E
:1041600083FC0090B4F9000007F0C0F9314607F075
:104170003BF908F093F8154C064695F8C1001C3C35
:10418000DFF86890A4F11C08C8B1A246B4F9020097
:10419000241DB4F90210401A01F000FB15F8C12FDC
:1041A000514202F0B3FB618808446080BAF9000014
:1041B000B4F90010401A01F0F1FA19E050E020E0E3
:1041C000100C014060000020640000204401002029
:1041D0002800002024000020B0010020B2010020AF
:1041E0002C0800200E00002035FA8E3C00002041F3
:1041F0002A78514202F08AFB2188084400B22080CC
:1042000001E0B4F9000007F071F98346009907F066
:10421000EBF80546B4F9020007F068F9824631462A
:1042200007F0E2F8294607F0D9F84D46494607F06D
:1042300011F907F069F9A8F80000444658463146DC
:1042400007F0D2F806465046009907F0CDF83146FF
:1042500007F072F8294607F0FDF807F055F960807D
:10426000F86B8047FEF7ADFCFEF7B7FBBDE8F84FF3
:10427000FEF707BCBDE8F88F03484178002901D05C
:104280000021417070470000D40A00202DE9F84356
:10429000FD4CFE4BFE490026B4F8EE209846A1F1F5
:1042A000100004F090FE08B101260EE0B4F8EE1004
:1042B000F74805F097F840B9B4F8EE10F44803F069
:1042C000FAFF10B9032004F0FFFAF24D5FF0000787
:1042D00094F8ED0006283CD2DFE800F00707192823
:1042E00033030220FDF7C9FB33E08DF800704FF473
:1042F0004870E749ADF802001039684603F0FDF94F
:1043000008B10120287094F8ED00012821D06EB189
:10431000DF49B4F8EE204346A1F1100004F053FE4B
:104320000220287094F8ED0002281DD0D8481038DB
:1043300004F052FF28B10320287094F8ED00032800
:1043400012D0D348103805F08AFE10B1042028702E
:104350000AE0287840B994F8ED0010B184F8ED70C7
:10436000B6E70220FDF789FBC948103005F03DF99A
:1043700038B9C748103003F067FA10B90420FDF7C8
:104380007CFB0220FDF76CFB28B1C14994F8E300E7
:10439000103909688847BE4914F8E20F0968884750
:1043A000A07803F06BFB10B90820FDF766FBBA4854
:1043B0006421B0F9282092FBF1F001FB102406B231
:1043C0000820FDF74DFBB54D90B1204607F08EF863
:1043D000B34907F009F80446304607F087F821464C
:1043E00006F0AAFFAF4906F0FFFF2860BDE8F8839A
:1043F0002F60FBE770B50546A34890F8040107F06D
:104400007EF80446284607F07AF8A74906F0ECFF44
:10441000A64907F01FF8214606F0E6FF07F08DF8E1
:1044200080B270BD70B500252C46002003F0C2F8A4
:1044300005440A2004F09CF9641C202CF5D3C5F334
:104440004F10FFF7D7FF904A022192F8053100BFC5
:1044500003FB01F4844202D8491C0629F8D394488E
:10446000017092F8060148439249088070BD2DE919
:10447000F05FDFF82092904E874FB9F80220824C0F
:104480000025C2B38D4900204FF4C878424501D1C0
:1044900041F8205051F8203036F910C0634441F8FB
:1044A000203026F8105004EB4003401CA3F8F850CD
:1044B0000328EBDB012A19D10868C83090FBF8F01B
:1044C00024F8F80F4868C83090FBF8F060808868DE
:1044D000C83090FBF8F1B9F80600081AA0807D8575
:1044E0000121F83CBD850846FDF7EBF8B9F802104C
:1044F000491EA9F802100420FDF7C7FA002873D05E
:104500006F4BDFF890816D491A8808F120080C3153
:10451000A8F1180A322A05D0F2B300209B46322AAD
:1045200014D015E034F8F80FA8F800006088A8F857
:104530000200A088A8F80400B7F82AC0AAF800C0B2
:10454000B7F82CC0F83CAAF802C0E6E741F82050C2
:1045500051F8203036F910C0634441F8203026F875
:10456000105004EB4003401CA3F8F8500328D6DB9E
:10457000012A1AD15348544B057001201870534B2F
:1045800002201870B8F8000024F8F80FB8F80200FC
:104590006080B8F8040000E00AE0A080BAF80030BB
:1045A0007B85BAF80200F83CB885521EABF80020B3
:1045B00047480278C2B105700A68322092FBF0F2D7
:1045C00024F8F82F4A6892FBF0F26280896891FB28
:1045D000F0F1B9F80600081AA0807D850121F83CA9
:1045E000BD850846FDF76DF8308834F8F81F401A8D
:1045F000308070886188401A7080B088A188401A25
:10460000B080BDE8F09F224810B5103841682A48B4
:104610008847BDE810402AE730B51E4C1E4AE068C6
:1046200092F831200146401C824200D10020294AE4
:104630001368224A183242F82130274952F82020C4
:104640000D682B449A1A0A60E06030BD70B52348AB
:10465000104C00682169411A01D5002070BD20610D
:104660000B4D60691035E8B328698047686880475A
:1046700028882169084420616A69194915489047CA
:1046800000206061022070BD9404002038090020E1
:10469000B80C00207C0100202C08002030000020F5
:1046A0008988883C000020413333534000F07F4527
:1046B00068010020EE0000207C000020880B002014
:1046C000E2000020D1000020CF000020CC0000201C
:1046D000D0000020A40000201C000020FC000020CE
:1046E000A8000020FFE7A8688047E8688047FFF738
:1046F00093FF0120606168882169084420610120DE
:1047000070BD2DE9F05FA34DA88800286AD0DFF8BE
:1047100088820024A3464FF47A79A8F10C06A88871
:10472000484507D104EB840208EB820146F824B027
:10473000C1F810B0994F56F8241037F9140001440D
:1047400046F8241006F0D2FE014604EB840208EB82
:104750008200824600F0F0F827F814B0904F27F856
:1047600014B0A888012837D1DAF81000012808DD34
:10477000401E06F0BBFE0146DAF80C0006F06AFEA9
:1047800000E0002008F036FA8246864890F8F400EF
:10479000A8B106F0B4FE514606F0E4FE0FD27E4901
:1047A000A5F80490C8F810B0C1F824B0C1F838B02A
:1047B000C6F808B0C6F804B0C6F800B00CE056F869
:1047C0002400012200F5FA7090FBF9F027F814009C
:1047D0000F210A20FEF768FC641C032C9FDBA888CD
:1047E000401EA8806D496E4A002000BF31F810308D
:1047F00032F810401B1B21F81030401C0328F5DB59
:10480000FFE6654810B54C30416864488847BDE80C
:10481000104076E710B564481024046003F07DF979
:104820006148001F04605B490120487010BD2DE9FC
:10483000F0415E48574C0068A169411A02D500203A
:10484000BDE8F0815A490844A0615A4803F02DF9A7
:10485000DFF864C14F4B00269CF80E005549514AC1
:1048600026339D1D88B1A069E061002002EB40075E
:10487000A7F8FE6031F8107023F8107025F810705A
:10488000401C0328F2D38CF80E60607868B1088869
:1048900032F8FE7FC01B088048885788C01B4880BC
:1048A00088889788FE3AC01B8880E069A0B3A76912
:1048B000381A424FB84219D23B480838026882F091
:1048C000080202605FF0000031F9102033F9104057
:1048D000A24201DA23F8102035F91040A24201DD8E
:1048E00025F81020401C0328EED315E00020E661D7
:1048F00033F9101035F91040214402EB400401EB6C
:10490000D17141F34F01401CA4F8FE100328EFD3EE
:1049100001210846FCF7D5FE012091E710B50120E2
:1049200004F0A7FC1020FDF7A3F82549002008603B
:1049300010BD234804F0F1BC2DE9F04104460069A4
:104940000E46401C206101281FD006F0CFFD2568CF
:1049500080462946304606F041FD0746414606F0AE
:1049600079FD294606F0E8FC054660602946304698
:1049700006F034FD0146384606F036FDA16806F023
:10498000DBFC2560E060A0605AE7666000202660DE
:10499000F9E700007C0100206C0C0020760000206C
:1049A000AC00002094040020140C0140FC00002006
:1049B000A086010088000020D40A002080C3C9011D
:1049C000B400002070B5F74CF74EC1B205466170D7
:1049D000306805F065FBA07961784840A071C5F3A7
:1049E00007216170306805F05BFBA0796178484071
:1049F000A071C5F307416170306805F051FBA079E3
:104A000061784840A071290E6170306805F048FB5C
:104A1000A07961784840A07170BD70B5E14CE24E5C
:104A2000C1B20546A170306805F03AFBA079A178C3
:104A30004840A071C5F30721A170306805F030FB34
:104A4000A079A1784840A07170BD10B50446D64841
:104A50002146006805F024FBD248817961408171CC
:104A600010BDD04AD148D179405C491CD171704702
:104A700000B5FFF7F6FF0346FFF7F3FF03EB002057
:104A800080B200BD10B5FFF7F3FF0446FFF7F0FF5B
:104A900004EB004010BD70B504460D462420FFF71E
:104AA000D4FF4D20FFF7D1FF0CB1212000E03E20C4
:104AB000FFF7CBFFBB4C0020A0712846FFF7C5FFD6
:104AC000207ABDE87040C0E701460020E3E70146D8
:104AD0000120E0E7B3488079B7E770B504460D469A
:104AE0000846FFF7F1FF03E014F8010BFFF7ADFFF5
:104AF0002800A5F10105EDB2F6D170BD10B5044650
:104B000003E000BFFFF7A1FF641C20780028F9D163
:104B100010BD2DE9F05FDFF88CB2DFF88892012735
:104B20004FF0000A0BF10C0B00251AE09F481538D6
:104B3000405D00EB40010BEB8108D8F8040006F063
:104B4000ACFB06460FB1B2440AE0002406E000BF09
:104B5000D8F80400005DFFF778FF641CB442F7DB6F
:104B60006D1C99F800008542E0DB002F05D00AF0AB
:104B7000FF00FFF7A9FF0027D6E7BDE8F09F70B55B
:104B80000246032300218A4803F074FF8649FF226E
:104B9000086086481521153806F039FB834D002042
:104BA000153D012428700220FCF75AFF20B1012096
:104BB00068700220A87003240420FCF751FF50B154
:104BC00003202855641C4FF40050FCF75EFF10B121
:104BD00004202855641C0220FCF742FF18B9082065
:104BE000FCF73EFF40B105202855641C06202855DF
:104BF000641C07202855641C2020FCF746FF10B1D8
:104C000008202855641C4FF48070FCF73EFF28B143
:104C10000A202855641C0B202855641C654E7079A9
:104C2000082801D00E2802D10C202855641C0D2024
:104C30002855641C0420FCF728FF10B111202855CA
:104C4000641C1320285596F82C01641C00B1012027
:104C5000FCF71BFF10B114202855641C5148047048
:104C600070BD2DE9F05F4F4EDFF840B14FF0000806
:104C7000317A504D504C514FC1464FF0010AABF1C3
:104C8000150B782978D011DC3046A1F16401007849
:104C9000142972D2DFE801F0FDFCFBFAF9F8F7F60F
:104CA000F5F4F3F2F1F0EFEEEDECEBEA4348D02946
:104CB000407873D018DCCB2971D00CDCC8292AD0FD
:104CC00004DCA0296CD0A42957D1E3E3C92937D04B
:104CD000CA29F9D152E0CC2963D0CD297CD0CE2984
:104CE0007BD0CF29F0D1A6E0D62977D00ADC4FF0CF
:104CF0000008D12973D0D22972D0D32971D0D429F8
:104D0000E2D1D0E1EF2914D0F0296BD0FA296AD092
:104D1000FE29D9D187E32A4D002400BFFFF7A8FE62
:104D200025F81400641C082CF8D30020FFF7CCFEF3
:104D3000D4E3FFF79DFEA085FFF79AFE6085F4E7B8
:104D4000FFF78FFEF872FFF78CFE1E490870FFF721
:104D500099FE1D4C2060FFF795FE6060FFF788FE0E
:104D60001A490880FFF784FE19490880194801781C
:104D700041F002010170D8E77BE14BE35FF00003F3
:104D8000FFF76FFEE5186870FFF76BFEE872FFF73C
:104D900068FE5B1C68750A2BF2D3C6E727E323E0A5
:104DA00068E331E0B401002028090020F50C002060
:104DB00000380140940400202C080020D40A002070
:104DC000E60A0020DB0000204C01002076010020D4
:104DD00078010020640100200FE315E369E0D6E2CA
:104DE00072E07DE03CE314E300255F4608E000BF8D
:104DF000FFF73EFE795D6D1C04EB4101A1F8420016
:104E000030788542F4D390E7FFF72BFE04F81F0FAC
:104E1000FFF727FE6070FFF724FE2071FFF721FEE9
:104E20006071FFF71EFEA071FFF71BFEA070FFF779
:104E300018FEE07079E7FFF71BFEFFF719FE25F873
:104E4000D00FFFF715FE6880FFF712FEA880FFF76E
:104E50000FFEA4F8B600FFF70BFEFFF713FEFFF7F7
:104E600007FE00EB80004000208513E0EAE16AE2E3
:104E7000CBE1E4E15BE2F2E1CEE1B4E19BE189E187
:104E80007DE16AE157E139E12AE124E1EEE0BAE0AF
:104E90003FE029E0FFF7E5FD85F83400FFF7E1FD8D
:104EA00085F83600FFF7DDFD85F83500FFF7D9FD01
:104EB0003BE7FF4D002400BFFFF7DAFD25F81400A3
:104EC000641C082CF8D330E700289CD1FFF7C9FDFB
:104ED00085F89403022801D985F8948300219EE285
:104EE000FFF7C6FDF3498DE20720FFF7EDFDE62051
:104EF000FFF7ABFD6879FFF7A8FD0020FFF7A5FDE0
:104F000095F8190100B10820EB490843FFF75AFD55
:104F1000E4E20B20FFF7D8FDE848008800B2FFF775
:104F20007CFD03F004F900B2FFF777FD0220FCF7E7
:104F300097FD04460420FCF793FD44EA4004082052
:104F4000FCF78EFD44EA80042020FCF789FD44EA4A
:104F5000C0041020FCF784FD44EA0010FFF75DFD5B
:104F6000F9783A79490041EA8201BA79002041EAA8
:104F7000C2017A79367841EA42117A7AD44641EA16
:104F80008211CF4AD37941EAC311137A41EA03214E
:104F9000537A41EA4321FB7941EA83213B7A41EA92
:104FA000C321BB7A41EA0331537B41EA4331937B0E
:104FB00041EA8331137C41EA0341137941EA031149
:104FC000537C41EA4341937C41EA8341D37C127D87
:104FD00041EAC34141EA025479785F460C4300221A
:104FE00008E0BB5C0CFA03F3234202D00CFA02F196
:104FF0000843521CB242F4D3FFF7E4FC95F8940343
:10500000FFF723FD6AE21220FFF75EFDAD48AE4DCB
:105010004FF000040088B0F5806F0BD935F914000B
:10502000C11700EB5170C010FFF7F7FC641C032C94
:10503000F4D306E035F91400FFF7EFFC641C032CF1
:10504000F8D3A24D002400BF35F91400FFF7E5FCAA
:10505000641C032CF8D39E4D002400BF35F91400C6
:10506000FFF7DBFC641C032CF8D337E210219948CE
:1050700033E03820FFF728FD5FF0000604EBC6059B
:1050800035F9740FFFF7C9FCB5F90200FFF7C5FC4D
:10509000B5F90400FFF7C1FCA879FFF7D6FC761C30
:1050A000082EEBD31AE20020FFF70EFD5FF000069A
:1050B000FFF7DEFC04EBC60525F8740FFFF7D8FCFC
:1050C0006880FFF7D5FCA880FFF7CBFC761CA871A1
:1050D000082EEDD302E210217F48FFF7FEFCFDE130
:1050E0001020FFF7F1FC7D4D002400BF35F91400BE
:1050F000FFF793FC641C082CF8D3EFE11020FFF7B6
:10510000E3FCF87AFFF7A1FC75480078FFF79DFCF7
:10511000744C2068FFF756FC6068FFF753FC724838
:10512000008800B2FFF779FC7048008800B2FFF7F2
:1051300074FC6F482BE00520FFF7C6FC6D48008823
:1051400000B2FFF76AFC6C48B0F90000FFF765FC9D
:105150006A48007800F0010052E70620FFF7B4FC2F
:10516000674D002435F91400FFF757FC641C022C2E
:10517000F8D36448B0F90000FFF74FFCAEE1062019
:10518000FFF7A2FC60480068FFF71CFC5F4800883E
:1051900000B2F1E70720FFF797FC5D480078FFF7C2
:1051A00054FC0020FFF739FC5A48008800B2FFF792
:1051B00034FC0020E0E70720FFF786FC14F81F0FFF
:1051C000FFF743FC6078FFF740FC2079FFF73DFCD8
:1051D0006079FFF73AFCA079FFF737FCA078FFF77A
:1051E00034FCE0780CE71E20FFF76EFC0025661902
:1051F0007078FFF72AFCF07AFFF727FC707DFFF745
:1052000024FC6D1C0A2DF2D368E12F20FFF75CFC13
:105210004148FFF773FC61E14006000EFFF754FCC4
:1052200000255F4607E0785D04EB4000B0F94200DE
:10523000FFF7F3FB6D1C30788542F4D34EE1FFF7A6
:1052400068FC4BE1FFF740FC00245D4603E0285D6D
:10525000FFF7FBFB641C30788442F8D33EE1162054
:10526000FFF732FC0020FFF7D8FB35F9D00FFFF72E
:10527000D4FBB5F90200FFF7D0FBB5F90400FFF746
:10528000CCFBB4F9B600FFF7C8FB0020FFF7C5FB65
:105290000020FFF797FBB4F928000A2190FBF1F0FA
:1052A00000B2FFF7BAFB95F83400FFF7CEFB35E00C
:1052B00054090020B201002004000080DC0000201E
:1052C000300B0020820100208200002070000020AE
:1052D00088000020BC0000203C090020E60A0020D5
:1052E000DB0000204C010020760100207801002026
:1052F000660100207201002074010020640100207A
:1053000034000020B0010020600000202C000020AC
:10531000DA000020EC00002098DB000895F8360049
:10532000FFF793FB95F83500FFF78FFB2DE0082082
:10533000FFF7CAFB0024601CC0B2FFF786FB641CA9
:10534000082CF8D3CAE0FFF78CFB04461220FFF7C5
:10535000BBFB14B1102C02D004E0954800E0954846
:10536000D0E900892046FFF770FB4046FFF72AFB93
:105370004846FFF727FB90480068FFF723FB002013
:10538000FFF74BFB0020FFF748FB002038E6FFF754
:1053900068FB0546FFF776FB0646FFF773FB84467E
:1053A000FFF770FB0446FFF763FBFFF761FBFFF7B6
:1053B00058FB85B1102D7FF4C2AC7E49C1E9006C69
:1053C0000CB17D4804607D4A0220091D10707948A7
:1053D00001F075F8A9E47648002CC0E9006C87F864
:1053E000078087F80CA0F5D0734804609DE400287E
:1053F000F0D10120FCF725FB97E40028EAD17049A1
:105400004FF4C870088090E40028E3D187F80EA01C
:105410008BE418B10020FFF75AFB5FE00121002068
:10542000FCF74FF981E40820FFF74EFB6548674A17
:10543000674D016864481268B1FBF0F1B2FBF0F00F
:1054400000EB4002C2EBC01001EBC000E88000247A
:1054500035F91400FFF7E1FA641C042CF8D33DE0A1
:105460000420FFF731FBB4F92C00FFF7D6FAB4F9AA
:105470002A0081E60C20FFF727FB56480068FFF75B
:10548000A1FA5448001D0068FFF79CFA5148083003
:1054900000683BE5504D29780AEB8100C0B2FFF768
:1054A00013FB2878FFF7D1FA00244C4E4C4FDFF85D
:1054B0003481DFF834910EE0305DFFF7C6FA385DD5
:1054C000FFF7C3FA18F80400FFF7BFFA19F8040051
:1054D000FFF7BBFA641C28788442EDD3BDE8F05F87
:1054E000FFF7F8BA70B54148414C424E00780025AC
:1054F00040B3BDE87040FBF78FBD306804F0E3FDBA
:10550000617951B1012921D0022924D0032928D061
:1055100004292ED0052944D131E0242803D00021CC
:10552000617179B901E00121FAE73349497849B954
:10553000232808D0314991F89513814231D10120B7
:1055400003F0E3F92DE0FBF767FD2AE04D2804D1D5
:105550000220607125E03C2801D00020F9E70320FB
:10556000F7E740281CD82071E570E571A071042090
:10557000EFE72072A1794140A1710520E9E7E178C8
:105580002279914207D2A2794240A2711C4A50541A
:10559000491CE17005E0A179814201D1FFF761FB6F
:1055A0006571306804F08CFD0028A6D170BD000044
:1055B000540100205C01002064000020CD00002088
:1055C0007E0100202C04002040420F003004002007
:1055D0006A010020E8F7FF1F7A010020450B002038
:1055E000550B0020650B0020750B002000000020EB
:1055F000B401002028090020D40A002094040020CF
:10560000F50C00202DE9F047F94C607905F077FFA3
:10561000DFF8E093494605F01DFFF74D2860E07B79
:1056200005F06DFF494605F015FFF44EEE60686029
:10563000A07905F064FFF24F394605F00BFF1035F5
:105640002860207C05F05BFF494605F003FF686099
:10565000A07E05F054FFDFF8AC83414605F0FAFE6A
:10566000C5E90206E07905F04AFF394605F0F2FE89
:1056700010352860607C05F042FF494605F0EAFEDF
:105680006860E07E05F03BFF414605F0E3FEC5E9BA
:105690000206BDE8F08770B506460325002000F03D
:1056A00035FF4FF48070FCF7F0F900281ED0D24C83
:1056B000183C667003F04DF8A06000206060D2488E
:1056C00090F81C0100B90125FFF79CFFCF482B463D
:1056D00000EB061000214268CD4803F0CBF9CD491C
:1056E0004860BDE87040012000F010BF70BD2DE99A
:1056F000F041C548C74DC04C90F81C11C34E6868B6
:10570000183C11B1012945D106E0617806EB011181
:10571000496804F0DBFC3AE004F0DBFC00B32078DD
:10572000012802D02069F0B124E003F012F8616989
:105730000746401A64282FD32069052811D206EBAA
:1057400000104168686804F0C1FC607806EB001046
:105750008168686804F0A7FC2069401CC4E904075C
:1057600018E0022014E0607806EB001041686868D9
:1057700004F0ACFC20698C2809D2A4495031095CA2
:10578000686804F08DFC2069401C206102E0032061
:1057900000F0BCFE00206060BDE8F08144F2506182
:1057A000884201DDA0EB41009B49884202DA48F6BD
:1057B000A041084470472DE9F047064650689946D5
:1057C00014460D46301A05F091FE296805F042FE98
:1057D0002061A768394605F001FE8046844890F8AC
:1057E000C00005F08CFE8D4905F0FEFD01464FF02E
:1057F0007E5005F02FFE2D68294605F09DFD0146DF
:10580000284605F027FE414605F0EEFD394605F035
:1058100093FD2061C4E901600146D9F8080005F054
:10582000E3FDBDE8F04705F06FBE2DE9F0411D46F0
:1058300014460E4605F05AFE696805F0D5FD31683C
:1058400005F0D2FD216805F077FD2060ED68074680
:10585000284605F059FE064685F0004005F054FE46
:105860000546384605F050FE3246294601F04EF80E
:1058700005F03CFE2060BDE8F04105F045BE70B586
:10588000674CD4E90D01401AFFF788FF0028D4E9DE
:105890000D01A0EB010002DDFFF780FF02E0FFF742
:1058A0007DFF404241F29411884228DAD4E90D018B
:1058B000401A05F01BFE5B4905F096FD0646E06BBD
:1058C00005F01DFE0546304607F0CEF8294605F0E6
:1058D0008BFD05F019FE00B240F6B832208251422D
:1058E00001F014F8616B084448F6A04160648842F6
:1058F00000DD401A002800DA0844606470BD606B67
:10590000FBE72DE9FE4F0546FFF7B9FF444842F299
:105910002831406C081A05F0E9FD424905F064FDA4
:10592000044606F0BBFC0190204607F09DF800906D
:105930000024284605F0DAFDDFF8E4A0DFF8B8908F
:10594000DFF8E4B00AF1300A09F180090290344826
:105950001A3030F9140005F0C9FD05465DF8241031
:10596000029805F041FD294605F038FD05F0CCFD13
:1059700000B24FF47A7255462AF81400514200F0F2
:10598000C5FF1D4900B225F81400203100F0C7FD05
:1059900004EB8406184B2249074609EB8602904621
:1059A00035F9140020332C31FFF73FFF124B1C490F
:1059B0000744424635F9140020332C31FFF7FBFE33
:1059C000384400B240F6B8325D462BF8140051421C
:1059D00000F09CFF25F81400074859F826105830AD
:1059E000641C40F82610022CB1DBBDE8FE8F0000DD
:1059F0002C0800200000C842600D00200000FA447E
:105A00000000204100007A4494040020C8DB000814
:105A10000044004028090020B0B9FFFFDB0FC94057
:105A2000C8020020D3023739280100202DE9F05F99
:105A3000F84EDFF8E493DFF8E4B30024A6F1360A69
:105A4000F54956F82400583900F069FD3AF8141069
:105A5000F04F401A203FF04900B227F814004839AF
:105A600000F05DFD054637F9140056F8241004EBEC
:105A700084070844E84BE74909EB87029046483B16
:105A80002439FFF7D2FE2844E34BE2492BF81400F7
:105A90005D46424656F82400483B2439FFF78BFE0A
:105AA0004FF4FA62514200F031FF3AF914103131EB
:105AB000622900D8002035F8141040F6B8320844A6
:105AC00000B225F81400514200F020FF25F8140020
:105AD000D14859F827102830641C40F82710022CB0
:105AE000AEDBBDE8F09F70B505460868196814463E
:105AF000401A05F0FBFCC7495039096A05F074FCEF
:105B000005F002FD0146C348416029682268891AF0
:105B1000016070BD2DE9F0410F46DDE90685116891
:105B200000681E46081A05F0E1FC04463068396832
:105B3000401A05F0DBFCB7495039096A05F054FCFE
:105B40000646014605F050FC07462146084605F08A
:105B50004BFC394605F0F0FB07F04CF8B04905F076
:105B600043FC05F0EAFCC8F8000084F00040314630
:105B700006F06AFAAB4905F037FCAB4905F0DCFBEF
:105B800005F0C2FC2860002803DA48F6A04108446A
:105B9000286001E62DE9F0479E4CA448503C04F1F2
:105BA0004809D0E900566178B1B34FF07E50E16A00
:105BB00005F050FC8246D9F80400301A05F096FC36
:105BC000216A05F011FC514605F00EFC05F09CFC25
:105BD00007B2D9F8000004F11A08281A05F086FC6B
:105BE000514605F001FC05F08FFC01B204F12800DC
:105BF000B0F902203A4402EBD27242F34F02A8F805
:105C00000220B0F90030194401EBD17141F34F018A
:105C1000A8F800104280018001206070C9E9005698
:105C200037E510B5044605F061FC002C01DC80F07E
:105C300000407F4905F00EFC7E4905F0D5FB06F0DB
:105C40002DFB74495039086210BD10B57A4CE07ACA
:105C5000002812D07948007805280ED37349784A75
:105C60000868106049685160FFF7DBFF75486949B3
:105C70005039008888820120207310BD2DE9F0433F
:105C800064496548503978308E7A6B4B012502792A
:105C90000024062E29D004DC022E09D0032E04D1C4
:105CA00016E0122E33D0302E3DD00020BDE8F08318
:105CB0005E4A466856608668166000694FF47A72DC
:105CC00090FBF2F0604A1080C87AD8724D7350E0B1
:105CD0004079C00701D0032A03D00020C87210B158
:105CE00047E00120FAE7DC7243E0C27AD20702D033
:105CF000827A032A03D00022CA7212B102E0012282
:105D0000FAE7DC724D4A90F82F00107031E04F4BEB
:105D1000828A1A80806942F2107290FBF2F04C4A3B
:105D200010808D7325E04B4B102A1A7001D9102278
:105D30001A700022484E494FDFF824C1DFF8249141
:105D40001D7814E002EB420300EB830393F8088014
:105D500006F8028093F8098007F8028093F80B8018
:105D60000CF8028093F80C8009F80280521CAA42B9
:105D7000E8DB487B8A7B104098D04C738C73012001
:105D800094E72DE9F0412349002450390A4691F85F
:105D900009E092F807C0157A0CEB0003D78ADEB24F
:105DA0002246BEF1090F7CD2DFE80EF008050F1580
:105DB0001C235E6E7400622803D04A72B52802D09C
:105DC0006FE002205EE001205CE003224A7208736B
:105DD000C871087265E004224A72CE7172190A72A3
:105DE00088725EE005224A72CE7172190A72C88208
:105DF00057E006234B72731907EB0020CE7180B277
:105E00000B72C882B0F5007F01D9CA824A720A8338
:105E100047E0000018030020B80D002028010020F2
:105E20002C7D8E3FA00CB34500A00C464C010020F9
:105E30008096184B35FA8E3CD40A0020DB000020F7
:105E400054010020B00100207601002078010020DC
:105E5000660100207A010020450B0020550B002030
:105E6000650B0020750B0020CE7172190A720A8B27
:105E7000C82A01D2FE4B9854521C90B20883B842F3
:105E80000FD1072048720CE008234B72844508D0DC
:105E90004A7206E04A72854203D1FFF7EFFE00B175
:105EA0000124204678E470B50346002002460546EA
:105EB00015E02E2C04D1521C00290ED054181D556B
:105EC0009C5C00EB80004000A4F13006092E01D854
:105ED000303820440F2A01D3002070BD521C9C5C36
:105EE000002CE6D170BD2DE9F041002680463546F4
:105EF000374605F04DF90168444608F10F0004E00B
:105F0000844201D3002047E4641C22788A5C202A62
:105F1000F6D0404609E01EB106EB86025206160E88
:105F200010F8012B303E3244D6B2221A022AF2DC9B
:105F300009E01DB105EB85025206150E10F8012B84
:105F4000303D2A44D5B28442F3D820782E280ED191
:105F5000641C002007EB8702570022788B5C202B03
:105F600002D1303F1744641C401C0428F2DBC148B6
:105F70000621454307EBC70000EB071005EB800047
:105F8000B0FBF1F0BC494E4300EBC61004E42DE930
:105F9000F0470027B94C0546242815D0B44E2046BA
:105FA000F83EC0782C2D13D02A2D11D021460D2D6E
:105FB000497975D00A2D73D00F2802D23554401C70
:105FC000E07000296DD097E0A770E770277193E02B
:105FD0003754A0784FF0010928B1A179012921D0C7
:105FE000022966D07FE0A771307847287BD170788E
:105FF000502878D1B078472802D0522809D072E0D2
:10600000F07847286FD1307941286CD184F8069018
:1060100069E0F0784D2866D13079432863D10220B9
:10602000A07160E0DFF8588202280CD003280FD05E
:10603000042816D0052819D0062820D0072827D0F4
:1060400009282FD04FE08A48F838FFF74CFF05E0C9
:106050003078532847D1D8F800004042C8F80000F3
:1060600041E08348F838FFF73EFF05E030785728D5
:1060700039D1D8F804004042C8F8040033E0307841
:10608000302801D9012000E000207E49C8722AE0B2
:1060900077480021F838FFF706FF7B49087022E0B7
:1060A0002FE026E072480021F838FFF7FCFE774920
:1060B00018E0072802D008280ED014E06C4801210F
:1060C000F838FFF7F0FE41F2184148434FF47A7177
:1060D000B0FBF1F06E4905E065480121F838FFF7A3
:1060E000E2FE6C490880A078401CA070E7702A2D61
:1060F00004D0207968402071002091E584F8059053
:10610000FAE70029F8D0307800F037FA0501707806
:1061100000F033FA28442179C0B288426771EBD18C
:10612000A0790128E8D17BE52DE9FF5F5A49C0B28B
:1061300091F81C1119B1012904D002297DD1FFF772
:1061400026FF01E0FFF71DFE002876D0484CE83C12
:10615000A068E06002F0FDFAA0602020FBF788FC58
:106160004E484FF0000B0178012910D00121017039
:106170004448C17A002960D04349097805295CD395
:106180008246407830B19AF80C1031B108E080F8BE
:1061900000B0EDE78AF80CB002E008B1FFF755FD5A
:1061A000364805218E460278354C521CB2FBF1F37D
:1061B00001FB13223A490270002091F9009000BFC0
:1061C0002E4954F8203068312C4D41F820303549A3
:1061D000783593FBF1F145F82010274D00EB80074F
:1061E0006D424D4303EBC51342F2107593FBF5F579
:1061F000AEB2224D403525F810601D4D283D05EB0F
:1062000087071E4D57F822C0603555F8208047F8A3
:106210002230A8EB0C0C634445F8203093FBFEF3CE
:10622000154D694303EBC111144B7033B9F1010FE4
:1062300043F8201007D1B61E00E09EE0B6F5797F46
:1062400001D844F82010401C0228B9DB02F081FA82
:106250000A4D696A401A05F052F9134905F0FAF837
:10626000E86202F076FA68624FF07E51E86A1DE05B
:10627000300E002040420F002D310100C8020020E6
:106280004C010020D40A0020DB0000207601002011
:1062900078010020660100209404002064010020A1
:1062A000CD0000208096980000007A44884200DBF0
:1062B0000846E86203A902A8B74BCDE900011A1FFE
:1062C000211DB648FFF726FC02986426B0FBF6F0C5
:1062D000B349B44A57460880039890FBF6F0108003
:1062E0009AF80C0018B9A1F800B0A2F800B0FFF7B6
:1062F00051FC387A10B9F87900283ED0AA4901F14A
:10630000080000F11C07CDE900013B1D3A46211DA4
:10631000A248FFF7FFFB231DA04A391D3846FFF7AF
:10632000E2FBA24C94F90000012828D0022824D1D5
:106330009F4F0121B7F9C60000F0FCF8FFF7E1FA22
:1063400097F8C2009B4A18B1686C90FBF6F0108079
:10635000B7F8BE00E96B88420BD2D5E90D01401AAF
:10636000FFF71CFA002800DC404242F2107188421C
:1063700003DD01202070A88A1080BDE8FF9FFFF791
:1063800055FBFAE710B58C4C606828B909E06068E5
:1063900003F099FEFFF7C8FE606803F091FE002845
:1063A000F5D1864C207805282ED2DFE800F02D03A9
:1063B000031D0700BDE81040FFF799B9606805218B
:1063C000401C60606078401CC0B2B0FBF1F201FB81
:1063D0001200607002F0BDF97949A06000200870D9
:1063E0007849C87201200BE002F0B3F9A168401AA5
:1063F00040F6C411884207D92020FBF73EFB042059
:10640000BDE8104000F082B810BD2DE9F05FDFF864
:10641000ACA100246C4FDFF8B481DFF8B4910AF12D
:10642000480A25460AF1280B27F8145028F814507A
:1064300004EB840629F814500AEB860000F0A6F855
:106440000BEB860000F0A2F85C48983000EB860069
:1064500000F09CF8641C022CE6DBBDE8F09F2DE9FF
:10646000F04156480078032802D04FF0FF3019E57C
:10647000584D4FF00808C5F8008010262E604E4C8D
:106480002F1D606803F01CFE50B1C7F800806068E3
:1064900003F019FE0146206803F002FEC5F80080F3
:1064A000206803F00DFE0028EBD03E60206803F06A
:1064B0000AFE0146606803F0F3FD2E60E1E77CB55B
:1064C000394C026824342260096861600068FFF773
:1064D000A8FB3549314E01F10800CDE90001231D2B
:1064E0002246311D3046FFF715FBA4F15805331D38
:1064F000686B68643246211D2046FFF7F4FA686B2A
:10650000A8632B48B0F8C40068827CBD10B52B4C42
:1065100020700020206102F01CF9606110BD10B5F0
:106520000C4604F0E3FF216804F05EFFBDE8104074
:1065300004F0EABF70B51C4C343CE26B21B1B0EB07
:10654000520F0BD3500809E0904200D3104618496F
:1065500000B2B1F8C410814200DB0846B4F9125011
:1065600000B2A84208DD1C49E06A04F03DFF04F0D7
:10657000CBFF284400B2608270BD3038C0B2092819
:1065800001D9C01FC0B200F00F00704700210160A8
:106590004160816070470000580100204C010020DC
:1065A0007201002074010020FC020020CD000020B8
:1065B0002C080020B201002028090020480D0020EE
:1065C000DB000020D40A00200C0100202C01002058
:1065D00028010020100C01400000C842F0B5404ADC
:1065E000404C1178E9B192F805C01779032104F104
:1065F0001C035E1816F8015CFD4005F00F05072D21
:1066000009D213F801E016F8016C06EA0C060EEB4D
:10661000062644F82560891CC9B21029E9D3002157
:106620001170314907280ED2937863B151782E4A00
:10663000104490F8080149B154F820004FF47771E4
:1066400001EB500006E0B1F81201F0BD34F8200073
:1066500000F5777080B2F0BD70B5214C012605467B
:10666000A67002F05CF8A168421AC4E9020241F285
:1066700088300021824200D9E1701A4AE0781C3249
:1066800015540F2802D0401CE07070BD17482670CA
:10669000018070BD70B504461348114990F810216F
:1066A000032007252AB1012A08D108714D71012064
:1066B00003E002220A7148710020487001234FF460
:1066C000E1320B490B4802F0D5F901460A48C16096
:1066D0000CB10A492160457470BD014800787047CB
:1066E00048030020F80E002094040020DE00002063
:1066F000596600080044004028090020DD650008B4
:1067000070B57C4C06460125207880B902F021F84E
:10671000A1683231884207D32570012002F033F896
:1067200002F017F8A06070BD20780028FBD002F0BE
:1067300010F8A16831448842F5D30020207002F09F
:1067400022F802F006F86C49A060087808B1401EF3
:106750000870657070BDF8B5664D8DF800008DF855
:1067600001108DF802208DF80330A8791DF8001073
:1067700044292DD04C2929D04D2925D04E292AD065
:1067800032240026032806D274B12046FFF7B8FF52
:10679000A879032808D301F0DCFFA968001B884210
:1067A00002D95548AE7106706878012801D0002CD6
:1067B00009D1A879032801D2401CA8716E702E70EF
:1067C000002001F0E0FFF8BD6424DAE7C824D8E730
:1067D0004FF4FA64D5E70024D3E72DE9F047DFF85A
:1067E0001CA10546434C9AF80D004FF00109002604
:1067F00010B184F8029000E0A6704FF40070FBF72F
:1068000044F93F4F18B33F493F484FF0020C91F80D
:10681000B430B0F9000003EB830282420FDA97F83C
:106820000180B8F1000F0AD084F8049091F8B510F7
:10683000194401EB8101814201DA84F804C08242EB
:1068400003DA797809B984F804C000B926712020E8
:10685000FBF706F940B19AF80A1011B99AF80B0043
:1068600008B1F87AA8B1E6702079022814D001287E
:1068700017D0E078012817D0A078012817D0042D70
:1068800019D0022D1ED0012D1ED0607901281ED0F6
:1068900022E084F80390E7E74E22442311464C207F
:1068A0000DE04D234C2208E04D234E2201E04D2304
:1068B0005322532102E044234D224D215320BDE8B1
:1068C000F04748E7442305E044234E22F5E7787873
:1068D00010B14E234D22ECE70748007818B1BDE80F
:1068E000F04732200CE72670BDE8F047002001F0A9
:1068F0004ABF000058030020CC000020300B0020CD
:10690000D40A00202C080020DE000020884201DA92
:10691000084670479042FCDD104670472DE9FE4F57
:1069200097499748E831B0F9E600B1F90050B1F95C
:10693000024010B90DB9002C7ED0924A002111708E
:1069400004F0D4FD904F394604F04EFDDFF83C8250
:10695000414604F07FFD0646284604F0C7FD39464F
:1069600004F042FD414604F075FD0546204604F062
:10697000BDFD394604F038FD414604F06BFD074685
:10698000304605F08BFC0290304606F06DF8019021
:10699000284605F083FC0646284606F065F80546BD
:1069A000384605F07BFC0446384606F05DF800905A
:1069B0002046029904F018FD81463146204604F035
:1069C00013FD80460299009804F00EFD834621468F
:1069D000019804F009FD8246DDE9001004F004FD91
:1069E0006B4C074686F00040C4F80080009904F024
:1069F000FBFCC4E901052946504604F0F5FC594664
:106A000004F09AFCE0602946384604F0EDFC494663
:106A100004F0E7FC20610198314680F0004004F06A
:106A2000E3FC60612946484604F0DEFC394604F088
:106A3000D8FC2946A06100E00BE0584604F0D4FCE5
:106A4000514604F079FCE0613046029904F0CCFC38
:106A50002062BDE8FE8F2DE9F0470546B0F90080C1
:106A6000B0F90260B0F9040004F040FD484C8246E1
:106A7000A16904F0B9FC0746304604F037FD8146B1
:106A8000E16804F0B1FC0646404604F02FFD804664
:106A9000216804F0A9FC314604F04EFC394604F0AC
:106AA0004BFC05F0BBFC28805046E16904F09CFCDF
:106AB00007464846216904F097FC0646404661684F
:106AC00004F092FC314604F037FC394604F034FC03
:106AD00005F0A4FC68805046216A04F085FC074656
:106AE0004846616904F080FC06464046A16804F00F
:106AF0007BFC314604F020FC394604F01DFC05F017
:106B00008DFCA880BDE8F087092A11D2DFE802F0E9
:106B1000100509161C21262A2E0002880A804288A8
:106B200003E042880A8002880CE04A8080888880DE
:106B300014480078002822D108468CE70288524287
:106B40000A8042885242F0E7428852420A80028814
:106B5000EBE7028852420A8042880CE042880A80B1
:106B6000028808E002880A80428803E04288524294
:106B70000A80028852424A8080884042D7E77047A4
:106B80009404002064030020DB0F494000003443DC
:106B9000240F002042490844424990F8080151F866
:106BA00020004FF4777101EB500080B2704770B550
:106BB000044601F0B4FD3C49024640F6C41548685D
:106BC000131A0020AB4200D948704A604A780AB9CB
:106BD0000F2C0AD1087032B1324B20331344182ADB
:106BE00003F8014C02D0521C4A7070BD01220A7099
:106BF000487070BD10B5044629480021294BB0F8F3
:106C000012014200A2F5F76243F82120491C08292D
:106C1000FADB0523254A2649264801F02BFF0146C9
:106C20002548C1600CB1254921600821417410BD7F
:106C30001D4B10B5187840B11A484FF000022030B3
:106C4000817DC908C90702D01A70002010BD1C49F7
:106C5000401C0A8030F8011CC1F30A0411490C6081
:106C60000488C4F3CA044C600468C4F38A348C609A
:106C7000B0F80340C4F34A04CC608488C4F30A1417
:106C80000C614468C4F3CA344C61B0F80740C4F3E3
:106C90008A048C6100894009C8611A70012010BD06
:106CA00094040020480F002068030020A086010003
:106CB000AF6B00080044004028090020956B0008D5
:106CC000DE00002034490844344990F8080151F8A6
:106CD0002000C0F3CF00704710B5044601F01FFD3F
:106CE0002F4900234A68821AB2F57A6F00D94B7097
:106CF00048604878E2B298B1022815D0152802D22F
:106D0000264C183C2254401CC0B248708A78052496
:106D100004EB4202824202D14B700120087010BD88
:106D2000A82CFCD10B70EBE78A70E9E710B504469C
:106D300001234FF4E1321B491B4801F09BFE1B4924
:106D4000002CC86001D01A48206010BD144910B54D
:106D5000087830B1114A0020183A08705378012B96
:106D600001D0002010BD134B18808878082801D965
:106D70000820887000208978084C08E002EB400366
:106D8000B3F803305BBA44F82030401CC0B28842EC
:106D9000F4D3012010BD0000940400209C0F0020BB
:106DA00070030020D96C000800440040280900202E
:106DB000C56C0008DE00002010B5D54C5E28A26826
:106DC00007D05D280CD001461046BDE8104003F006
:106DD00067B95D21104603F063F93E21A068F4E72E
:106DE0005D21104603F05CF93D21A068EDE72DE937
:106DF000F041132000F043F9C64C2068002800DC65
:106E00004042C54D90FBF5F000B200F04AF91B205E
:106E100000F035F92068002800DC40420A2690FB8B
:106E2000F6F042F2107790FBF7F107FB110000B289
:106E300000F037F9232000F022F92068002801DA59
:106E4000532000E04E2000F02CF9122000F017F93A
:106E50006068002800DC404290FBF5F000B200F0D2
:106E600020F91A2000F00BF96068002800DC40428D
:106E700090FBF6F090FBF7F107FB110000B200F079
:106E800010F9222000F0FBF86068002801DA572092
:106E900000E04520BDE8F04100F003B99F4890F8BC
:106EA0002B11002903D1D0F82001FDF768BE7047EF
:106EB0009A4890F82B01002803D14FF41650FDF7A3
:106EC0005EBE7047924810B5806803F0F9F808B1CB
:106ED000002010BD012010BD91494968401A7D284D
:106EE00001D301207047002070472DE9F047FFF7DC
:106EF000E9FF00287ED001F02CFC0246FFF7ECFFF2
:106F0000002877D0864D874FDFF81C826A6028788A
:106F1000DFF81892401C2870002400BF04F1240000
:106F2000C0B200F0ACF8388804F0E9FA064638F947
:106F3000140004F0DBFA314604F08CFA494604F000
:106F400053FA04F0E1FA00B200F0ABF8641C032C31
:106F5000E4DB302000F093F87548008800B200F0C0
:106F6000A0F800F099F828784FF06404800727D142
:106F7000102000F084F86F4E306890FBF4F000B2FF
:106F800000F08FF8212000F07AF8306890FBF4F1DF
:106F900004FB1100002800DC404200B200F081F840
:106FA000142000F06CF86448B0F9000000F079F8A3
:106FB0001C2000F064F8002000F073F800F06CF87A
:106FC0002878400735D1022000F059F85B484FF08F
:106FD0000A08B0F9001091FBF8F000B200F061F877
:106FE0000220FAF752FDE0B100F065F854486E2136
:106FF000007800E041E048431521B0FBF1F63A206B
:1070000000F03DF8B6FBF4F738B200F04AF83B2048
:1070100000F035F804FB1760401DB0FBF8F000F0FD
:1070200040F82020FAF71CFD08B1FFF7E0FE00F061
:1070300033F82878282820D10020287001F089FB17
:107040004FF47A71B0FBF1F43C25B4FBF5F6B6FBD6
:10705000F5F005FB1067172000F011F8380200B2B8
:1070600000F01FF8182000F00AF805FB164000F0A9
:1070700018F8BDE8F04700F00FB8BDE8F08770B52C
:10708000234C05465E21A06803F00AF82946A06853
:10709000BDE8704003F004B81D485E21806802F02E
:1070A000FFBF10B50446C0B2FFF786FEC4F3072049
:1070B000BDE8104080E670B52148224E40F634020B
:1070C00000783178164DB0FBF1F050432A22B0FB26
:1070D000F2F06A88B2FBF1F301FB13214FF6FF7265
:1070E00002EA011141EA0024C0F303200443062010
:1070F000FFF7C5FF20B2FFF7D4FF68883178401C46
:1071000080B2B0FBF1F201FB1200688070BD00009C
:10711000280900204C010020A086010094040020D2
:1071200078030020820100208200002000007A44C1
:107130002C00002020000020B0010020EA000020E8
:10714000DA000020680100204D4890F82A0108B1BB
:107150000020704701207047494890F82A01012813
:1071600000D00020704710B54FF40060FAF78DFC96
:10717000002812D04020FAF788FC414928B991F83C
:107180002B0101280AD0022808D0FFF7E5FF18B12B
:1071900091F82B01002800D0012010BD002010BD67
:1071A00010B5FFF7D1FF08B1FFF778FEFFF7D4FF66
:1071B000002803D0BDE8104000F00AB910BD3049E6
:1071C000012091F82B21002A07D191F82C0128B138
:1071D0002C48007D002800D0012070472A484078C4
:1071E000F8E770B5294D2878002814D0FFF7E7FF9D
:1071F0000446687884420ED054B1FFF7A5FF08B169
:10720000FFF756FEFFF7A8FF20B100F0DCF801E021
:10721000FFF7C6FF6C7070BD10B54020FAF735FC63
:10722000174C10B9002084F82B01FFF79CFF174979
:10723000087094F82B111648012906D0022906D0AF
:1072400001688160BDE81040CBE71249F9E71249B7
:10725000F7E70E4810B50078002810D0FFF7AFFF11
:1072600000280CD0FFF770FF08B1FFF73EFEFFF7D4
:1072700073FF002803D0BDE8104000F0AEB810BD89
:1072800094040020300B0020D40A0020800300204A
:1072900028090020E41500202C1800202DE9F047D3
:1072A0007F4F0D4680460221B86802F015FF002688
:1072B00034464FF47A796D1E0BE000BF18F80400D5
:1072C00081198EB200F0BCF8484601F045FA641C02
:1072D000E4B2AC42F2DBF0B200F0B2F8484601F0A2
:1072E0003BFAB868BDE8F047012102F0F5BEF0B501
:1072F0006C4801786C4881766C49C97A00295ED067
:107300006B4C662180F8291022686A4DD10F4172BA
:1073100092FBF5F1684BC9B24B4302EB431202EB0F
:107320004202530042F21072B3FBF2F702FB173332
:10733000FEB201EBC10707EB011106EB810181727F
:10734000090AC1720373190A417363685A4CD90F51
:10735000817393FBF5F1C9B24C4303EB441303EB88
:1073600043035B00B3FBF2F502FB153201EBC103F3
:10737000ECB203EB011104EB8101C173090A017442
:107380004274110A81744D4964220988B1FBF2F1FB
:1073900001EBC1014FF6FF7202EA8101C171090AD6
:1073A000017247490988C174090A0175454909886C
:1073B0004175090A8175444909780177F0BD20219A
:1073C00080F82910F0BD36480121806802F084BEA3
:1073D00033480321806802F07FBE70B5304C29E04D
:1073E000A06802F070FE0546052001F0C1F98A2D63
:1073F00002D08E2D1ED11BE02020FAF731FBC8B140
:107400002C21294803F00AFF27487C2101708A219A
:107410004170A021C1707D2180F82B100021817066
:107420000171FFF764FF2C211F48FFF737FF01E0D0
:1074300000F00BF8A06802F043FE0028D0D170BD28
:1074400001461748806802F02BBE174810B52E2160
:107450002C3003F0E3FE14487C212C301B4A0170D1
:107460008E214170E021C1707D2180F82C10002117
:107470008170017112788277C1770275417514228B
:107480000276427681834FF4FA7141834821418428
:10749000782180F82410BDE810402E21FEE600007F
:1074A00028090020DB000020BC0F0020D40A0020A7
:1074B0004C010020A0860100CBF3FFFF78010020E3
:1074C000720100207601002074010020DA00002003
:1074D0002DE9F0410646007890B008B1012500E0A2
:1074E0000025DFF8D880404602F0C8FF34480090FD
:1074F00000243448CDE90104012725B10220CDE95B
:107500000304802002E0CDE90374002005904FF4CD
:107510008070069080000790202008900002CDE93E
:1075200009046946404603F016F80121404603F07D
:107530003CF88DF830500B948DF831704FF460208A
:10754000CDE90D040DB1022000E001201C4C8DF8A6
:107550003C004C3C0BA9204602F0FCFE0323012218
:107560000421204602F04BFF2DB131780323022283
:10757000204602F044FF0121204602F014FF0121C1
:10758000204602F006FF204602F017FF204602F0D8
:1075900019FF0028FAD1204602F01BFF204602F016
:1075A0001DFF0028FAD10121204602F01EFF10B075
:1075B000BDE8F081034931F810007047080002402F
:1075C0004C240140820300202DE9FF47DFF86C8145
:1075D000814698F80000D0B300273E463D463C4621
:1075E000641CE4B202AB08223221532000F063FD98
:1075F0009DF808009DF80910202C00EB012000B236
:1076000007449DF80A009DF80B1000EB012000B222
:1076100006449DF80C009DF80D1000EB012000B20F
:1076200005449DF80F0000F07F0001D20028D7D15B
:1076300097FBF4F0ADF8000096FBF4F0ADF8020013
:1076400095FBF4F0ADF8040088F802401EE0FFE777
:1076500002AB06223221532000F02DFD9DF80800D8
:107660009DF8091000EB0120ADF800009DF80A001C
:107670009DF80B1000EB0120ADF802009DF80C0006
:107680009DF80D1000EB0120ADF8040098F80120E2
:1076900049466846FFF738FABDE8FF8770B5274DC1
:1076A00004464FF0080228784FF02D0100284FF0D3
:1076B00053000ED000F0F9FC0A223121532000F0D3
:1076C000F4FC0C222C21532000F0EFFC90223821F6
:1076D00008E000F0EAFC0A223121532000F0E5FC2A
:1076E0000A222C21532000F0E0FC154940F2091039
:1076F000002C088000D06C7070BD38B505460020A5
:107700008DF800000F480C460F49006888420AD0E7
:107710006B4601220021532000F0CDFC18B19DF8EA
:107720000000E52801D0002038BD04492878087001
:107730000648206006486060012038BD86030020AE
:107740008201002030040020001BB7009D76000855
:10775000C975000810B54FF48044204602F082FF3E
:10776000012805D1204602F08BFFB949012008709D
:1077700010BD70B50D46B649B64A0646888853898D
:10778000B2F91440C01A13895843B2F91230C01329
:10779000DB02044493FBF4F31844D06100EB800057
:1077A000082202EB40000411886800F0D0F806B10E
:1077B0003060002D00D02C6070BD38B5A44C20780E
:1077C00010B96088401C60806B460322F621772048
:1077D00000F071FC9DF800009DF80110000440EAE3
:1077E00001209DF8021008439A49B1F92010C1F117
:1077F0000801C840A06038BD9648342190F82000A8
:1078000001EB80109249C2B200200870F421772069
:1078100000F04BBC38B58E4C207810B96088401C05
:1078200060806B460222F621772000F044FCBDF810
:10783000000040BAA08038BD854900202E22087083
:10784000F421772000F031BC2DE9F0430446824852
:10785000824985B00068884203D1002005B0BDE8A8
:10786000F083DFF8EC9199F8010008B10120F5E709
:107870004FF40055ADF80C5002208DF80F00102089
:10788000774E8DF80E0003A9304601F067FF6F00B8
:10789000ADF80C7004208DF80E0003A9304601F0FD
:1078A0005DFF35610E21022001F08EFF00208DF872
:1078B000080008208DF809004FF00108019747469D
:1078C0008DF80A8001A802F097FE28208DF810009C
:1078D0000F208DF811008DF812008DF8137004A898
:1078E00002F005FD142000F043FF6B460122D02179
:1078F000772000F0E0FB574F9DF800000321F8755A
:107900003984552801D07561A7E76B460122D12142
:10791000772000F0D0FB9DF8000000F00F013976D1
:107920000009787600F05CF889F8018041F2707007
:10793000208046F6781060804A4860604A48A0601F
:107940004A48E0604A4820614A4860618EE770B565
:107950004049CA69B1F90E40A2F57A6202FB02F30E
:107960001D136C43E512B1F90240B1F904605443B0
:1079700005EBE424B1F9005004EB850591F82040B3
:10798000A54056437213B1F90C601B135E4302EB22
:107990002642921C9210C98802F50042AD1C514348
:1079A000C90B4CF25032A0EBA500E2405043B0F1BD
:1079B000004F03D24000B0FBF1F002E0B0FBF1F069
:1079C00040000112494340F6DE3251432A4A09146D
:1079D000424301EB224101F6CF6100EB211070BD63
:1079E00000B587B06B461622AA21772000F063FB12
:1079F000BDF8000041BA17480180BDF8021049BA2D
:107A00004180BDF8041049BA8180BDF8061049BA1A
:107A1000C180BDF8081049BA0181BDF80A1049BA01
:107A20004181BDF80C1049BA8181BDF80E1049BAE8
:107A3000C181BDF8101049BA0182BDF8121049BACF
:107A40004182BDF8141049BA818207B000BD000020
:107A50008C0300201810002030040020001BB70009
:107A6000001001403978000815780008F9770008FF
:107A7000BB7700087377000843E3FFFF38B504467F
:107A800000208DF800006B4601220A211E2000F024
:107A900012FB18B19DF80000482801D0002038BD25
:107AA0000CB18D480470012038BD7FB5054602AB8E
:107AB000062203211E2000F0FEFABDF8080040BA9D
:107AC00000B203F013FD844C241D216803F08CFCEC
:107AD00003F01AFDADF80000BDF80A0040BA00B28C
:107AE00003F004FDA16803F07FFC03F00DFDADF889
:107AF0000400BDF80C0040BA00B203F0F7FC616866
:107B000003F072FC03F000FDADF80200201F2946CF
:107B100002786846FEF7F8FF7FBD2DE9F0476F4811
:107B200000246F49006825468EB02E464FF00108AC
:107B300088420CD14FF48050ADF8280002208DF817
:107B40002B0004208DF82A000AA9664808E066493F
:107B5000884207D14FF48040ADF828000AA9634855
:107B600001F0FCFD322000F003FE112200211E2056
:107B700000F09BFA602201211E2000F096FA64209A
:107B800000F0F6FD6846FFF790FFDFF858A1DFF838
:107B9000609100270AF10C0A012202211E2000F048
:107BA00084FA322000F0E4FD6846FFF77EFFBDF95D
:107BB0000210BDF90400BDF900200D441444064430
:107BC000814201DA0B4600E00346934201DD104694
:107BD00002E0814200DA0846484502DC4FF0000826
:107BE00008E0DAF8001081F01001CAF800107F1CDC
:107BF0000A2FD1DB122200211E2000F056FA0027A6
:107C0000012202211E2000F050FA322000F0B0FDC7
:107C10006846FFF74AFFBDF90020BDF90210BDF923
:107C20000400A41A6D1A361A814201DA0B4600E0EC
:107C30000346934201DD104602E0814200DA084625
:107C4000484502DC4FF0000808E0DAF8001081F047
:107C50001001CAF800107F1C0A2FD1DB204603F068
:107C600045FC244F0146384603F0F4FB1A4C20F043
:107C70000040241D2060284603F038FC01463846A9
:107C800003F0E8FB20F000406060304603F02EFC7B
:107C90000146194803F0DEFB20F00040A06070228E
:107CA00000211E2000F001FA202201211E2000F0F8
:107CB000FCF9002202211E2000F0F7F9642000F0F8
:107CC00057FDB8F1000F04D14FF07E502060606086
:107CD000A0600EB0BDE8F0879803002030040020BB
:107CE00000127A00000C0140001BB7000010014098
:107CF00000F0FFFF00406F4601C05E4630B587B020
:107D000005464FF44060ADF8140002208DF81700CE
:107D10001C208DF8160005A9FB4801F01FFDFB4C47
:107D2000E56000F007FAE06802F0B0FC684602F097
:107D300018FD00224FF44071E06802F048FD002574
:107D4000ADF804504BF6FF70ADF806004FF48040DC
:107D5000ADF80C00EE4800900121E06802F00FFD44
:107D60006946E06802F0A5FC4FF4A06002F0BAFAA0
:107D700022208DF810008DF811508DF8125001203E
:107D80008DF8130004A802F0B2FA21208DF810003B
:107D90008DF8115004A802F0AAFA07B030BD38B52A
:107DA000DA4CE068818A009111F4706F01D00121F2
:107DB0002170009911F4E06F25D0018B00224FF45F
:107DC000806102F004FD009880051CD4E068018801
:107DD000890518D40188C9050CD50188C905FCD4CA
:107DE000012102F0E0FCE06801888905FCD4FFF77E
:107DF00085FF08E0012102F0D6FC00224FF440711B
:107E0000E06802F0E4FCE068818A21F4706181821C
:107E10000020207138BDC2E72DE9F041BB4CE0687D
:107E2000818A4FF00105C9B2CA074FF0000627D07A
:107E3000018821F400610180012102F0BEFCE6709E
:107E4000607A20B1607860B9A079FF2809D06179A3
:107E50000022E06802F0C8FCA079FF2848D0FF208B
:107E6000C9E06570E079022804D1E068018841F436
:107E70000061018061790122E06802F0B5FC37E021
:107E80008A074FF4806745D5BFF3508FE07901280A
:107E900010D1607A70B1607860B10021E06802F0C2
:107EA0008CFCBFF3508FE068018B012102F07BFC5A
:107EB000A57018E0E068008BBFF3508FE0790228CE
:107EC00008D1607A30B1607820B10021E06802F01A
:107ED00074FC06E0E079032805D1607A18B1607877
:107EE00008B1002200E001223946E06802F06FFC90
:107EF00094F90310E079401C814209D16670A078A2
:107F000028B100224FF44071E06802F060FC267155
:107F1000BDE8F0814A0753D5A570627A7B4949785C
:107F2000CAB3C9B3E17902291FD9002102F045FC87
:107F3000E06802F056FC94F9031062695054491C41
:107F4000E1700121E06802F02EFCA570E06802F00B
:107F500048FC94F9031062695054491CE1700122F5
:107F60003946E06802F033FC25E0012102F01BFCF9
:107F7000E06802F036FC94F9031062695054491C21
:107F8000E170E06802F02DFC94F90310626950542E
:107F9000891CE1700FE000E000E009B9217A31B1FD
:107FA000012102F000FCE078401CE07003E00121B8
:107FB00002F0EFFB6570E0680188C905FCD497E723
:107FC0004A061AD502F00DFC94F903106269505468
:107FD000491C48B2E070E179C01C814204D1002202
:107FE0003946E06802F0F3FBE17994F9030081423D
:107FF000E5D100F10100E0707AE70906DFD594F9D8
:1080000003104B1C5AB20BD02369595CE27002F08A
:10801000E6FBE07994F9031088423FF45AAF67E732
:10802000E270A17902F0DBFB607A00287FF451AFA7
:10803000E0790028F1D05BE7EEE6B0E6ECE670B55B
:10804000324C4FEA400047F230556071A171012077
:1080500020720021617223616361E27120712170DD
:10806000E068818889050ED40188C90505D4018896
:108070008905FCD4012102F08CFB01224FF44071F0
:10808000E06802F0A4FB207910B16D1EFBD104E082
:108090001DB1207880F0010070BD6089401C6081B6
:1080A000E068FFF72BFE002070BD07B502AB012290
:1080B000FFF7C5FF0EBD70B5144C4FEA400047F204
:1080C00030556071A17100202072012161726361DD
:1080D0002361E27121712070E068818889050ED4E6
:1080E0000188C90505D401888905FCD4012102F065
:1080F00050FB01224FF44071E06802F068FB2079E8
:1081000040B16D1EFBD10AE0000C0140A803002025
:10811000801A06001DB1207880F0010070BD6089D2
:10812000401C6081E068FFF7E9FD002070BD2A482F
:10813000408970472DE9F84F4FF44067ADF8007063
:108140004FF0020A8DF803A01420DFF890B08DF8EC
:1081500002006946584601F001FB204D10352F60A2
:10816000DFF8789000262C1505F1040809F10809BC
:1081700002E00A2000F0F0FAD9F800004005F8D536
:10818000C8F800400A2000F0E7FA2C600A2000F04E
:10819000E3FA761CF6B2082EEED34FF40069464699
:1081A000C8F800900A2000F0D7FA34600A2000F0E6
:1081B000D3FA2C600A2000F0CFFAC5F80090ADF891
:1081C00000708DF803A01C208DF802006946584607
:1081D00001F0C4FABDE8F88FA8030020000C0140AC
:1081E00038B504466B4602221B216820FFF763FF67
:1081F000BDF8000043F2903140BA08444FF48C714E
:10820000B0FBF1F02330208038BD1FB5044602AB2F
:1082100006221D216820FFF74EFFBDF80800214609
:1082200040BA02B2D01702EB90708010ADF8000097
:10823000BDF80A0040BA02B2D01702EB907080106D
:10824000ADF80200BDF80C0040BA02B2D01702EB44
:1082500090708010ADF804002F4842786846FEF711
:1082600053FC1FBD70B50446192000F081FA0022AE
:1082700015216820FFF719FF10B9032000F024FB37
:10828000254D1621287840F018026820FFF70DFFD1
:10829000002217216820FFF708FF01223D216820F6
:1082A000FFF703FF01223E216820FFF7FEFE002CAE
:1082B00000D06C7070BD70B504460D46192000F0FA
:1082C00057FA002215216820FFF7EFFE00281CD086
:1082D00012482060124860601248A0601248E060B6
:1082E0000D48622D12D004DC0A2D13D0142D05D1B7
:1082F0000EE0BC2D06D0B5F5807F01D0032102E051
:10830000002100E001210170012070BD0221FAE787
:108310000421F8E70521F6E7C00300206582000884
:108320000B820008E181000818449231FEB5064630
:1083300014460D46684602F031FD0120ADF80400F8
:108340000021ADF80050ADF80610ADF80810ADF8FA
:1083500002406946304602F071FCFEBD2DE9F04155
:108360001646E14A1F4602EB0015E04A02EB0014F4
:108370000A463146206801F02EFBD4E9010118229B
:1083800000F0A5F9217B3A46206800F05DF9A07B5A
:1083900018B10121206802F013FD0121206802F0CC
:1083A00005FD207B30B1042807D008280CD00C280C
:1083B00006D10CE02068343001E0206838302860B5
:1083C000AE802846BDE8F08120683C30F7E72068A1
:1083D0004030F4E72DE9F0410546C3480F4600EB75
:1083E0000516C248B27100EB05142822D4E9010138
:1083F00000F06DF9217B00222068FFF797FF012232
:108400004FF6FF71204601F003FB3A46294620460D
:1084100001F0C4FA3046D5E770B5B54800240289AA
:1084200042810181891A8BB240F68C218B4201D99D
:10843000C47070BDAE49A3F2EF2540F2DB56AD4AE1
:10844000C978B5421BD2082919D2A74DE0350429B5
:1084500025F8113007D2C588AB4204D9012305792C
:108460008B402B43037103790F2B08D10471B2F9B0
:108470000030142B02DD143B138000E01480491CF3
:10848000C170148070BD70B5974A984B02EB001212
:1084900003EB0013D47918681B7B8CB151811489CC
:1084A000914D091B91819479E03525F81410002431
:1084B000D47122461946FFF739FF8E48048070BDFB
:1084C00011810121D171BDE87040022219462DE7CA
:1084D000854AA1F57A71F03252F82000828800684E
:1084E0004A434FF47A7192FBF1F1018070477E4A62
:1084F000F03252F820000068018070472DE9F04109
:1085000004467B4D218A0020E980A17901B1022037
:10851000617801B1401C784900264FF4FA7851F88F
:108520002070BA5D02F00F0002F0F001FF2A6CD05B
:10853000A2781AB1022865D0032863D0E2783AB154
:1085400004285FD005285DD006285BD0072859D0C5
:10855000E2790AB1824255D011F0300F02D0227870
:1085600002B90021227932B1A27922B9082801D0BA
:10857000092800D1802162792AB1A2791AB9021F93
:10858000032A00D88021CA0605D500225B49FFF7DF
:1085900021FF082008E08A0608D5AA785849FFF785
:1085A00019FFA87800F10100A8702BE04A0617D542
:1085B0002389434501D9082100E00121514A4A435A
:1085C000B2FBF3F292B2A389FFF7C8FE0146464A16
:1085D0002878F03242F8201000F10100287011E0F4
:1085E00009060FD56189474AE389B2FBF1F18AB2E6
:1085F0000121FFF7B3FE0146434A687842F8201094
:10860000401C6870761C0E2E8BDB4048E860208989
:10861000404501D93E48E8600020D3E6344A13784B
:10862000984201D2D26810477047314A527890423E
:1086300004D2354A52F82000006801807047324960
:10864000403931F8100070477FB5064615460C4694
:10865000684602F099FB7020ADF800000120ADF8EB
:1086600002000020ADF804000220ADF80800C001AF
:10867000ADF80650ADF80C0074B1042C15D0082CE0
:108680001CD00C2C07D16946304602F023FA082191
:10869000304602F0BEFB7FBD6946304602F06FF9FE
:1086A0000821304602F09FFB7FBD6946304602F04C
:1086B0009BF90821304602F09CFB7FBD694630469D
:1086C00002F0CEF90821304602F09DFB7FBD08B5CF
:1086D000ADF800108DF8022002218DF803106946D4
:1086E00001F03CF808BD00003C1000201CDD000833
:1086F000C4030020DE000020DCDC00081984000830
:108700008784000840420F005C110020EF840008BD
:10871000D184000881484168491C4160704710B508
:108720007E484FF0E02341689A694468A142FAD13B
:108730000368006803EB4304C4EBC313C2EBC3023A
:10874000B2FBF0F001EB4102C2EBC11100EBC10042
:1087500010BD72484068704730B50546FFF7DFFF2F
:108760004FEA0004FFF7DBFF001BA842FAD330BD3D
:1087700030B504464FF47A7502E02846FFF7ECFF67
:10878000641EFAD230BD6549896808474FF48051AC
:1087900008B1634801E06248001F016070474FF470
:1087A000805110B15E48001F00E05D4801607047D5
:1087B0002DE9F04F8DB0044618225A49684602F060
:1087C00014FD0327204601F0D6FC0121564802F093
:1087D00071F8012144F61D2002F063F801210846DA
:1087E00002F056F802F081F84FF6FF70ADF818006D
:1087F0004B484FF0000A8DF81AA006A9143800F073
:10880000ADFF06A9494800F0A9FF06A9484800F0B5
:10881000A5FF4848416841F000714160464DDFF8CE
:108820001C813E4E2968414501D1454800E045483C
:10883000B0600020FFF7A7FF3C4908201031086016
:1088400010200860A946002483466D46D9F8001020
:10885000414506D105EBC4008179142901D180F886
:1088600006B005EBC401091D55F8340000F076FF91
:10887000641CBC42EAD307A801F0C4FF3249079840
:10888000B0FBF1F0306031484FF47A710068B0FB12
:10889000F1F0B0F1807F0CD220F07F414FF0E0206A
:1088A000491E41612A4AF0211170C0F818A0072121
:1088B00001612848FFF722FA00F0CFFF6420FFF79C
:1088C00057FF0DB0BDE8F08F184A10211432116027
:1088D0000821121F11600446151F40F2DB104443AB
:1088E000286880F010002860286880F00800286060
:1088F000A01EFFF73DFF0120FFF745FF1920FFF7FE
:1089000037FF0020FFF73FFFEAE710B11349124895
:1089100008600F491248173908607047D4030020D7
:1089200014080140ECDC000807004000000C014086
:10893000001001400000014030040020001BB7007F
:108940009F8700088D87000840420F002C040020FC
:1089500023ED00E000580040EFBEADDEF04F0020F8
:108960000400FA057CB5F74C0D46F7492160A0607C
:10897000A4F53070606100F58070A0614FF48070E4
:10898000E0602061F1482063F04801211438606301
:10899000880301F086FF02208DF803000002ADF885
:1089A000000018208DF80200E94EA80703D569469B
:1089B000304600F0D3FE4FF48060ADF80000482050
:1089C0008DF80200E80703D06946304600F0C6FE85
:1089D0000E208DF8040001208DF805008DF80600AA
:1089E0008DF8070001A801F082FC20467CBD2DE92E
:1089F000FC41D44C0D464C34D3492160A06080200A
:108A0000E06040202061A4F5867060618030A06144
:108A1000D0480121A064480401F04CFF02268DF8E3
:108A200003600420ADF8000018208DF80200C84F44
:108A3000A80703D56946384600F090FE0820ADF837
:108A4000000048208DF80200E80703D06946384648
:108A500000F084FE26208DF8040001208DF805002A
:108A60008DF806608DF8070001A801F040FC204653
:108A7000BDE8FC812DE9F04389460746B64900244C
:108A8000B4488FB01E4690468F4204D11946104616
:108A9000FFF768FF05E0874204D119461046FFF74B
:108AA000A6FF044600252562E561A562C4F82C9066
:108AB000A76465622671C4F80880CDF82C80ADF8F3
:108AC0003050700707D54FF40050ADF83200C01099
:108AD000ADF8340003E0ADF83250ADF83450ADF8E5
:108AE0003850ADF83650F00702D00420ADF836000B
:108AF000B00705D5BDF8360040F00800ADF83600E7
:108B00000BA9384602F0AEF90121384602F002FA0C
:108B1000684601F03DFD381D00904FF48050CDE9CE
:108B2000090580200495CDE905050795F00723D0B8
:108B3000206BD8B1E068CDE9025020200890606930
:108B40000190206B01F09AFC6946206B01F003FD57
:108B50000121206B01F029FD01224021384602F05D
:108B6000FBF9206B01F036FD206405E0012240F2A4
:108B70002551384602F0D8F9B00724D5606BE0B132
:108B800020690390102008950290606B01F076FC3C
:108B90006946606B01F0DFFC01220221606B01F08D
:108BA0000FFD0021606B01F013FD606B4560012239
:108BB0008021384602F0D0F905E0012240F2277109
:108BC000384602F0B1F90FB02046BDE8F0837FB51A
:108BD00004460020ADF80400ADF808000091ADF89F
:108BE0000600ADF80C00ADF80A0020790D46C0076C
:108BF00002D00420ADF80A002079800705D5BDF821
:108C00000A0040F00800ADF80A006946A06C02F0C6
:108C100029F9A5607FBD7047826A81691144426B62
:108C2000D160D0E9092100238A4205D9511A426B4B
:108C30005160416A816204E00269511A426B5160DD
:108C4000836280F84430406B012101F0AEBC016BBF
:108C500011B14968006C01E01C3003C8814201D0A9
:108C60000120704700207047416B11B190F844001B
:108C70007047243003C8814201D101207047002091
:108C8000704710B50146036BC268406943B10B6C75
:108C9000D21A805C5B1E0B6401D1CA680A6410BDE5
:108CA0000B6AC05C5B1CB3FBF2F402FB14320A6279
:108CB00010BD436A8269D154416A0269491CB1FB03
:108CC000F2F302FB13114162416B19B10968C90744
:108CD00006D1A1E7806C012240F2277102F024B98D
:108CE000704710B5174C4FF4005001F076FC00218E
:108CF000606B01F05AFCD4E90901884203D0204698
:108D0000BDE8104088E7012084F8440010BD0D49FB
:108D1000886C028812060ED5D1E909329A420BD02E
:108D20008B699A5C8280886A0A69401CB0FBF2F306
:108D300002FB130088627047002240F2277102F0A4
:108D4000F3B800003C14002004DD00085800024085
:108D500000080140004400400038014070B5184C44
:108D6000A06C0588A90610D58088E16A09B18847FA
:108D70000BE0E26961698854E069E16800F1010093
:108D8000B0FBF1F201FB1200E06128060FD5D4E937
:108D9000091088420CD0A169085CA16C8880A06A87
:108DA0002169401CB0FBF1F201FB1200A06270BD12
:108DB000A06CBDE87040002240F2277102F0B4B808
:108DC00088140020FEB52C4C0125207878B10128AC
:108DD00023D0022820D164208DF8000027488DF888
:108DE000015000264078E0B38DF802503CE07A2034
:108DF0008DF8000022486B460222B0F90000FF21E6
:108E0000C0F1B40000EBD070C0F347008DF8010052
:108E10006D20FFF714F92570FEBD1A4E79208DF8EC
:108E20000000B6F900000A2590FBF5F05A30B42294
:108E30000021FDF76BFD8DF80100B6F90200B422A8
:108E400090FBF5F05A300021FDF760FD8DF802002F
:108E50006B460322FF216D20FFF7F1F802202070FE
:108E6000FEBDFFE78DF802606B460322FF216D20F7
:108E7000FFF7E5F82670F3E7E0030020D40A0020AE
:108E8000B0010020340000201FB5044602AB0622CA
:108E900043216820FFF70FF9BDF80800214640BACA
:108EA00002B2D01702EB90708010ADF80000BDF850
:108EB0000A0040BA02B2D01702EB90708010ADF8F1
:108EC0000200BDF80C0040BA02B2D01702EB90705D
:108ED0008010ADF804007C4842786846FDF714FE27
:108EE0001FBD38B504464FF40050ADF80000022015
:108EF0008DF8030004208DF802007448744900685E
:108F0000884202D16946734804E07349884203D11C
:108F10006946724800F022FC80226B216820FFF72E
:108F2000C4F80520FFF724FC002219216820FFF770
:108F3000BCF803226B216820FFF7B7F80222372123
:108F40006820FFF7B2F8604D1A2168202A78FFF7F1
:108F5000ACF818221B216820FFF7A7F810221C216B
:108F60006820FFF7A2F8002C00D06C7038BD1FB548
:108F7000044602AB06223B216820FFF79CF8BDF8AF
:108F80000800214640BAADF80000BDF80A0040BA1A
:108F9000ADF80200BDF80C0040BAADF804004A4834
:108FA00082786846FDF7B0FD1FBD47494C4ACB7833
:108FB00013B14FF4FF6301E04FF480531380002896
:108FC00000D0887070472DE9FE4F81469846924642
:108FD0000D462320FFF7CCFB6B460122752168204C
:108FE000FFF769F8002804D09DF80000682802D037
:108FF0000020BDE8FE8F062201AB11466820FFF776
:109000005AF89DF809009DF80710C007400F01F0BD
:10901000010140EA41009DF805102B4C01F00101CF
:1090200008434FF001064FF0000704D0012833D069
:1090300002280DD02CE06B4601220C216820FFF79E
:109040003AF89DF8000010F00F0021D0042823D03A
:10905000E7702449C9F8001023492448C9F80410CE
:109060002860234868602348E860B8F1000F02D008
:10907000E17888F800105046BAF1620F19D00DDC83
:1090800005281ED00A281AD0BAF1140F0BD114E00B
:109090000520FFF719FCDCE7E670DAE7BC2806D00C
:1090A000BAF5807F01D0032004E0277003E026702A
:1090B00001E00220207001209BE70420FAE7052050
:1090C000F8E70620F6E70000E10300203004002066
:1090D00000127A00000C0140001BB7000010014094
:1090E00082010020AB8F00086F8F0008E38E00081C
:1090F000898E0008194492311FB5044602AB06223E
:1091000001211C20FEF7D7FFBDF80800214640BA18
:1091100040F38D02D01702EB90708010ADF8000084
:10912000BDF80A0040BA40F38D02D01702EB9070F0
:109130008010ADF80200BDF80C0040BA40F38D027B
:10914000D01702EB90708010ADF80400334802781D
:109150006846FDF7D9FC1FBD38B504462020ADF8A0
:10916000000002208DF8030004208DF802006946FB
:109170002B4800F0F3FA00222A211C20FEF795FF6D
:1091800002220E211C20FEF790FF03220F211C203B
:10919000FEF78BFF12222B211C20FEF786FF0222F6
:1091A0002C211C20FEF781FF01222D211C20FEF71F
:1091B0007CFF00222E211C20FEF777FF05222A21AA
:1091C0001C20FEF772FF17494FF48070002C0880B6
:1091D00001D01248047038BD38B5044600208DF81F
:1091E000000011481149006888420CD06B460122EA
:1091F0000D211C20FEF75FFF28B19DF800002A28F2
:1092000003D01A2801D0002038BD0949216009493E
:10921000616002494870012038BD0000E50300206C
:10922000000801408201002030040020001BB7002C
:1092300059910008F9900008434810B50068434C64
:10924000A188084203D0FFF76AFAA0600AE0FFF79E
:1092500066FAA168884205D9401A3B2190FBF1F0DB
:1092600061690860E068BDE8104001F009BAE3E711
:10927000E2E7FEB50125354C022110B1012810D1DD
:1092800009E04FF4807060804000A080E060092019
:109290002070172004E06580A180E1602570072020
:1092A00060706088ADF800001026274F8DF80260CE
:1092B0008DF80310083F6946384600F04FFAA08841
:1092C000ADF8000004208DF802006946384600F031
:1092D00045FA2178012000F077FAE06801F0D0F932
:1092E000E068019000208DF808008DF809608DF885
:1092F0000A5001A801F080F994F9010000F01F0163
:109300008D4040094FF0E02101EB8000C0F8005192
:10931000FFF71FFA3C382061FEBD70B50546FFF728
:1093200018FA0A4C21693C3188420CD3C4E904057F
:1093300005496088083108600B20FFF70DFA0249E3
:1093400060880C31086070BD080C0140E803002003
:109350001FB5044602AB0622A8216820FEF7ABFE2B
:10936000BDF80800214640BA02B2D01702EB907057
:109370008010ADF80000BDF80A0040BA02B2D01764
:1093800002EB90708010ADF80200BDF80C0040BAFE
:1093900002B2D01702EB90708010ADF8040026489E
:1093A00042786846FDF7B0FB1FBD70B504466420E7
:1093B000FFF7DEF9F02223216820FEF776FE10B9D0
:1093C0000320FFF781FA0520FFF7D2F91A4D20217B
:1093D000287840F00F026820FEF767FE002C00D0CE
:1093E0006C7070BD38B504460D461920FFF7C0F902
:1093F0006B4601220F216820FEF75DFE9DF80000FC
:10940000D32801D0002038BD0C4820600C48606093
:109410000C48E0600848362D05D04E2D07D05D2D54
:1094200007D0002100E040210170012038BD8021DB
:10943000FAE7C021F8E7000000040020AB93000821
:1094400051930008DDE9A7312DE9F04FB74C834671
:109450008E46608926890102B5484FF0000A4068AF
:10946000421AA6FB027CA0884FEAE2754FEA10413F
:109470004FEA00430AFB02C006FB05064FEAD7107D
:1094800040EA466013EB000941EBE611E688638889
:10949000A6FB02C84FEA53404FEAC3370AFB0283D8
:1094A00006FB05364FEA1C2343EA0663FB1840EB34
:1094B0002620A689A6FB027C0AFB02C206FB052425
:1094C0004FEAD75242EA44224FF4FA654FEAE45495
:1094D000521944F10004A246551B74F1000448DA05
:1094E000944D5519A5FB05674AF1FF3404FB057738
:1094F00005FB047C0525A6FB05480CFB058500271C
:1095000006FB07556F104FEA340CB9EB0C0961EB01
:109510000701A40844EA85741B1B60EBA500864D77
:10952000551B7AF1FF3424DA40F2DC555619A6FBBC
:1095300006474AF1000505FB067706FB0575072679
:10954000A4FB06C805FB0686002704FB0767B9EBEA
:109550000C0961EB07010B27A4FB07C805FB078576
:10956000002604FB065464104FEA3C055B1B60EBCD
:1095700004006F4CA5680024A5FB036704FB03737C
:1095800005FB0030740D44EAC0244015B4EB090318
:1095900060EB0100410441EAD330BBF1000F01D080
:1095A000CBF80000BEF1000F01D0CEF80020BDE8DE
:1095B000F08F10B500F072F85D49886010BD5C480E
:1095C000012200784030C1B27720FEF76EBD10B5A1
:1095D00000F064F85649486010BD554801220078F3
:1095E0005030C1B27720FEF760BD2DE9FE4305463D
:1095F00052485349006888420FD04FF40054ADF8E8
:10960000004002208DF8030010204E4E8DF802001D
:109610006946304600F0A2F874610A20FFF7A8F806
:1096200001AB0122A0217720FEF745FD002823D0C1
:1096300001221E217720FEF738FD4FF42F60FFF73F
:109640008BF80024DFF8E4802646A02707EB4400CF
:10965000C1B202AB022277200296FEF72CFDBDF8C4
:10966000080040BA28F81400641C082CEEDB2F48D0
:1096700000F026F810B10020BDE8FE8342F2107021
:1096800028806880304868603048A8603048E860CA
:1096900030482861304868610120EDE708B56B4625
:1096A000032200217720FEF706FD9DF800009DF8BB
:1096B0000110000440EA01209DF80210084308BD93
:1096C000F0B5C289002102F47F4502F00F040123A6
:1096D000C5810A4630F8126006B10023521C082AE0
:1096E000F8DB4FF0FF36F3B90022D30722F0010375
:1096F00002D0C35C594002E0C35A81EA1321082317
:109700000F0401D581F4C05149005B1E002BF7DC2A
:10971000521C102AE9DB2543C581C1F30330844282
:1097200001D10020F0BD3046F0BD0000D41400206F
:109730000404002030F8FFFF24FAFFFF300400206B
:10974000001BB70000100140DB950008CF95000812
:10975000BF950008B395000849940008F0B50023B0
:109760004FF0010C0A880CFA03F52A4228D04FEA80
:10977000D30200EB82064FEA437491F802E04FEA0D
:10978000D46734680EF00F025FEACE6E03D591F80D
:1097900003E04EEA02024FF00F0E0EFA07FE24EA33
:1097A0000E04BA40224332608A78282A02D0482A1E
:1097B00003D005E0C268AA4301E0C2682A43C26040
:1097C0005B1C102BCED3F0BD10B58A0721F003042B
:1097D0000649130F21440F228C689A4094438C60F1
:1097E0008A68984002438A6010BD00000000014072
:1097F0004FF4805108B14E4801E04D48001F016010
:1098000070472DE9F04104464A4817460D46008846
:10981000484E0C3E1CE015B115F8010B00E0FF208E
:1098200080460221304601F0A5FC0028F9D04146CF
:10983000304601F09BFC0121304601F09BFC0028E2
:10984000F9D0304601F094FCC0B20CB104F8010B21
:109850007F1EE0D20120BDE8F081F0B501218C032C
:1098600089B0204601F026F80121204601F034F8A5
:1098700018208DF816004FF42040ADF814002C4E3F
:1098800003208DF81700143E05A93046FFF766FF48
:10989000ADF8144004208DF8160005A93046FFF7F6
:1098A0005DFFA010ADF8140010258DF8165005A925
:1098B0003046FFF753FF1F4E0C3E304601F00CFCC4
:1098C0004FF48270ADF8020068010024ADF80A0080
:1098D0000720ADF81000ADF804400220ADF80E40AE
:1098E000ADF806000127ADF80040ADF80870ADF8FE
:1098F0000C506946304601F013FC0121304601F05E
:109900002BFC0DA0006806900120FFF771FF0422D8
:1099100006A907A8FFF775FF0020FFF769FF9DF86C
:109920001D00EF2802D0204609B0F0BD3846FBE705
:10993000140C01400C3800409F0000002DE9F0415C
:1099400080461D4616460C46084600F0F5F80746C8
:10995000404600F0E6F807EB8000C0B2102805D2C0
:109960007A4901EB0010856004710673BDE8F0814F
:1099700051B104290BD008290CD00C290DD101229A
:109980005FF0100101F027BA01220221FAE701225B
:109990000421F7E701220821F4E7704770B50D466E
:1099A0000446017B134600682A46FFF7C7FF217B68
:1099B0002068BDE87040DBE708B58DF800000020A6
:1099C0008DF8010001208DF802008DF80300684633
:1099D00000F08DFC08BDFEB5064614460D466846EF
:1099E00001F0C9F95A486D1E44435A48ADF8045075
:1099F00069460068B0FBF4F0401EADF8000000209E
:109A0000ADF80600ADF80200304600F07FFFFEBD65
:109A100010B504460068FFF7DEFF0121206801F061
:109A2000C5F9607BBDE81040C6E770B5054608463D
:109A300000F082F80446284600F073F804EB80003A
:109A40004249C0B201EB001070BD2DE9F041424E19
:109A500007460024305D30B1042817D0082828D0EC
:109A60000C2839D04FE00221384601F0E7F90128EF
:109A700049D10221384601F0EDF900213846FFF7BF
:109A8000D4FF0546384601F0D0F937E004213846C6
:109A900001F0D4F9012836D10421384601F0DAF971
:109AA00004213846FFF7C1FF0546384601F0BFF9EB
:109AB00024E00821384601F0C1F9012823D108210A
:109AC000384601F0C7F908213846FFF7AEFF0546D2
:109AD000384601F0AEF911E01021384601F0AEF938
:109AE000012810D11021384601F0B4F90C21384674
:109AF000FFF79BFF0546384601F09DF9AA6801462D
:109B00000AB1287B9047641CE4B2042CA2D32DE751
:109B100012489AE74FF0804097E7114895E71148BF
:109B200093E701460020104A01E0401CC0B252F801
:109B300020308B42F9D1704701460020064A01E0EF
:109B4000401CC0B2135C8B42FAD17047E414002071
:109B500040420F002C040020FCDD0008002C0140D6
:109B600000040040000800401004002090F8423239
:109B7000D0F83401001D05C80BB109B102E009B1EC
:109B800002617047426170470189406889B248228A
:109B900000F00BBAFEB5064614460D46684601F0C5
:109BA000FDF80120ADF804000021ADF80050ADF83B
:109BB0000610ADF80810ADF802406946304601F0D5
:109BC0003DF8FEBD002180F83912012280F83822CC
:109BD00090F83B22012A0BD180F83B1290F84212F8
:109BE00009B1002200E00222006B017B0068D1E78E
:109BF0007047C268016A521E914201D3002100E001
:109C0000491C016270470179C90713D0B0F84012AE
:109C100041F34022521C01F0010306D02BB1036A2C
:109C20004269C1F34701D154E3E7B0F84612491C39
:109C3000A0F84612704730B590F83B12002910D1B9
:109C400090F83A12012390F8392208E0B0F8404227
:109C500003FA01F52C43491CA0F84042C9B28A42DC
:109C6000F4D830BD10B5044690F8380200281ED153
:109C700094F83902401CC0B284F83902092805D092
:109C80000A2814D194F83B0220B109E02046BDE82F
:109C90001040D0E7B4F8400240F00100A4F84002C0
:109CA0002046FFF7B0FF2046BDE810408AE710BD10
:109CB000D0E90910814201D101207047002070478E
:109CC00010B5044690F83C02002290B194F83D0291
:109CD00048B3B4F83E0200F001014008A4F83E0287
:109CE0002046FFF743FF94F83D02401E84F83D02F2
:109CF00010BD2046FFF7DCFF0028F9D1A16AA36957
:109D0000481CA062595C2369984200D3A2624FF4B8
:109D1000007004F50F7440EA410060800A20607012
:109D20000120207010BD84F83C2210BD00EBC00162
:109D300001EB801010B5A34901EBC0042046FFF7EA
:109D4000BFFF2046BDE810408CE770B506469E4830
:109D50000D464FF480310068034600BFB3FBF2F4B8
:109D60008C4203D3012BF9D95B08F7E79749B0FB85
:109D7000F1F0C2B2A1B23046FFF74AFEAFF2530291
:109D800029463046BDE87040FFF708BE70B500EBCD
:109D9000C00101EB80108B4901EBC0042079C007A2
:109DA00026D094F838020025012610B3206B00213C
:109DB000006801F038F894F83C0220B1B4F844028D
:109DC000401CA4F8440294F8420208B1022200E0C8
:109DD0000022206B017B0068FFF7DCFE84F83B6209
:109DE00084F8395284F83A52A4F8405284F8385230
:109DF00070BD94F83B02012803D194F8390284F82D
:109E00003A022046FFF717FF94F83B0228B184F886
:109E10003B5294F8420238B904E084F83B6294F86B
:109E2000420208B1022200E00022206B017B0068A0
:109E3000BDE87040AEE670B50D4604460AB100229A
:109E400000E00222217B2068FFF7A4FEAFF2C302EC
:109E500029462046BDE87040FFF7A0BD0189406853
:109E600089B2102200F0A1B84FF4807200F13401E1
:109E7000C26041610021026100F59C730162C0E98A
:109E800006318162416270472DE9F0410446504835
:109E90002060032020711D4616460F462046FFF71E
:109EA000E3FF002084F83C02012184F8381284F892
:109EB000390284F84252A4F84402A4F84602D4F8C5
:109EC0003401FFF7CBFF206BFFF75EFE0121204638
:109ED000FFF74CFE3220FEF74BFC32463946D4F8F1
:109EE0003401FFF732FF2A463946206BBDE8F041C6
:109EF000A1E770B504463348364A002502631032A4
:109F00000B46C0F8342122462946FFF7BDFF3248F0
:109F100001210460017170BD034630482D49203194
:109F200001631031C0F834112B490A680121ABE7F5
:109F30000179C90703D0D0E90721914202D14FF03E
:109F40000000704702D9A1EB020003E0C06808449A
:109F5000A0EB0200C0B2704700B503460079C0070D
:109F600010D01846FFF7E4FF00280BD05969D869D4
:109F7000095CDA68521E904201D2401C00E00020C9
:109F8000D861084600BD027992070AD5436A826902
:109F9000D154416A0269491CB1FBF2F302FB13116F
:109FA0004162704770470171704708B5ADF8001005
:109FB0008DF8022002218DF803106946FFF7CEFBD1
:109FC00008BD0000E41500202C04002040420F00D2
:109FD00000DE00085CDD0008200400202C180020B2
:109FE0001FB5044602AB062202211820FEF763F8D3
:109FF0009DF808009DF80910800800EB0120ADF8DD
:10A0000000009DF80A009DF80B10800800EB01206D
:10A01000ADF802009DF80C009DF80D10800800EBD3
:10A020000120ADF804001A48214602786846FCF782
:10A030006BFD1FBD10B5044608220F211820FEF746
:10A0400034F80E2210211820FEF72FF811494FF492
:10A050008050002C088001D00D48047010BD38B528
:10A06000044600208DF8000001466B4601221820AE
:10A07000FEF721F818B19DF80000FB2801D0002060
:10A0800038BD0548206005486060012038BD0000EB
:10A09000280400208201002035A00008E19F00086C
:10A0A00002681268104770B50C46054603E02A683E
:10A0B00028461268904714F8011B0029F7D170BD9B
:10A0C0000168496808470168896808470268D268DA
:10A0D0001047016809690847026852691047000083
:10A0E0007648016841F0010101604168744A1140FD
:10A0F00041600168734A11400160016821F48021C8
:10A100000160416821F4FE0141604FF41F0181604C
:10A110006D49C00308607047684A10B550686B4BC2
:10A1200010F00C016A4803D0042903D0082903D099
:10A13000036016E0416813E05168536801F4701140
:10A140004FF0020413F4803F04EB914106D05368B2
:10A150009B03436800D55B084B43E9E75D4B5943DC
:10A16000016051685A4AC1F303110832515C026818
:10A17000CA40026010BD7EB4002400944FF4E01386
:10A1800001944E49CDE90134534A0D6845F48035B8
:10A190000D608D6945F010058D614FF4A0650E6866
:10A1A00006F400360196009E761C0096019E16B9B4
:10A1B000009EAE42F3D10E68B60301D5022414E02E
:10A1C0000E6846F001060E6000940C6804F002046C
:10A1D0000194009C641C0094019C14B9009CAC4246
:10A1E000F3D10C68A40734D5012402943B4C2568B4
:10A1F00045F010052560256825F0030525602568D4
:10A2000045F0020525604C684C604C684C604C6819
:10A2100044F480644C60146824F0704414602C4C46
:10A220002A4D65604D6825F47C154D60156845F034
:10A2300000451560284A121FD56825F40045D560F1
:10A24000926815044FF4801204D5254D65601446BC
:10A2500001E0FEE71C460194029C012C29D0022C4F
:10A2600011D150B10198904202D14FF4A01003E0F7
:10A27000984202D14FF4001001904868019A42F4CC
:10A28000803210434860086840F0807008600868B9
:10A290008001FCD5486820F003004860486840F021
:10A2A000020048604868C0F381000228FAD17EBCF1
:10A2B00032E7486840F46010E4E700000010024014
:10A2C0000000FFF8FFFFF6FE08ED00E000127A0044
:10A2D0002C04002000093D00041001400020024031
:10A2E000001BB70018490843184908607047F0B5CB
:10A2F0000F21C478027801234FF0E026DCB1134C23
:10A300002468457804F4E064C4F5E064240AC4F1E8
:10A310000407E1408478BD400C402C4321010C4CE3
:10A320001155007800F01F018B40400906EB8000BA
:10A33000C0F80031F0BD02F01F008340500906EB69
:10A340008000C0F88031F0BD0000FA050CED00E09F
:10A3500000E400E010B54268464B0C791A400B68E7
:10A3600042EA0422134343608368434A1340D1E91D
:10A37000024222434C7943EA44031A438260C26A90
:10A38000097C22F47002491EC9B242EA0151C1623D
:10A3900010BD0029816802D041F0010101E021F0E7
:10A3A0000101816070470029816802D041F4807109
:10A3B00001E021F4807181607047816841F00801FB
:10A3C00081607047014600208968090700D5012097
:10A3D0007047816841F004018160704701460020A8
:10A3E0008968490700D5012070470029816802D09B
:10A3F00041F4A00101E021F4A0018160704770B533
:10A40000072409290AD9C568A1F10A0606EB460600
:10A41000B440A543B3401D43C56007E0056901EBA7
:10A420004106B440A543B3401D4305611F23072ADD
:10A4300009D2446B521E02EB820293409C4391402E
:10A440000C43446370BD0D2A09D2046BD21F02EB8A
:10A45000820293409C4391400C43046370BDC46AE4
:10A460000D3A02EB820293409C4391400C43C4623C
:10A4700070BD0000FFFEF0FFFDF7F1FF01684FF631
:10A48000FE72114001600021016041608160C16085
:10A490005749574A0839904203D1486840F00F00A5
:10A4A00006E0534A1432904204D1486840F0F0006C
:10A4B000486070474E4A2832904203D1486840F4C1
:10A4C0007060F5E74A4A3C32904203D1486840F454
:10A4D0007040EDE7464A5032904203D1486840F45C
:10A4E0007020E5E7424A6432904203D1486840F464
:10A4F0007000DDE73E4A7832904203D1486840F070
:10A500007060D5E73B4A111F904203D1086840F0C4
:10A510000F0006E0374A1432904204D1086840F038
:10A52000F00008607047334A2832904203D108682F
:10A5300040F47060F5E72F4A3C32904203D108683E
:10A5400040F47040EDE72B4A50329042EAD108685F
:10A5500040F47020E5E730B5036847F6F0729343A6
:10A560000C6A8A682243D1E904452C4322438C6952
:10A570002243CC6922434C6A22438C6A22431A4309
:10A580000260CA6842600A6882604968C16030BD82
:10A590000021016041608160C160016141618161B0
:10A5A000C16101624162816270470029016802D085
:10A5B00041F0010102E04FF6FE7211400160704768
:10A5C000002A026801D00A4300E08A430260704713
:10A5D00041607047406880B27047C10003D50549AB
:10A5E000091F086070470249083948607047000039
:10A5F000080002400804024030B52349837902680C
:10A6000053B30B6893430B600A1D13680468A3439C
:10A61000136002790A4413680468234313601A4ADA
:10A62000083213680468A3431360131D1C6805688F
:10A63000AC431C604479102C05D021440A680068A2
:10A6400002430A6030BD1168046821431160196833
:10A6500000680143196030BD0079084401689143E6
:10A66000016030BD084A014600201268064B0A40CE
:10A6700014331B680B4202D0002A00D0012070471F
:10A680000149143108607047000401405A4910B56F
:10A6900088424FF0010101D14C0501E04FF48004E4
:10A6A000204600F019F92046BDE81040002100F0D6
:10A6B00013B970B50446808886B00D4620F03F0679
:10A6C000684600F09FF84D490298B0FBF1F189B25D
:10A6D0000E43A680228822F001022280484B2A687D
:10A6E0009A421CD85200B0FBF2F080B2042800D28B
:10A6F0000420491C2184A083208840F00100208090
:10A7000021884FF6F5300140A8886A891043084334
:10A710002080A88929890843208106B070BDEB8874
:10A72000A3F53F46FF3E05D102EB4202B0FBF2F03B
:10A7300080B208E002EBC20303EB0212B0FBF2F0BE
:10A7400080B240F48040020501D140F001004FF496
:10A75000967251434FF47A72B1FBF2F140F400402B
:10A76000C7E741F288310160002181804BF6FF721A
:10A77000C280018141814FF480418181704700296D
:10A78000018802D041F0010101E021F001010180C6
:10A7900070470029018802D041F4807101E021F462
:10A7A0008071018070470029018802D041F4007156
:10A7B00001E021F40071018070470029018802D076
:10A7C00041F4806101E021F4806101807047002A3A
:10A7D000828801D00A4300E08A4382807047018268
:10A7E0007047008AC0B2704712B141F0010101E028
:10A7F00001F0FE01018270470054004040420F000A
:10A80000A086010030B53C494A683C4B12F00C046C
:10A8100005D03B4A042C126803D0082C24D00360D6
:10A8200000E002604A680F2303EA1212354B9C5C79
:10A830000268E24042604C68072505EA14241C5D6A
:10A8400022FA04F484604C6805EAD4241B5DDA40E3
:10A85000C2604968032303EA91312A4B1B1F595CEC
:10A86000B2FBF1F1016130BD4B684C6803F4701329
:10A870004FF0020514F4803F05EB934305D04C687C
:10A88000A40300D552085A43CBE71F4A5343C6E7F7
:10A89000194A0029516901D0014300E08143516107
:10A8A0007047154A0029916901D0014300E08143B6
:10A8B00091617047104A0029D16901D0014300E03D
:10A8C0008143D16170470C4A0029D16801D001430E
:10A8D00000E08143D1607047074A0029116901D027
:10A8E000014300E08143116170470348416A41F030
:10A8F00080714162704700000010024000127A002F
:10A90000300400204804002000093D0030B50288D2
:10A91000FD4BFE4C98420DD0A0420BD0B0F1804FC1
:10A9200008D0FB4DA84205D0FA4DA84202D0FA4DFE
:10A93000A84203D122F070054A882A43F74DA84265
:10A9400006D0F74DA84203D022F44075CA882A43A6
:10A9500002808A8882850A88028598420AD0A042AD
:10A9600008D0F04A904205D0EF4A904202D0EF4A18
:10A97000904201D1097A01860121818230BD30B532
:10A98000028C22F001020284028C8388048B22F064
:10A99000020224F073050C882C430D8915434A8864
:10A9A0002A43D94DA8420BD0D84DA84208D0DD4D3E
:10A9B000A84205D0DC4DA84202D0DC4DA8420DD102
:10A9C00022F008054A8923F440732A4322F0040543
:10A9D0008A882A438D891D43CB892B438380048336
:10A9E000C9888186028430BD70B5028C22F01002C5
:10A9F0000284028C8488038B0D8823F4E6464FF68C
:10AA0000FF7303EA052535430E8922F0200203EA8D
:10AA1000061616434A8803EA02123243BA4EB0427F
:10AA200002D0BA4EB04215D122F080064A8924F4F1
:10AA3000406403EA0212324322F040068A8803EAA5
:10AA4000021232438E8903EA86062643CC8903EA42
:10AA50008404344384800583C9880187028470BDDF
:10AA600070B5028C22F480720284028C8488838BFD
:10AA70000D8823F073031D4322F400730E894FF6F3
:10AA8000FF7202EA06261E434B8802EA0323334381
:10AA90009D4EB04202D09D4EB04215D123F40066C7
:10AAA0004B8924F4405402EA0323334323F48066A1
:10AAB0008B8802EA032333438E8902EA0616264373
:10AAC000CC8902EA0414344384808583C988818751
:10AAD000038470BD70B5028C22F480520284048C11
:10AAE0008288838B0D8823F4E6464FF6FF7303EAD2
:10AAF0000525354324F400560C8903EA0434344315
:10AB00004E8803EA063626437F4CA04202D07F4C93
:10AB1000A04205D122F480448A8903EA82122243AA
:10AB200082808583C988A0F84010068470BD828B1E
:10AB300022F440628283828B4FF6FF7303EA012185
:10AB40000A4382837047828B22F00C028283828BBD
:10AB50000A4382837047028B22F440620283028B95
:10AB60004FF6FF7303EA01210A4302837047F0B5F1
:10AB7000048C24F010040484078B048C4FF6FF75BA
:10AB800027F4734705EA03333B4305EA02221A43DD
:10AB90005D4B05EA011698420ED05C4B98420BD0F3
:10ABA000B0F1804F08D05A4B984205D0594B98428B
:10ABB00002D0594B984205D124F02001314341F095
:10ABC000100104E024F0A0030B4343F010010283C2
:10ABD0000184F0BD028B22F00C020283028B0A4337
:10ABE0000283704770B5048C24F001040484058B43
:10ABF000048C4FF6FF7606EA0313134325F0F305A2
:10AC0000414A2B4390420ED0404A90420BD0B0F1C3
:10AC1000804F08D03E4A904205D03E4A904202D032
:10AC20003D4A904202D124F0020201E024F00A02DF
:10AC30000A4342F001010383018470BD2DE9F05FF6
:10AC40000D4604460888304FDFF8C0C0DFF8C080EA
:10AC50004988AA882B894FF0804960B3042832D0F4
:10AC60004FF6FF7E082836D0208C9B4620F480507B
:10AC70002084A38B268C704600EA022223F47343BF
:10AC80001A4300EA0B3010430EEA013EBC420BD0DF
:10AC9000644509D04C4507D0444505D01D4A94422F
:10ACA00002D01D4B9C425AD126F4005141EA0E01BC
:10ACB00041F4805158E02046FFF794FFE988204690
:10ACC000BDE8F05F86E72046FFF751FFE9882046A0
:10ACD000BDE8F05F3FE7208C20F480702084B4F85A
:10ACE0001CA0208C0EEA031313432AF0F30A0EEA89
:10ACF000012B43EA0A03BC4220D064451ED04C45D8
:10AD00001CD044451AD013E0002C0140003401400F
:10AD10000004004000080040000C0040001000400B
:10AD20000014004000400140004401400048014040
:10AD30004A4A944202D04A4A944204D120F4007014
:10AD400040EA0B0002E020F42060084340F48070E9
:10AD5000A3832084E9882046BDE8F05FF3E626F46B
:10AD600002420A4342F48051A08320462184E988AC
:10AD7000BDE8F05FDBE64FF6FF71818000210180C6
:10AD8000C180418001727047002101804180818033
:10AD9000C180018141818181C18170470021018091
:10ADA000418001228280C180018170470029018891
:10ADB00002D041F0010101E021F001010180704762
:10ADC000002930F8441F02D041F4004101E0C1F3F2
:10ADD0000E0101807047002A828901D00A4300E0F9
:10ADE0008A4382817047028B22F008020A43028361
:10ADF0007047028B4FF6FF7322F4006203EA0121D1
:10AE0000114301837047828B22F008020A43828338
:10AE10007047828B4FF6FF7322F4006203EA012130
:10AE200011438183704781847047808E7047008F03
:10AE30007047808F7047B0F840007047024600208E
:10AE4000138A92890B4202EA010202D0002A00D042
:10AE500001207047C943018270470000000800408C
:10AE6000000C004030B50446008A85B00D464CF613
:10AE7000FF710840E98801432182A1894EF6F31051
:10AE80000140A8882A8910436A890A431043A08197
:10AE9000A08A4FF6FF410840A9890143A182684674
:10AEA000FFF7B0FC3048844201D1039800E00298DB
:10AEB000A1890904002900EBC00101EB00102968F9
:10AEC00002DA4FEA410101E04FEA8101B0FBF1F003
:10AED0006422B0FBF2F14FEA01114FEA11136FF057
:10AEE00018056B4300EB8300A3891D044FF0320368
:10AEF00006D503EBC000B0FBF2F000F0070005E060
:10AF000003EB0010B0FBF2F000F00F0008432081CB
:10AF100005B030BD0029818902D041F4005101E023
:10AF200021F400518181704710B5C1F3421301F043
:10AF30001F040121A140012B07D0022B07D01430A0
:10AF4000002A026805D00A4304E00C30F8E710300C
:10AF5000F6E78A43026010BD002A828A01D00A43C4
:10AF600000E08A43828270470038014039483849FE
:10AF700041603949416070473648016941F08001BC
:10AF80000161704733490420CA68D20701D001200B
:10AF90007047CA68520701D502207047C968C906C0
:10AFA000FBD50320704700B50346FFF7EBFF02E037
:10AFB000FFF7E8FF5B1E012803D0002B00D105201E
:10AFC00000BD002BF4D1FAE770B505464FF43026EA
:10AFD0003046FFF7E8FF042811D11E4C206940F0ED
:10AFE000020020616561206940F040002061304628
:10AFF000FFF7D9FF216941F6FD721140216170BD53
:10B00000F8B5064600204FF4005C00900D466046FF
:10B01000FFF7C9FF042816D10E4C206940F001004B
:10B02000206135806046FFF7BEFF41F6FE770428B9
:10B0300006D1B61C280C009630806046FFF7B3FF9F
:10B04000216939402161F8BD0249C860704700009C
:10B050002301674500200240AB89EFCD1448154914
:10B06000026800608A4203D01348804713480047B3
:10B07000134E4FF0090030601248016821F07061F2
:10B08000016041020160104C182020600F491048F7
:10B0900008601048D0F800D040680047FEE7FEE79F
:10B0A000FEE7FEE7FEE7FEE7FEE7FEE7FEE7FEE778
:10B0B000F04F0020EFBEADDEE1A00008ED0000087B
:10B0C0001810024004000140140C0140000C014023
:10B0D0004434434400F0FF1F2A4910B588420AD186
:10B0E000841401212046FFF7EEFB2046BDE8104006
:10B0F0000021FFF7E8BB2449884202D10121041452
:10B1000004E0224988420AD10121C4132046FFF7F6
:10B11000E3FB2046BDE810400021FFF7DDBB10BD7A
:10B1200030B502884C8802F441530A88CD88224306
:10B130008C882C4322430C8922434C8922438C89DE
:10B140002243CC8922431A430280828B22F400627C
:10B150008283098A018230BD0029018802D041F032
:10B16000400101E021F0400101807047818170477A
:10B17000808970470246002012890A4200D00120CF
:10B18000704700000030014000380040003C0040A3
:10B1900000487047DCDF0008A0F16101192900D8E0
:10B1A000203870472DE9F05F994615460F468346D3
:10B1B0004FF0FF36DDF828A011E0A819441009FB74
:10B1C000047080460146584652469047002802D0F7
:10B1D00004DA254603E04046BDE8F09F2646A5EB8D
:10B1E00006000128E9DC0020F6E740EA01039B079E
:10B1F00003D009E008C9121F08C0042AFAD203E0EC
:10B2000011F8013B00F8013B521EF9D27047D2B24F
:10B2100001E000F8012B491EFBD270470022F6E73F
:10B2200010B513460A4604461946FFF7F0FF2046BC
:10B2300010BD421E12F8013F002BFBD111F8013B5B
:10B2400002F8013B002BF9D1704730B505462A467C
:10B250000B4612F8010B13F8014B08B1A042F8D0CD
:10B260001CB1002802D06D1CF1E7284630BD10B596
:10B27000044604E00B7800F8013B03B1491C521E60
:10B28000F8D2204610BDCAB2401E10F8011F8A42F3
:10B2900002D00029F9D100207047421C10F8011B90
:10B2A0000029FBD1801A704770B50F4D00B928688E
:10B2B000002412E00A4602E09E4203D0521C13789A
:10B2C000002BF9D1DAB2224305D02BB124B10021F1
:10B2D00000F8011B04E00446401C0678002EE9D16A
:10B2E0002860204670BD0000580400202DE9F04180
:10B2F0000546002090460E46044600E0641C444586
:10B300000BD2285D00F058F90746305D00F054F983
:10B31000381A02D1295D0029F0D1BDE8F08170B55D
:10B32000064600F059FC046805460A220021304612
:10B3300000F048F92C6070BDF0B480EA0102D40F2F
:10B340004200B2EB410F02D20246084611464A00C3
:10B3500042D0C30DDDB2C1F3C752AD1A202D35DA8C
:10B36000C1F3160141F4000204B15242C5F12006B6
:10B3700002FA06F12A411044B3EBD05F23D0C4B1E6
:10B38000012DA0EBC35009DCF0BC4FF0004202EAF3
:10B39000C35200F50000DBB200F055B9400000F1E7
:10B3A000807000EBC350A0F1807040EAD17049007A
:10B3B00009E0490841EAC071A0EBC35000F5000064
:10B3C000400800EBC350F0BC00F034B961420122E8
:10B3D00002EB4101001BF6E7F0BC704781F0004131
:10B3E000AAE780F00040A7E780EA010210B502F06A
:10B3F0000043400026D04A0023D04FEA106101EB01
:10B400001261C0F35600C2F3560240F4000042F449
:10B410000002A0FB0220A1F17F014FEA00401404CA
:10B4200001D000F1010050EA124001D44000491E51
:10B43000C2B20C0604EBD010401C4008802A02D097
:10B4400003E0002010BD20F00100002900DA0020F8
:10B45000184310BD30B480EA010202F0004530F01C
:10B46000004221F0004015D0A0B1C0F3C753C2F391
:10B47000C754C2F31601C0F31600E41A41F40001E8
:10B4800040F400027D34914201D3641C00E0490085
:10B49000002C02DA30BC002070474FF4000000237B
:10B4A000914201D3891A034340084FEA4101F7D181
:10B4B00051B1914202D14FF0004105E002D24FF06C
:10B4C000010101E06FF0010103EBC450284430BCDE
:10B4D00000F0B0B8420005D0C0F3C75252429142CA
:10B4E00001DC0020704700EBC1507047C10F80EABB
:10B4F000E0700844CA079623002100F0A4B8962300
:10B500000022114600F09FB800F0004220F00040F9
:10B51000C10DC0F3160040F400007F2901DA0020BD
:10B520007047962903DCC1F19601C84001E09639C5
:10B530008840002AF4D04042704720F00040C10DFE
:10B54000C0F3160040F400007F2901DA00207047A4
:10B55000962903DCC1F19601C840704796398840AE
:10B5600070470000002801DBC0F10040002901DB2A
:10B57000C1F1004181427047002801DBC0F1004069
:10B58000002901DBC1F100418842704730B50B460C
:10B59000014600202022012409E021FA02F59D4203
:10B5A00005D303FA02F5491B04FA02F52844151ED7
:10B5B000A2F10102F1DC30BDA0F14101192900D84E
:10B5C000203070472DE9F04791460F4680460446EB
:10B5D000002614F8015B2DB1FFF7DAFD0068405D2D
:10B5E000C007F6D12B2D02D02D2D18D0641E4A464F
:10B5F0003946204600F0E1F927B13968A14201D16E
:10B60000C7F8008071054FF002040BD540420028B6
:10B6100003DD00F0E1FA0460A007BDE8F08746F41E
:10B620008066E4E70028F8DA00F0D6FA04606FF0EC
:10B630000040F2E70029A8BF7047401C490008BF3E
:10B6400020F00100704710B4B0FA80FC00FA0CF052
:10B6500050EA010404BF10BC704749B1CCF120048A
:10B6600021FA04F411FA0CF118BF01212143084317
:10B67000A3EB0C01CB1D0106000A002BBEBF00206E
:10B6800010BC704700EBC35010440029A4BF10BC8D
:10B690007047401C490008BF20F0010010BC7047F3
:10B6A000F0B4002802DCF0BC00207047C0F3C751A2
:10B6B000C0F3160040F40000CA0701D14000491E43
:10B6C0003F2202EB6105002211464FF4000626FAE4
:10B6D00001F31344D418844201D8001B1A464000D9
:10B6E000491C1729F3DD5100814202D24FF0FF318E
:10B6F00000E0002102EBC550F0BCFFF79BBF10B586
:10B7000041000CD0C0F3C751962908DC7E2909DC22
:10B7100006DB410204D000F0004040F07E5010BD36
:10B72000002010BDC1F19604C4F1200100FA01F11E
:10B73000E040FFF77FFFA04010BD2DE9FE4F80469F
:10B7400081EA0300C00F0C46009021F0004123F075
:10B750000045B8EB0200A94105D24046214690467B
:10B760001C460B46024623F00040104304D14046DD
:10B77000214603B0BDE8F08F270DC7F30A00C3F3DD
:10B780000A510290401A0190402866DAC3F3130070
:10B7900040F4801B0098924620B10023D2EB030AAC
:10B7A00063EB0B0B01985946C0F14002504600F084
:10B7B000D3F806460D4650465946019A00F0EBF87C
:10B7C00010EB08006141002487EA115284EAE77314
:10B7D0001A433BD0009A3AB3019A012A4FEA075222
:10B7E00010DC001B61EB02014FF0004202EA07523D
:10B7F000CDE90042001C41F5801132462B4600F095
:10B8000038F9B6E7001B61EB0201001C41F580131B
:10B8100000185B412018A2F5001747EB030140EA2E
:10B82000D570B6196D4111E06D084FEA360645EA4C
:10B83000C0754FEA0752001B61EB0201001C41F585
:10B84000801149084FEA30000019514132462B4619
:10B8500003B0BDE8F04F00F0FFB8009801224000AF
:10B860000023D0EB020263EBE073009821464FEA1D
:10B87000E074B8EB000061EB0401E9E783F00043FA
:10B880005BE781F0004158E710B500F0004420F07C
:10B890000040C20DC0F3160040F400007F2A07DA12
:10B8A0007D2A00DA7D22763A00FA02F1002008E0D3
:10B8B000962A09DCA2F1760100FA01F1C2F19602A2
:10B8C000D040FFF7B7FE01E0963A9040002C00D040
:10B8D000404210BD00F0004230F000400AD0C10DDF
:10B8E00001F56071C0F3160042EA0151C208400739
:10B8F0001143704700200146704701F0004330B407
:10B9000021F0004150EA010206D00A0DA2F5607252
:10B91000C1F31301002A02DC30BC00207047440F41
:10B9200044EAC104C100E01830BC00EBC250FFF78C
:10B9300081BE0000064C074D06E0E06840F00103C0
:10B9400094E8070098471034AC42F6D3F4F7D2FBE2
:10B9500034EA000854EA0008202A04DB203A00FAFE
:10B9600002F1002070479140C2F1200320FA03F356
:10B97000194390407047202A04DB203A21FA02F054
:10B980000021704721FA02F3D040C2F12002914019
:10B99000084319467047202A06DBCB17203A41FAA4
:10B9A00002F043EAE07306E041FA02F3D040C2F14C
:10B9B000200291400843194670472DE9F05F824606
:10B9C0000078002715468B460AF10104B946302855
:10B9D00001D09DB113E014F8010B0127782803D0A2
:10B9E000582801D045B10AE00DB1102D07D100272C
:10B9F000102514F8010B02E0082500E00A250026B6
:10BA0000B0460EE005FB080005FB06F1012701EB3F
:10BA100010461FFA80F8B6F5803F00D3B94614F8F7
:10BA2000010B294600F077F80028EBDABBF1000F94
:10BA300005D00FB1641E00E05446CBF80040B9F1C8
:10BA4000000F06D000F0C8F802210160C81EBDE852
:10BA5000F09F48EA0640FAE710B5002B08DA401CD0
:10BA600041F1000192185B411A4301D120F001001D
:10BA700010BD2DE9F04D92469B4611B1B1FA81F20D
:10BA800002E0B0FA80F220329046FFF765FF0446EC
:10BA90000F4640EA0A0041EA0B0153465A46084362
:10BAA00003D120463946BDE8F08D114653EA010026
:10BAB00015D0C8F140025046FFF75DFF05460E461F
:10BAC000504659464246FFF747FF084301D0012040
:10BAD00000E00020054346EAE0762C4337430A980D
:10BAE0004FEA4453A0EB08004FEAD4240A304FF049
:10BAF000000244EA47544FEAD72502D50020014608
:10BB0000D1E7010510196941DDE9084500196941CE
:10BB1000BDE8F04DA0E73A2800D2303820F02002EE
:10BB2000412A01D3A2F13700884201D34FF0FF3000
:10BB3000704770B501EB020410F8015B15F00703C4
:10BB400001D110F8013B2A1106D110F8012B03E0B6
:10BB500010F8016B01F8016B5B1EF9D12B0705D4BE
:10BB60000023521E0FD401F8013BFAE710F8013B05
:10BB700002F10202A1EB030303E013F8015B01F8F9
:10BB8000015B521EF9D5A142D6D3002070BD000042
:10BB90000FB4054B10B503A9044A029800F0E8F869
:10BBA00010BC5DF814FB00007D2500085C0400203B
:10BBB0004100080218BF04200A0E18BF40F001001F
:10BBC0004FF07F4232EA010108BF40F00200012835
:10BBD00008BF05207047000000487047600400203F
:10BBE0006FF05E010807FFF775BC00002DE9F04D0E
:10BBF0000E4614464FF07F41B1EB440F9EBF4FF00D
:10BC0000FF313160BDE8F08D4FF0004040EA042183
:10BC1000C4F3C7507838431100F01F00DFF814C197
:10BC2000C0F12002FC445CF823500CEB83038540F8
:10BC3000D3F804C02CFA02F72F439D680CFA00FCDD
:10BC400025FA02F8DB6805FA00F023FA02F240EA6E
:10BC500002054CEA080CA7FB0132ACFB01C0A5FBB6
:10BC6000015101EB0C058D4234BF4FF0010C4FF038
:10BC7000000CC1186144BCF1000F02D0814202D90E
:10BC800003E0814201D2012000E00020104400F1D5
:10BC900020024FEA92188006CA0C40EA42304F0355
:10BCA000C6F80080FFF722FC82463846FFF727FCE3
:10BCB0006FF01201FFF70EFC07462846FFF71FFC46
:10BCC0006FF02501FFF706FC834639465046FFF723
:10BCD00033FB5946FFF730FB00F500656FF30B05AA
:10BCE00051462846FFF77AFB3946FFF777FB59465E
:10BCF000FFF777FB1049FFF777FB07460F49284608
:10BD0000FFF772FB3946FFF717FB07460C49284639
:10BD1000FFF76AFB3946FFF70FFB14F0004F08BF2F
:10BD2000BDE8F08DC8F1805180F000403160BDE881
:10BD3000F08D0000B8230000DB0FC92F22AAFD29D7
:10BD40000000C92F02E008C8121F08C1002AFAD15A
:10BD500070477047002001E001C1121F002AFBD18B
:10BD6000704700000149086070470000600400202F
:10BD70002DE9FF4F8BB09A460F4605460026C9E0D5
:10BD8000252837D100246D1C6649A04601222B7856
:10BD9000203B02FA03F0084202D004436D1CF6E790
:10BDA00028782E2817D115F8010F44F004042A280A
:10BDB0000ED06FF02F022878A0F1300109290AD89F
:10BDC00008EB880102EB410100EB01086D1CF2E772
:10BDD00057F8048B6D1C287869283FD006DC0028B2
:10BDE00071D063280CD0642804D137E0732811D0B7
:10BDF00075284ED052460D99904706F1010688E00D
:10BE000017F8040B8DF8000000208DF80100E946BA
:10BE1000012003E057F8049B4FF0FF3061074FF01B
:10BE2000000401D40AE0641C44450DDA8442FADBC4
:10BE300019F804100029F6D106E0641C8442FCDBEA
:10BE400019F804100029F8D1264404E019F8010B70
:10BE500052460D999047641EF8D25AE001CF4FF038
:10BE60000A0B002804DAC0F100004FF02D0102E0B7
:10BE7000210504D52B218DF82410012103E0E107D1
:10BE800005D02021F7E70DF1200908910CE00021F1
:10BE9000F9E701CF4FF00A0BF9E75946FFF776FBB8
:10BEA00001F1300209F8012D0028F6D1ADEB0900AF
:10BEB00000F1200B600701D44FF00108D84503DDE5
:10BEC000A8EB0B0001E029E000208046002406E0FA
:10BED00009A85246005D0D999047761C641C08988D
:10BEE0008442F5DB04E0302052460D999047761CE1
:10BEF000B8F10001A8F10108F5DC05E019F8010B23
:10BF000052460D999047761CBBF10001ABF1010B35
:10BF1000F4DC6D1C287800287FF432AF0FB0304677
:10BF2000BDE8F08F092801002DE9F04104464FF0EB
:10BF30001A4000EB4400B0F1C85F20461AD94FF018
:10BF4000CC41B1EB440F84BF3548BDE8F0814FF0E0
:10BF50007F41B1EB440F04D2BDE8F0410121FFF76E
:10BF6000B9BA0120FFF7FEFEBDE8F0410021084606
:10BF7000FFF770BA4FF0FC41B1EB440F1CD224F034
:10BF800000404FF07E51FFF72CFA4FF0FF31FFF7E2
:10BF9000A1FA074600F02EFE14F0004F1DBF214EFF
:10BFA000214D80F00040002608BF35464FF040414B
:10BFB000FFF71AFA044605E01C4E1D4D0146FFF737
:10BFC00013FA07461B493846FFF70EFA1A49FFF7DE
:10BFD000B3F93946FFF708FA1849FFF7ADF93946C2
:10BFE000FFF702FA1649FFF7A7F93946FFF7FCF900
:10BFF0001449FFF7A1F9804639462046FFF7F4F9C6
:10C000004146FFF7F1F9074629462046FFF7E9F9CF
:10C010003946FFF7E3F93146BDE8F041FFF78CB947
:10C02000DB0FC93F0000494022AA7D3A0000C93F0A
:10C0300022AAFD3924FE1C3DC78AD83C1E67383D24
:10C040001B93993DAFAA2A3E2DE9F0474FF0684275
:10C0500002EB40030C460546B3F1654F3CBF02EBD3
:10C060004102B2F1654F3FD34FF07F42B2EB400F38
:10C0700028BFB2EB410F03D2BDE8F047FFF75CB930
:10C0800040EA01035B0008BF44F0FF410AD0B2EB75
:10C09000400F08BFB2EB410F06D125F0804024F0DD
:10C0A000804105460C461FE0B2EB400F12BF5FEA2D
:10C0B000410245F0FF4004F0004115D04FEA410233
:10C0C00092EA400310D4002AB4BF4FF03E564FF01E
:10C0D0009F463146FFF788F9054631462046FFF76F
:10C0E00083F9044628462146C0F3C753C1F3C7521B
:10C0F0009A1A1B2A06DD10F0004F14BF5448554809
:10C10000BDE8F08712F11A0F17DA11F0004F06D0D0
:10C1100010F0004F0CBF50485048BDE8F087214652
:10C120002846FFF797F90446FFF742FD042808BFA9
:10C13000FFF756FD2046BDE8F0874200B2EB410F05
:10C1400025D910F0004F19BF454F464E464F474E78
:10C15000224685F0004415460A4680F0004110460C
:10C160000A1A5200B2F1807F3ED248404049DFF8BF
:10C1700004A110F0004F18D04FF03F483846FFF7A9
:10C180002DF9074651463046FFF728F917E011F020
:10C19000004F04BF00263746E2D010F0004F19BF11
:10C1A000354F364E364F374EDAE74FF07C5838462B
:10C1B000FFF7C2F8074651463046FFF7BDF806467E
:10C1C00041462846FFF710F92146FFF7B5F88246A9
:10C1D00021464046FFF708F92946FFF702F9514684
:10C1E000FFF738F9044604E021462846FFF732F904
:10C1F00004460146FFF7F8F880462349FFF7F4F8B4
:10C200002249FFF799F84146FFF7EEF82049FFF77A
:10C2100093F84146FFF7E8F81E49FFF78DF84146CD
:10C22000FFF7E2F81C49FFF787F80546414620462C
:10C23000FFF7DAF82946FFF7D7F83146FFF77CF821
:10C240002146FFF779F83946BDE8F047FFF774B8A3
:10C25000DB0FC9BFDB0FC93FDB0F4940DB0F49C014
:10C260000000C9BF22AAFDB90000C93F22AAFD39BA
:10C270000060ED3EC30ACE37000049C022AA7DBA55
:10C280000000494022AA7D3A2DAD65BD8FB8D53D4D
:10C290000FB511BE61C84C3EA8AAAABE2DE9F8434D
:10C2A0000446024650486946B0EB420F09D94FF0A8
:10C2B000E640B0EB420F94BF00204FF0FF300090FB
:10C2C00034E04A4B22F0004083422BD948492046B3
:10C2D000FFF78AF8FFF713FA8046FFF715F900F029
:10C2E0000300009043494046FFF77EF80546424967
:10C2F0004046FFF779F8064640494046FFF774F894
:10C3000007463F494046FFF76FF82146FFF769F8B7
:10C310003946FFF763F83146FFF760F82946FFF723
:10C320005DF802E01046FFF761FC04462546009CDC
:10C33000002C18DA6800B0F17F4F3CBF4FF07E5000
:10C34000BDE8F88309D14FF00100FFF70BFDBDE810
:10C35000F84300210846FFF77DB82846BDE8F843BA
:10C360000121FFF7B7B8294614F0010F08461CD089
:10C37000FFF73AF806462349FFF736F82249FFF758
:10C3800030F83146FFF730F82049FEF7D5FF314647
:10C39000FFF72AF82946FFF727F82946FEF7CCFFD2
:10C3A00014F0020F1CD0BDE8F883FFF71DF8054616
:10C3B0001749FFF719F81749FEF7BEFF2946FFF79F
:10C3C00013F81549FEF7B8FF2946FFF70DF84FF0AF
:10C3D0007E51FEF7B1FF14F0020F08BFBDE8F883ED
:10C3E00080F00040BDE8F883B61F927E490E4946B2
:10C3F00083F9223F1A61342C0020A23300A0FD39BA
:10C400000000C93F336D4C39DA82083CA0AA2ABE2D
:10C41000B93AB2BACA9F2A3DDDFFFFBE70B50546E4
:10C42000FFF732FA04464000801C0DD12846FFF782
:10C4300066F905462046FFF759F82946FFF792F8B6
:10C440001CBF0120FFF78EFC204670BD2DE9F04D8A
:10C450000F460E46A0F50001804604464FF00070DE
:10C4600084B04FF07E554FF0000B00EB47004FF0CB
:10C470007F4AB1F1FE4F04D2B0F1804F80F00181CC
:10C4800041E0B0F1804F3ED304F1FF40B0F1FE4FE8
:10C490001FD200BF28F00048C6F3C75044467F288B
:10C4A00009DB97287DDAC0F19600012101FA00F03E
:10C4B000411E314209D00120FFF754FC04B0002195
:10C4C000BDE8F04D0846FEF7C5BF304218BFFE4D2F
:10C4D000D7E0600000281CBF4FF08070B0EB440F25
:10C4E0000BD91B214046FEF7F5FF804604466FF04E
:10C4F0001A0B10F0004FCDD1C3E0A4F50000B0F14D
:10C50000FE4F1BD2BDE0B0F1007F11D300213846B1
:10C51000FFF728F806D16000002818BFBAEB440FD7
:10C5200071D8B1E706F0004040F0FC563746ABE763
:10C53000B0F1807F38BFA6F50007A5D324F00040F6
:10C540006FF0FF42E14B8118994210D326F0004171
:10C550000A449A420BD3B4F17E5F18BF5FEA4602E9
:10C5600051D0B0F1FF4F98BFB1F1FF4F06D904B0E1
:10C5700039464046BDE8F04DFEF7DEBEB4F1FF4F50
:10C5800010D0C6F3C7507F2809DB972812DAC0F114
:10C590009600012101FA00F0411E314206D0002030
:10C5A00009E06EE016F0004F5DD127E0304218BF81
:10C5B000012000D1022014F5000F13D024B3B4F1F0
:10C5C000004F27D014F1814F56D04FF0FE40B0EB12
:10C5D000440F94BF01200020012101EBE671884245
:10C5E00041D10BE016F0004F02D001283FD03AE0D5
:10C5F000012802BFB64804B0BDE8F08D4FF0FF40FF
:10C6000004B0BDE8F08D37E016F000400ED104B064
:10C61000BDE8F08DB6F1FF4F25D016F5000F05D01F
:10C6200016F0004F18D008B101280AD00220FFF7F9
:10C6300099FB04B00021BDE8F04D4FF07E50FEF7AD
:10C6400009BF0220FFF78EFB04B04146BDE8F04D64
:10C650004FF07E50FEF7FEBE002804BF04B0BDE8D8
:10C66000F08D012803D004B00020BDE8F08D04B0A7
:10C670004FF00040BDE8F08D04B04FF07E50BDE8B3
:10C68000F08D94482044B0F5005F44D84046FFF751
:10C6900021F90022904BFFF7F1F8FFF72EF904463D
:10C6A0006FF00101FEF716FF8C49FEF79AFE214656
:10C6B000FEF79AFE4FF07C51FEF793FE06462146A8
:10C6C0000846FEF791FE80F000403146FEF78CFEF2
:10C6D000804683492046FEF787FE0646814940464C
:10C6E000FEF782FE804680492046FEF77DFE4146E9
:10C6F000FEF722FE044601463046FEF71DFE00F519
:10C70000006B6FF30B0B59463046FEF767FE214670
:10C71000FEF712FED4E004F58020C00C00F00F06F6
:10C72000C0F307107F38A4EBC05483443046FEF7B3
:10C73000DDFE6FF00301FEF7CDFE4FF07E51FEF7F8
:10C74000FBFD014602902046FEF748FE0190204680
:10C750000299FEF7F1FD00F500686FF30B080090F9
:10C7600041460298FEF73AFE2146FEF7E5FD0290AB
:10C770004FF07E500099FEF76DFE01460090019843
:10C78000FEF732FE00F500646FF30B0420460299B9
:10C79000FEF72AFE029041462046FEF725FE01994B
:10C7A000FEF71FFE0299FEF719FE0099FEF71CFE28
:10C7B000014600902046FEF7BFFD0146FEF714FE3D
:10C7C00080464A49FEF710FE4449FEF7B5FD414652
:10C7D000FEF70AFE804600212046FEF77BFE019010
:10C7E00020460099FEF7A8FD4146FEF7FDFD0446F0
:10C7F00000210098FEF76EFE2146FEF79DFD804663
:10C8000001460198FEF798FD00F500646FF30B04F4
:10C8100021460198FEF7E2FD4146FEF78DFD804678
:10C8200033492046FEF7E0FD009032494046FEF7CE
:10C83000DBFD804630492046FEF7D6FD4146FEF737
:10C840007BFD804601460098FEF776FD00F500640A
:10C850006FF30B0421460098FEF7C0FD4146FEF73A
:10C860006BFD80462548784450F8361000EBC60032
:10C87000019146684FEA0B10FEF738FE00903146F2
:10C880004046FEF759FD2146FEF756FD0199FEF799
:10C8900053FD0099FEF750FD00F5006B6FF30B0B95
:10C8A00058460099FEF79AFD0199FEF797FD21463B
:10C8B000FEF794FD3146FEF791FD4146FEF791FDEE
:10C8C000804607F500641BE0000080BFFFFF3F00CB
:10C8D000000080FF001080C00000F03FABAAAA3E1D
:10C8E00000B0B8413BAAB841D49A38BB7EE24C3E76
:10C8F00000B038423BAA3842D49AB8BBAE1500000B
:10C900006FF30B0421463846FEF768FD07462146C3
:10C910005846FEF769FD064639462046FEF70CFDEF
:10C920004146FEF761FD044639465846FEF75CFD78
:10C930002146FEF701FD074601463046FEF7FCFCA6
:10C9400000F500646FF30B0421463046FEF746FD08
:10C950003946FEF7F1FC804601462046FEF7ECFC26
:10C96000FEF792FF07460611FEF7C0FD2146FEF7CF
:10C9700038FD4146FEF7E0FC04463549FEF734FD3C
:10C980003449FEF7D9FC2146FEF72EFD3249FEF769
:10C99000D3FC2146FEF728FD0146304807F00F047E
:10C9A000784450F82400FEF71FFD2D49794451F8D2
:10C9B0002410FEF7C1FC2B49794451F82410FEF7EE
:10C9C000BBFC06F17D01FC2908D23146FEF782FD51
:10C9D00004B02946BDE8F04DFEF706BD06F1BF01E3
:10C9E000B1F5BF7F16D83146FEF774FD2946FEF734
:10C9F000FBFC0446BAEB440F1AD060000CD0204672
:10CA0000FFF7D6F8042808BFFFF7EAF8204604B07D
:10CA1000BDE8F08D002E0BDA0220FFF7A3F9FFF737
:10CA2000DFF80146284604B061F31E00BDE8F08D32
:10CA30000220FFF797F961214FF0E040FEF74AFD31
:10CA40000146284604B061F31E00BDE8F08D0000E9
:10CA5000FC596337C9FF753A1872313D74150000EF
:10CA600028150000DC1400002DE9F84304460246B6
:10CA700053486946B0EB420F09D94FF0E640B0EB9E
:10CA8000420F94BF00204FF0FF30009034E04D4B38
:10CA900022F0004083422BD94B492046FEF7A4FCEC
:10CAA000FEF72DFE8046FEF72FFD00F003000090FC
:10CAB00046494046FEF798FC054645494046FEF784
:10CAC00093FC064643494046FEF78EFC0746424922
:10CAD0004046FEF789FC2146FEF783FC3946FEF707
:10CAE0007DFC3146FEF77AFC2946FEF777FC02E032
:10CAF0001046FFF77BF804462546009C002C1DDA03
:10CB00006800B0F17F4F09D22846FFF751F804289A
:10CB100008BFFFF765F82846BDE8F88308D1012073
:10CB2000FFF720F9BDE8F84300210846FEF792BC64
:10CB30002846BDE8F8430121FEF7CCBC294614F095
:10CB4000010F08461ED0FEF74FFC05462349FEF7AD
:10CB50004BFC2349FEF7F0FB2946FEF745FC214933
:10CB6000FEF7EAFB2946FEF73FFC4FF07E51FEF749
:10CB7000E3FB14F0020F08BFBDE8F88380F000402B
:10CB8000BDE8F883FEF730FC06461749FEF72CFC9B
:10CB90001649FEF726FC3146FEF726FC1449FEF73F
:10CBA000CBFB3146FEF720FC2946FEF71DFC29464B
:10CBB000FEF7C2FB14F0020FE0D1BDE8F8830000DD
:10CBC000B61F927E490E494683F9223F1A61342CE2
:10CBD0000020A23300A0FD390000C93FB93AB2BA23
:10CBE000CA9F2A3DDDFFFFBE336D4C39DA82083C17
:10CBF000A0AA2ABE70B50546FEF752FD044620F0F5
:10CC00000040C0F1FF40C00F08D025F00040C0F147
:10CC1000FF40C00F04BF0120FFF7A4F8204670BDFD
:10CC20008AE00008E7E0000845E1000887E0000826
:10CC30008EE0000835E0000830E0000875E00008EC
:10CC400025E000083FE1000838E00008F8E00008AF
:10CC500054E100084FE00008B8E0000860E0000878
:10CC60001EE0000881E00008DAE0000820E100088A
:10CC700013E10008B1E0000800000000C6E0000871
:10CC80002FE1000895E000084BE10008EDE0000806
:10CC900034E10008A6E000086CE000082BE1000881
:10CCA00046E0000802E100085EE1000808E1000833
:10CCB000CAE0000843E0000800000000D5E00008DA
:10CCC0003FE00008D0E000085CE0000802E1000856
:10CCD0002BE1000858E0000800000000A9E8000867
:10CCE00028E000080FE0000869E8000817E00008E5
:10CCF000FBE200080000000084E8000817E80008D4
:10CD0000330300087FE80008D7E600088D03000819
:10CD100046E70008B6E70008AD06000883E600080D
:10CD20009EE500085F07000874E70008A9E800080E
:10CD3000D508000824E30008F7E40008F708000815
:10CD400074E40008C3E40008C10900087EE6000896
:10CD5000A9E80008D90900087AE600089BE600085F
:10CD6000050A0008E5E60008E2E70008D10C000823
:10CD700033E70008A3E30008570D0008ACE2000801
:10CD800000E00008E70D0008D8E30008A6E7000867
:10CD9000AF08000870E70008F5E70008210E00085A
:10CDA00069E700085DE70008690F0008DBE5000897
:10CDB000A9E8000813100008F2E2000802000000D1
:10CDC000A004002000000000282300003FE200082B
:10CDD00000000000A204002000000000010000008C
:10CDE00072E1000802000000A6050020B004000067
:10CDF000A4060000DAE2000802000000640500203A
:10CE000000000000D0070000E6E200080200000079
:10CE10006605002000000000D007000034E2000892
:10CE2000020000006805002000000000D00700009C
:10CE3000A2E4000802000000A80500200000000095
:10CE4000D0070000ABE4000802000000AA050020A3
:10CE500000000000D00700005AE8000802000000AF
:10CE60006A05002000000000D007000064E400080C
:10CE7000020000006C05002000000000D007000048
:10CE800078E10008020000006E05002000000000AC
:10CE9000D0070000B4E20008020000007005002086
:10CEA00000000000D00700005CE300080200000062
:10CEB0007205002032000000007D00004DE30008F4
:10CEC000020000007405002032000000F2010000A2
:10CED00091E5000800000000AC0500200000000003
:10CEE00001000000A1E1000800000000AD050020E5
:10CEF0000000000064000000EBE6000801000000F4
:10CF0000AE050020FFFFFFFF01000000C6E600089D
:10CF10000000000029080020300000007E00000012
:10CF200086E3000804000000B4050020B0040000FF
:10CF300000C2010082E3000804000000B8050020E0
:10CF4000B0040000004B0000ADE10008000000004C
:10CF5000BC0500200000000001000000C3E1000843
:10CF600000000000BD0500200000000001000000DE
:10CF700000E3000800000000B005002000000000F1
:10CF80000400000096E3000801000000B105002045
:10CF9000000000000400000009E300080000000099
:10CFA000A4050020000000000300000088E600083F
:10CFB00000000000BE05002000000000010000008D
:10CFC000D3E7000800000000BF05002000000000BB
:10CFD0000200000053E4000800000000C00500202B
:10CFE000000000000100000088E2000800000000CE
:10CFF000980500200A000000C800000060E2000858
:10D0000000000000990500200A0000003200000026
:10D010004DE20008000000009A0500200A00000010
:10D02000320000000BE50008000000009B05002016
:10D0300000000000090000003EE6000800000000BB
:10D0400076050020000000000800000068E10008EC
:10D05000000000007705002000000000080000002C
:10D0600003E4000800000000780500200000000034
:10D070000800000064E50008030000007A050020B5
:10D080004CFFFFFF6801000022E4000803000000DD
:10D090007C0500204CFFFFFF680100003EE800080F
:10D0A000030000007E0500204CFFFFFF6801000028
:10D0B00009E600080100000080050020FFFFFFFFD7
:10D0C0000100000017E300080000000081050020B7
:10D0D0000000000005000000F3E500080200000069
:10D0E0008A0500206400000084030000E1E10008DC
:10D0F0000000000088050020000000008000000003
:10D10000FAE3000802000000820500200000000091
:10D110000001000010E70008020000008405002064
:10D1200064000000E803000021E70008020000009E
:10D130008605002064000000E8030000B7E6000850
:10D14000000000002C08002000000000010000008A
:10D150002BE20008000000009808002000000000FA
:10D160002000000028E200080000000099080020CC
:10D170000000000064000000DDE400080000000082
:10D180009A08002001000000FA00000073E2000885
:10D19000000000009B0800200000000001000000CB
:10D1A000BEE30008000000009E0800200000000010
:10D1B0009600000092E20008020000009C08002097
:10D1C000010000008403000035E3000800000000B7
:10D1D0004B08002000000000FA0000002DE60008C7
:10D1E000000000004C080020000000006400000067
:10D1F000D9E10008000000004D08002000000000F8
:10D200006400000035E60008000000004E08002021
:10D2100000000000640000003DE300080000000082
:10D220004F08002000000000640000006BE30008CD
:10D230000000000050080020000000006400000012
:10D240002CE300080000000051080020000000004E
:10D250006400000097E70008020000005208002068
:10D26000E8030000D007000088E800080000000084
:10D27000E008002000000000C800000097E8000857
:10D2800000000000E108002000000000C8000000CD
:10D29000C8E2000802000000E2080020E8030000E5
:10D2A000D0070000F1E1000802000000E4080020BF
:10D2B00064000000D00700001DE500080100000028
:10D2C000AF05002000000000040000001FE6000879
:10D2D00001000000E6080020FFFFFFFF0100000042
:10D2E00049E6000801000000E708002000000000F7
:10D2F0000100000039E7000800000000E8080020F5
:10D3000000000000FF00000001E70008000000002E
:10D310005A08002000000000FA0000000BE200089C
:10D32000000000005C080020000000006400000015
:10D330001AE20008000000005B0800200000000066
:10D3400064000000B4E40008000000006C08002045
:10D3500000000000010000003CE4000803000000A1
:10D3600058080020D4FEFFFF2C0100007CE50008D7
:10D370000300000056080020D4FEFFFF2C0100002F
:10D38000DDE30008000000005D0800200000000050
:10D3900030000000EBE300080500000060080020FA
:10D3A000000000000100000034E500080500000056
:10D3B0006408002000000000010000007FE7000872
:10D3C00005000000680800200000000001000000C7
:10D3D000E3E500080300000054080020B0B9FFFF97
:10D3E0005046000066E600080000000031080020FA
:10D3F00000000000C80000008EE4000800000000EB
:10D400003B08002000000000C80000008DE100087B
:10D41000000000004508002000000000C8000000D7
:10D420005BE6000800000000320800200000000059
:10D43000C800000083E40008000000003C08002051
:10D4400000000000C800000082E1000800000000A9
:10D450004608002000000000C800000070E6000838
:10D46000000000003308002000000000C800000099
:10D4700098E40008000000003D08002000000000C3
:10D48000C800000097E100080000000047080020E5
:10D4900000000000C80000004FE700080200000084
:10D4A000EA08002000000000D00700000DE400089A
:10D4B00000000000EE080020000000000100000055
:10D4C000CDE5000802000000F00800200A0000007E
:10D4D000D007000071E8000802000000F2080020F8
:10D4E0000A000000D007000074E3000800000000FC
:10D4F000ED08002000000000640000004BE400087C
:10D50000000000002E08002000000000C8000000FD
:10D5100034E400080000000038080020000000008B
:10D52000C80000002CE400080000000042080020B1
:10D5300000000000C80000008AE5000800000000AC
:10D540002D08002000000000C800000075E500085C
:10D55000000000003708002000000000C8000000A4
:10D560006EE50008000000004108002000000000F7
:10D57000C800000054E80008000000002F08002048
:10D5800000000000C80000004EE800080000000095
:10D590003908002000000000C800000048E800082A
:10D5A000000000004308002000000000C800000048
:10D5B00091E7000800000000300800200000000093
:10D5C000C80000008BE70008000000003A080020B7
:10D5D00000000000C800000079E70008000000001B
:10D5E0004408002000000000C80000005CE50008BE
:10D5F000000000003408002000000000C800000007
:10D6000054E50008000000003E0800200000000073
:10D61000C80000004CE50008000000004808002099
:10D6200000000000C800000046E5000800000000FF
:10D630003608002000000000C800000040E5000897
:10D64000000000004008002000000000C8000000AA
:10D650002EE50008000000004A080020000000003D
:10D66000C8000000414552543132333400000000FC
:10D670000000803F00000000A8AAAA3F00000000B0
:10D680000000803F000080BFB0AA2ABF0000000059
:10D690000000803F0000803FB0AA2ABF00000000C9
:10D6A0000000803F000000000000803F000080BFBD
:10D6B0000000803F000080BF000000000000803FAD
:10D6C0000000803F0000803F000000000000803F1D
:10D6D0000000803F00000000000080BF000080BF0D
:10D6E0000000803F000080BF0000803F000080BF3E
:10D6F0000000803F000080BF000080BF0000803F2E
:10D700000000803F0000803F0000803F0000803F1D
:10D710000000803F0000803F000080BF000080BF0D
:10D720000000803F0000803F00000000000000007B
:10D730000000803F000080BF0000000000000000EB
:10D740000000803F00000000A8AAAA3F0000803F20
:10D750000000803F000080BFB0AA2ABF000080BF49
:10D760000000803F0000803FB0AA2ABF000080BFB9
:10D770000000803F00000000A8AAAA3F000080BF70
:10D780000000803F000080BFB0AA2ABF0000803F99
:10D790000000803F0000803FB0AA2ABF0000803F09
:10D7A0000000803FD0B35DBF0000003F0000803F1D
:10D7B0000000803FD0B35DBF000000BF000080BF0D
:10D7C0000000803FD0B35D3F0000003F0000803F7D
:10D7D0000000803FD0B35D3F000000BF000080BF6D
:10D7E0000000803F00000000000080BF0000803F7C
:10D7F0000000803F000000000000803F000080BF6C
:10D800000000803F000000000000803F000080BF5B
:10D810000000803F000080BF000080BF00000000CB
:10D820000000803F000000000000803F0000803FBB
:10D830000000803F0000803F000080BF000000002B
:10D840000000803F000000BFD0B35D3F0000803F7C
:10D850000000803F000000BFD0B35DBF0000803FEC
:10D860000000803F0000003FD0B35D3F000080BF5C
:10D870000000803F0000003FD0B35DBF000080BFCC
:10D880000000803F000080BF00000000000080BF5B
:10D890000000803F0000803F000000000000803F4B
:10D8A0000000803F000080BF0000803F000080BF7C
:10D8B0000000803F000080BF000080BF0000803F6C
:10D8C0000000803F0000803F0000803F0000803F5C
:10D8D0000000803F0000803F000080BF000080BF4C
:10D8E0000000803F000080BF0000803F0000803FBC
:10D8F0000000803F000080BF000080BF000080BFAC
:10D900000000803F0000803F0000803F000080BF9B
:10D910000000803F0000803F000080BF0000803F8B
:10D920000000803FF704353FF70435BF0000803F1B
:10D930000000803FF70435BFF70435BF0000803F8B
:10D940000000803FF70435BFF704353F0000803FFB
:10D950000000803FF704353FF704353F0000803F6B
:10D960000000803F00000000000080BF000080BF7A
:10D970000000803F000080BF00000000000080BF6A
:10D980000000803F000000000000803F000080BFDA
:10D990000000803F0000803F00000000000080BFCA
:10D9A0000000803F0000803F000000BF0000803F7B
:10D9B0000000803F000000BF000080BF0000803FEB
:10D9C0000000803F000080BF0000003F0000803F5B
:10D9D0000000803F0000003F0000803F0000803FCB
:10D9E0000000803F0000003F000080BF000080BFBB
:10D9F0000000803F000080BF000000BF000080BF2B
:10DA00000000803F000000BF0000803F000080BF9A
:10DA10000000803F0000803F0000003F000080BF0A
:10DA20000000803F000000000000803F0000803FB9
:10DA30000000803F000080BF000080BF00000000A9
:10DA40000000803F000000000000803F000080BF19
:10DA50000000803F0000803F000080BF0000008089
:10DA60000000803F000080BF0000803F000080BFBA
:10DA70000000803F000080BF000080BF0000803FAA
:10DA80000000803F0000803F0000803F0000803F9A
:10DA90000000803F0000803F000080BF000080BF8A
:10DAA0000000803F000000000000000000000000B7
:10DAB0000000803F000000000000000000000000A7
:10DAC0000000803F0000000000000000000080BF58
:10DAD0000000803F00000000000000000000803FC8
:10DAE00000000000000000000301000070D60008E4
:10DAF00004000000A0D6000804000000E0D60008E2
:10DB00000201000020D70008000100000000000012
:10DB10000600000040D7000806000000A0D700085B
:10DB200001010000000000000400000000D800080F
:10DB30000600000040D8000808000000A0D8000837
:10DB40000800000020D9000808000000A0D9000843
:10DB500001010000000000000001000000000000C2
:10DB600000010000000000000400000020DA0008AE
:10DB70000600000060DA000800010000000000005C
:10DB800002010000C0DA00080101000000000000EE
:10DB90000000000000000000524F4C4C3B50495424
:10DBA00043483B5941573B414C543B506F733B50AA
:10DBB0006F73523B4E6176523B4C4556454C3B4D44
:10DBC00041473B56454C3B000000000000C20100AD
:10DBD000FBE900081EEA00080100000000E1000067
:10DBE000D9E90008C5E9000802000000009600001D
:10DBF0008FE90008B1E9000803000000004B0000B5
:10DC00006DE9000859E900080400000080250000C3
:10DC1000A9E80008A9E80008B56206010300F005BC
:10DC200000FF19B56206010300F00300FD15B5629F
:10DC300006010300F00100FB11B56206010300F0CC
:10DC40000000FA0FB56206010300F00200FC13B5F4
:10DC50006206010300F00400FE17B562060103002E
:10DC60000102010E47B562060103000103010F49DD
:10DC7000B56206010300010601124FB562060103F9
:10DC8000000112011E67B5620616080003070300B3
:10DC90000000000031E5B56206080600C80001007A
:10DCA0000100DE6A1048494A4B4C4D44454647FF47
:10DCB000202122232425262748494A4B4C4DFF107A
:10DCC00048498A8B8C8D84858687FF2021222324D6
:10DCD00025262748498A8B8C8DFF0000B0DC000880
:10DCE000A4DC0008CBDC0008BFDC0008000C01400D
:10DCF00008001002000C0140100010020008014052
:10DD000000101402B38C00084F8C0008838C0008AC
:10DD1000CF8B0008698C0008178C000800000040B9
:10DD20000008014001000000001C0000000000404D
:10DD30000008014002000000041C00000000004038
:10DD40000008014004000000081C00000000004022
:10DD500000080140080000000C1C00000004004006
:10DD60000008014040000000001D000000040040C9
:10DD70000008014080000000041D00000004004075
:10DD8000000C014001000000081D000000040040DC
:10DD9000000C0140020000000C1D0000002C01409E
:10DDA0000008014000010000001B0100002C0140A0
:10DDB00000080140000800000C1B010000080040A2
:10DDC000000C014040000000001E00000008004060
:10DDD000000C014080000000041E0000000800400C
:10DDE000000C014000010000081E00000008004077
:10DDF000000C0140000200000C1E00000004080C92
:10DE0000879F0008319F0008599F0008A59F0008C0
:10DE1000B19C0008A79F000800000000000000005F
:10DE20000000B33FB2BE7D3A00002E40DFCF513834
:10DE300000007E40BF51FABA00E0A44019DAC3BA2C
:10DE400000E0C840C2ED8AB90040EB40CD1F2CBABB
:10DE5000001006412AFFFABA00C01541DFCFD137C2
:10DE600000D024419A97703A0050334189478E364A
:10DE700000404141E75B9D3800B04E41C00A98B96F
:10DE800000A05B41558F943A00306841DA92C0BAE5
:10DE90000040744162B3C63A0000803F00A0853F55
:10DEA00000908B3F00C0913F0030983F00F09E3FB4
:10DEB00000F0A53F0050AD3F0000B53F0000BD3F62
:10DEC0000060C53F0020CE3F0040D73F00C0E03F8C
:10DED00000C0EA3F0020F53F000000007D36AC396D
:10DEE0007D3C3839EBDCF438320A7E39124C263965
:10DEF0009B6AED39A4EE83397F661E39F6398A397B
:10DF00002B426539A48211395B991F39C3EECD3993
:10DF1000DDE7C637A5A22F390000803FC3AA853FA1
:10DF2000C2958B3FD3C3913FF037983F32F59E3F68
:10DF3000D7FEA53F3F58AD3FF304B53FA408BD3F12
:10DF40002A67C53F8C24CE3FFD44D73FDFCCE03F5E
:10DF5000C7C0EA3F7D25F53F00404040404040407B
:10DF600040404141414141404040404040404040AC
:10DF70004040404040404040400502020202020250
:10DF8000020202020202020202202020202020209F
:10DF900020202002020202020202909090909090B3
:10DFA0001010101010101010101010101010101071
:10DFB00010101010020202020202888888888888E5
:10DFC00008080808080808080808080808080808D1
:10DFD00008080808020202024000000059DF000899
:10DFE000000000006E83F9A22915444ED15727FC8A
:10DFF000C0DD34F5999562DB4190433CAB6351FE43
:10E00000696E64657820283020746F203229004DB5
:10E0100050553630353000424D413238300056547C
:10E0200041494C34005934004144584C3334350094
:10E0300048455836005936004F43544F5838004130
:10E040004343003344004641494C53414645004157
:10E050004952504C414E45004750532B4D414700CB
:10E0600048454C495F39305F444547004C45445F63
:10E0700052494E4700464C59494E475F57494E4713
:10E080000048455836480042490054524900474923
:10E090004D42414C00494E464C494748545F41432C
:10E0A000435F43414C00534F465453455249414C02
:10E0B00000435553544F4D0048454C495F31323071
:10E0C0005F4343504D0050504D00564152494F0060
:10E0D0004241524F004759524F0050504D5F544FEC
:10E0E0005F534552564F005155414450004D4F54D7
:10E0F0004F525F53544F50004F43544F464C41547E
:10E100005000534F4E415200504F5745524D4554C9
:10E1100045520053494E474C45434F5054455200D9
:10E120004455414C434F50544552004750530056BC
:10E1300042415400534552564F5F54494C54004895
:10E1400045583658005155414458005345524941AD
:10E150004C5258004F43544F464C4154580054457C
:10E160004C454D4554525900616C69676E5F61635F
:10E1700063006D69647263006E65757472616C33FF
:10E1800064006770735F706F73725F6400677073B1
:10E190005F706F735F64006770735F6E61765F645A
:10E1A00000666C6170735F737065656400736F66A1
:10E1B0007473657269616C5F315F696E76657274E4
:10E1C000656400736F667473657269616C5F325F5A
:10E1D000696E766572746564007468725F6D6964F7
:10E1E000006D6F726F6E5F7468726573686F6C64D8
:10E1F000006661696C736166655F6465746563740C
:10E200005F7468726573686F6C64006163637879CA
:10E210005F6465616462616E64006163637A5F6418
:10E2200065616462616E64007961776465616462EE
:10E23000616E64006D696E636F6D6D616E64006523
:10E240006D665F61766F6964616E636500766261B9
:10E25000746D696E63656C6C766F6C746167650074
:10E26000766261746D617863656C6C766F6C7461F5
:10E27000676500616C745F686F6C645F666173747E
:10E280005F6368616E676500766261747363616C79
:10E2900065007468726F74746C655F636F72726529
:10E2A0006374696F6E5F616E676C650070726F6634
:10E2B000696C65006465616462616E6433645F7497
:10E2C00068726F74746C65006661696C7361666511
:10E2D0005F7468726F74746C65006D696E746872D7
:10E2E0006F74746C65006D61787468726F74746CAF
:10E2F00065006C6F6F7074696D65004E6F6E6500C0
:10E300006770735F747970650073657269616C72B0
:10E31000785F74797065006163635F6861726477C8
:10E320006172650066656174757265007470615F25
:10E33000726174650072635F7261746500726F6C04
:10E340006C5F70697463685F726174650073657295
:10E35000766F5F70776D5F72617465006D6F746F5B
:10E36000725F70776D5F72617465007961775F725B
:10E37000617465006E61765F736C65775F7261745E
:10E380006500736F667473657269616C5F62617555
:10E390006472617465006770735F62617564726155
:10E3A0007465006765742F736574206D6F746F7288
:10E3B000206F75747075742076616C756500746873
:10E3C000726F74746C655F636F7272656374696F8A
:10E3D0006E5F76616C75650073617665006261726F
:10E3E0006F5F7461625F73697A65006261726F5F0B
:10E3F0006E6F6973655F6C7066006779726F5F6CD2
:10E40000706600616C69676E5F6D6167006E617652
:10E410005F636F6E74726F6C735F68656164696E61
:10E420006700616C69676E5F626F6172645F7069DB
:10E4300074636800695F7069746368006163635F37
:10E440007472696D5F706974636800705F7069747D
:10E4500063680074656C656D657472795F73776964
:10E46000746368006465616462616E6433645F68EC
:10E4700069676800677073706173737468726F7531
:10E480006768006770735F706F73725F69006770B1
:10E49000735F706F735F69006770735F6E61765F43
:10E4A00069006D696E636865636B006D61786368B0
:10E4B00065636B006163635F756E61726D65646354
:10E4C000616C00706173737468726F756768206740
:10E4D000707320746F2073657269616C00616C7475
:10E4E0005F686F6C645F7468726F74746C655F6E84
:10E4F00065757472616C006C697374206F72202D85
:10E5000076616C206F722076616C00706F77657237
:10E510005F6164635F6368616E6E656C00727373E4
:10E52000695F6175785F6368616E6E656C00645FDA
:10E5300076656C006261726F5F63665F76656C0022
:10E54000695F76656C00705F76656C00645F6C6512
:10E5500076656C00695F6C6576656C00705F6C65F4
:10E5600076656C00616C69676E5F626F6172645F93
:10E57000726F6C6C00695F726F6C6C006163635FDB
:10E580007472696D5F726F6C6C00705F726F6C6C2F
:10E590000072657461726465645F61726D007072AF
:10E5A000696E7420636F6E666967757261626C650F
:10E5B0002073657474696E677320696E20612070C2
:10E5C00061737461626C6520666F726D006E617656
:10E5D0005F73706565645F6D696E007665727369FF
:10E5E0006F6E006D61675F6465636C696E6174690D
:10E5F0006F6E006D61785F616E676C655F696E63F9
:10E600006C696E6174696F6E007961775F636F6EBC
:10E6100074726F6C5F646972656374696F6E0079A0
:10E6200061775F646972656374696F6E0072635FBE
:10E630006578706F007468725F6578706F00616CE8
:10E6400069676E5F6779726F007472695F756E617A
:10E65000726D65645F736572766F006770735F706B
:10E660006F73725F70006770735F706F735F7000BD
:10E670006770735F6E61765F70006D6170006865D2
:10E680006C700064756D700074656C656D65747296
:10E69000795F70726F7669646572006D6170706920
:10E6A0006E67206F66207263206368616E6E656CB2
:10E6B000206F72646572007069645F636F6E74725C
:10E6C0006F6C6C6572007265626F6F745F63686116
:10E6D0007261637465720064657369676E20637547
:10E6E00073746F6D206D6978657200666978656412
:10E6F00077696E675F616C74686F6C645F64697280
:10E70000006163635F6C70665F666163746F720063
:10E710006779726F5F636D70665F666163746F7255
:10E72000006779726F5F636D70666D5F66616374B9
:10E730006F72006D6F746F720067696D62616C5FFC
:10E74000666C6167730064656661756C74730067FD
:10E7500070735F77705F7261646975730073686F5F
:10E76000772073797374656D2073746174757300A9
:10E77000736574006578697400645F616C7400622D
:10E7800061726F5F63665F616C7400695F616C7476
:10E7900000705F616C74007470615F627265616BC0
:10E7A000706F696E74007361766520616E642072AB
:10E7B00065626F6F7400726573657420746F206496
:10E7C000656661756C747320616E64207265626F3A
:10E7D0006F740074656C656D657472795F706F72CB
:10E7E00074006D69786572206E616D65206F7220AE
:10E7F0006C697374006E616D653D76616C75652042
:10E800006F7220626C616E6B206F72202A20666FBF
:10E8100072206C69737400666561747572655F6EF1
:10E82000616D6520617578666C6167206F7220622A
:10E830006C616E6B20666F72206C69737400616C22
:10E8400069676E5F626F6172645F79617700695FAB
:10E8500079617700705F79617700646561646261F6
:10E860006E6433645F6C6F77004D4D41383435789A
:10E87000006E61765F73706565645F6D61780063DB
:10E880006D697800617578006661696C73616665B1
:10E890005F64656C6179006661696C736166655F70
:10E8A0006F66665F64656C61790043414D53544106
:10E8B000423B0043414C49423B0047505320484FA4
:10E8C0004C443B0048454144465245453B00414E7F
:10E8D000474C453B0047505320484F4D453B004D6A
:10E8E00041473B0043414D545249473B0048454155
:10E8F0004441444A3B0041524D3B00484F52495A23
:10E900004F4E3B00564152494F3B004241524F3B14
:10E91000004245455045523B00474F5645524E4FE9
:10E92000523B004C4C49474854533B0050415353D1
:10E93000544852553B004C45444C4F573B004F53B5
:10E94000442053573B004C45444D41583B005445EF
:10E950004C454D455452593B0024504D544B323593
:10E96000312C31393230302A32320D0A00245055E0
:10E9700042582C34312C312C303030332C30303064
:10E98000312C31393230302C302A32330D0A002408
:10E99000505542582C34312C312C303030332C30FF
:10E9A0003030312C33383430302C302A32360D0AA6
:10E9B0000024504D544B3235312C33383430302A0A
:10E9C00032370D0A0024504D544B3235312C353737
:10E9D0003630302A32430D0A0024505542582C3428
:10E9E000312C312C303030332C303030312C353725
:10E9F0003630302C302A32440D0A0024505542580B
:10EA00002C34312C312C303030332C303030312C10
:10EA10003131353230302C302A31450D0A00245046
:10EA20004D544B3235312C3131353230302A31466C
:10EA30000D0A000054EA00080000002064040000F1
:10EA400032BB000850EB00086404002014260000CC
:10EA500054BD0008019A0320803FCBDC0502C102AF
:10EA60002F0113B735025C08021A03092EAB0111FE
:10EA70004BF6E8BC29491ACE0C290832021AFB0CC5
:10EA80002908297C130BE92A08082A0404190C29EF
:10EA90000832051ADF24290832061AC40C29083264
:10EAA000071AED0C290829591AAA0C290832091A43
:10EAB000E40C2908320A1AD50C2908320B1ABA0CB0
:10EAC0002908320C1A2C602908320D1A110C290859
:10EAD000320E1A460C2908320F1A360C2908321049
:10EAE0001A230C290832111AB348290832121A19AC
:10EAF00018290832131A3E0C290832141A4E0C2910
:10EB00000872150225FF0378803F022201021004DB
:10EB10007A03B4690401167A035D4AD933091021D6
:10EB200012010A1C029DC208342C01401A40921A9C
:10EB30004019290C89C414A24A048B127A3B380B61
:10EB4000020304060708090204064329106914C1D8
:04000005080000ED02
:00000001FF
